:020000021000EC
:10F000000000012039F5010061F5010063F5010000
:10F0100065F5010067F5010069F5010000000000D9
:10F020000000000000000000000000006BF501007F
:10F030006DF50100000000006FF50100ADA10300B7
:10F04000114A020073F501004D4D0200714A0200A1
:10F05000C54A020073F50100B94E020073F50100C4
:10F0600073F50100F1A1030073F5010073F50100D0
:10F0700073F50100DD57020073F5010073F501001F
:10F08000EDA10300D925020073F5010073F501001D
:10F09000E1260200D5E10300D516020073F5010058
:10F0A00073F5010073F5010073F5010073F50100BC
:10F0B00073F5010073F5010000000000000000007E
:10F0C00073F5010073F5010073F5010073F501009C
:10F0D00073F50100A959020073F50100000000005A
:10F0E0000000000000000000000000000000000020
:10F0F0000000000000000000000000000000000010
:10F1000000000000000000000000000000000000FF
:10F1100000000000000000000000000000000000EF
:10F4000010B5054C237833B9044B13B10448AFF35E
:10F4100000800123237010BD302D0020000000006B
:10F42000E0B5050008B5034B1BB103490348AFF332
:10F43000008008BD00000000342D0020E0B505006C
:10F44000154B002B08BF134B9D46A3F5803A0021B6
:10F450008B460F461348144A121A00F063F80F4BFC
:10F46000002B00D098470E4B002B00D0984700206F
:10F47000002104000D000D48002802D00C48AFF315
:10F48000008000F02BF8200029001CF049F800F063
:10F4900011F800BF0000080000000120000000007B
:10F4A00000000000302D0020F0CD00200000000002
:10F4B0000000000008B5074B044613B10021AFF36C
:10F4C0000080054B1868836A03B19847204600F016
:10F4D00031F800BF00000000D037050070B50D4DB9
:10F4E0000D4C641BA4100026A64209D10B4D0C4CF8
:10F4F00034F062F9641BA4100026A64205D170BD49
:10F5000055F8043B98470136EEE755F8043B984719
:10F510000136F2E7182D0020182D0020182D0020AC
:10F520001C2D002002440346934200D1704703F88B
:10F53000011BF9E7FEE700BF0649074A074B9B1A84
:10F5400003DD043BC858D050FBDC06F01BFBFFF783
:10F5500077FF0000ECB50500402C0020302D002086
:10F56000FEE7FEE7FEE7FEE7FEE7FEE7FEE7FEE773
:10F57000FEE7FEE71FB501238DF80030054B8DF83F
:10F58000080001916846D3E90012904705B05DF884
:10F5900004FB00BFC4BA002061DF704748DF70473A
:10F5A00010B50388012B11D8094A02EB03124388D6
:10F5B0005189CC1A032C09D4C3F57F43FD330B4486
:10F5C0005381002303804380184610BD0420FCE7CC
:10F5D00098BE002010B5124A0B6802EB001042687A
:10F5E00073B15888033003EB800302F580524FF665
:10F5F000FF749A4202D91868013004D1002009E052
:10F6000002F10803F1E79888A04204D0188810B1ED
:10F610000B60012010BD5888033003EB8003E8E73E
:10F6200098BE002073B5436804460D4613B31E4AC6
:10F6300011688B421ED3526893421BD813F003000B
:10F6400018D11A4A21891289914213D121689A68E6
:10F6500091420FD1164A5268934201D80A2004E021
:10F6600002F580529342F9D22880B0FA80F0400926
:10F6700002B070BD00232B801E46019601A9288888
:10F68000FFF7A8FF30B92B8801339BB22B80002BEA
:10F69000F3D0EDE7019B226899689142EED1636057
:10F6A000024B1B892381E3E7202D002080BC002032
:10F6B00098BE0020033083B240F2FD32934230B551
:10F6C0000ED909200BE0228965892A441A4492B296
:10F6D000B2F5806F08D2088062891344638130BD1F
:10F6E000024C20780028EED00720F8E798BE0020D2
:10F6F00010B50A494A788C78531CDBB29C4208BF8B
:10F7000000230C789C421FBF0370486802EB420242
:10F7100000EBC20008BF002010BD00BF14BE0020D7
:10F72000AADF7047A9DF7047A7DF704785DF704702
:10F730007FDF70477EDF7047084A30B500230C2416
:10F7400004FB03F18D5A854202D10A44508830BD32
:10F750000133082BF4D14FF6FF70F8E7EABB002025
:10F760006EDF704758B1CB0801F00701C25C01237E
:10F7700003FA01F10A4214BF184600207047012025
:10F780007047000070B50A4E3468054654B1706881
:10F7900060B1FF2D08D02946FFF7E4FF30B1F368D0
:10F7A00003FB0544204670BD0024FBE70446F9E74F
:10F7B0001CC00020012804D0043804288CBF00207D
:10F7C000012070478378013B072B07D8DFE803F05F
:10F7D0000706060606070409142303807047012361
:10F7E000FBE743689B8809339B08F6E770B5054D36
:10F7F0000646002455F8043B304601349847052C52
:10F80000F8D170BDFC390500114BF0B5002214266B
:10F810001D4606FB02F4E75A874212D12344142600
:10F8200000249A788A420AD001342246072A0BD84B
:10F8300006FB02F3EF5A874208D1EB18F1D11846C4
:10F84000F0BD0132082AE4D10023F8E70132EDE7E8
:10F850002CC0002030B5072185B0FFF7D5FF044646
:10F8600000283AD04568002D39D1007CFFF78AFF87
:10F870000721CDE902558DF80A1040B3E3680390E3
:10F8800003EB83031B019BB29B0802A8ADF8083071
:10F89000FFF798FF9DF80A00FFF78CFFD8B1114BD6
:10F8A0001B789B0715D5BDF808500DF106012846B9
:10F8B000FFF700FF48B9BDF80630A380E5800A4B8A
:10F8C000185C092803D005B030BD0928F7D90320FA
:10F8D000F9E70220F3E70846F5E70520F3E7002003
:10F8E000F1E700BF7CBC0020EC37050038B54FF6CF
:10F8F000FF73984218BF01300D4614BF84B2002434
:10F90000FF2C03D94FF6FF74204638BD2146284608
:10F91000FFF728FF0028F7D10134A4B2F0E7000078
:10F92000F8B5074D074E074600243378A34200DCA4
:10F93000F8BD55F8043B384698470134F5E700BF59
:10F940005CBC00200DBE00207DDF704779DF704772
:10F950006DDF704738B5074C051E04F1080318BF6A
:10F960001C4623682BB11A6822605B6828469847BA
:10F97000F7E738BD9CBB002037B5D0F818350A7DB5
:10F98000DBB28DF807300B7F9A4282BF0A699DF87F
:10F990000740D4540B7F0D7B0133DBB25A1C9542D8
:10F9A0000B7705D98B689B5CC0F81C3501200AE0F9
:10F9B0000C7D944201D9CB7EF6E7AB42F6D3A3424D
:10F9C0002CBF0020012003B030BD0023435082B083
:10F9D00043580193019B02B070472DE9F0470D7821
:10F9E0009DF820609DF824A004460F469946002DFE
:10F9F00060D1D0F8243192F800809BB14FF492711D
:10FA0000FFF7E3FF012363613B70B04550D1D4F8A9
:10FA10000431002B4CD04FF482712046FFF7D5FF04
:10FA200000251DE0D0F81C31FBB14FF48E71FFF7BB
:10FA3000CCFFD0F824311BB14FF492712046DFE7A0
:10FA400013789E4207D919F80330C0F81C35137893
:10FA500001331370D9E70123BAF1000F03D0C3615A
:10FA60002846BDE8F0874361CFE7D0F80831002B86
:10FA7000CBD04FF48471FFF7A8FFD0F82431002BCE
:10FA8000DAD113789E42C0D9D0F8181509F80310BE
:10FA900013780133DBB21370721E934205D1022337
:10FAA000C0F8003201232362AFE79E42FAD1ACE7EF
:10FAB0000125D5E74FF49271FFF787FF4FF48E7160
:10FAC000FFF783FF4FF48471FFF77FFF9FE72DE976
:10FAD000F3470C4605464FF4827120461F46904678
:10FAE000FFF773FF4FF49271FFF76FFF4FF48E71C2
:10FAF000FFF76BFF4FF48471FFF767FF0023012FBF
:10FB000085F8263085F8233008BF02224FF0010324
:10FB10000CBFC4F80022C4F80032236223602E68B0
:10FB200046BB05F1260A05F12309CDE900764346D7
:10FB3000524649462046FFF750FF0028F5D195F878
:10FB40002330EBB1D4F8C434C4F8C434C3B113F0D7
:10FB5000010F14BF4FF40240032048F2012213F0BA
:10FB6000020F18BF104613F0040F48F2022318BF0B
:10FB7000184606E040F28623AB60AB68C4F8043355
:10FB8000002002B0BDE8F0872DE9F3470C4605469A
:10FB90004FF4827120461F4616469DF82880FFF7D5
:10FBA00014FF4FF49271FFF710FF4FF48E71FFF7BF
:10FBB0000CFF4FF48471FFF708FF0023C4F80032F4
:10FBC00085F8263085F8233001232362A36095F859
:10FBD0002620974232D9B35CC4F81C3595F82630FC
:10FBE000013385F826302B687BBB05F1260A05F129
:10FBF0002309CDE900783346524649462046FFF7AF
:10FC0000ECFE0028F5D195F8233023B3D4F8C434A2
:10FC1000C4F8C434FBB113F0010F14BF4FF4024019
:10FC2000032048F2012213F0020F18BF104613F010
:10FC3000040F48F2022318BF18460DE0B8F1000F78
:10FC400001D0E361CFE76361CDE740F28623AB608B
:10FC5000AB68C4F80433002002B0BDE8F0872DE99A
:10FC6000F04793F9005090B00024013D6E46AD007E
:10FC70002746A446A0465FF0000E03E05FEA080EA8
:10FC8000BEEB050EB8EB0E0952F809A051F80E9024
:10FC9000A9FB0A9A14EB090457EB0A075CF1000C64
:10FCA0001EF1040EAE4501DCC645EBDD46F808400A
:10FCB0003C4667465FF0000C18F10408A845DADD01
:10FCC000B8EB450FDADD46F80840D3F8B0303146DE
:10FCD000984710B0BDE8F08713460A46FFF7BFBF4C
:10FCE000F0B5154689B01C4607460E461A46294609
:10FCF0006846FFF7F1FF23466A4639463846FFF764
:10FD0000AEFF23462A4669466846FFF7A8FF23460A
:10FD10006A4631463046FFF7A2FF09B0F0BD00EB5E
:10FD200081010023884200D3704751F8042D43EA33
:10FD300052030B60D307F5E710B5013A52B2130630
:10FD400001D5002010BD50F8224051F822309C42CD
:10FD500005D802F1FF32F2D24FF0FF30F2E7012076
:10FD6000F0E710B500235CB2A24200DC10BD51F8F0
:10FD7000234040F823400133F5E7013910B549B27B
:10FD8000041D0A06CBB204D4013954F82120002AFC
:10FD9000F7D001335BB273B103F18042013A50F8FE
:10FDA0002220002022B9013B00EB431318B210BD02
:10FDB00052080130F6E71846F9E7002310B51C4653
:10FDC0005AB2914200DC10BD40F823400133F7E7FE
:10FDD000C3F10803DB0070B50133002403A500BFA5
:10FDE0005B1920C940CAAD1B20C0184720C940CAB2
:10FDF000B54120C020C940CAB54120C020C940CA71
:10FE0000B54120C020C940CAB54120C020C940CA60
:10FE1000B54120C020C940CAB54120C020C940CA50
:10FE2000B54120C06441B4FA84F0400970BD00BF00
:10FE3000C3F10803DB0070B50133002403A500BF44
:10FE40005B1920C940CAAD1920C0184720C940CA53
:10FE5000754120C020C940CA754120C020C940CA90
:10FE6000754120C020C940CA754120C020C940CA80
:10FE7000754120C020C940CA754120C020C940CA70
:10FE8000754120C06441204670BD00BFF0B5082216
:10FE900089B00C460646FFF764FFCB6A03930B6BF1
:10FEA00004934B6B05938B6B0693CB6B07930027E7
:10FEB00008236A4669466846CDE901770097FFF74F
:10FEC000B7FF082305466A4631463046FFF7B0FFC4
:10FED000236B0393636B0493A36B0593E36B05445C
:10FEE000CDE906376A46082369466846FFF7A0FF52
:10FEF000082305446A4631463046FFF799FF236AD6
:10FF00000093636A0193A36A0293A36B0693E36B66
:10FF10000793054408236A4631463046CDE9047705
:10FF20000397FFF785FF636A0093A36AA26B0193AF
:10FF3000E36A02930492636BE26B0393CDE90523BA
:10FF4000236A0793054408236A4631463046FFF783
:10FF50006FFFE36A0093236B0193636B0293236A41
:10FF60000693A36A0793054408236A463146304640
:10FF7000CDE904770397FFF72BFF236B0093636BA7
:10FF80000193A36B0293E36B0393636A0693E36AA3
:10FF900007932D1A08236A4631463046CDE9047787
:10FFA000FFF716FF636B0093A36B0193E36B029360
:10FFB000236A0393636A0493A36ACDE90537236B2D
:10FFC00007932D1A08236A4631463046FFF700FF93
:10FFD000A36B0093E36BCDE90137636A0393A36AD4
:10FFE0000493E36ACDE90537636B07932D1A082361
:10FFF0006A4631463046FFF7EBFE2D1A0D4C0FD402
:020000022000DC
:1000000035B9082231462046FFF796FE01280FD069
:100010000823224631463046FFF7DAFE2D1AEFE775
:100020000823224631463046FFF702FF2D18F7D449
:1000300009B0F0BDFC3705002DE9F04391B00F4643
:100040001C220021804609A8FFF76CFA01251C221A
:10005000002101A80895FFF765FA394608AA11F9A9
:10006000046B009533461046FFF7E2FE314608A8C0
:10007000FFF783FE013804B2012C07DC32466946E3
:100080004046FFF76EFE11B0BDE8F0833A46684681
:100090006946FFF721FE10AB601103EB80001FFAE9
:1000A00084F909F01F0350F8202C05FA03F31342DA
:1000B00005D03B46424669466846FFF7D0FD09F148
:1000C000FF3424B2D8E770B5036813F00105064683
:1000D000144605D013460A460146FFF7A9FE054619
:1000E00021463046FFF71BFE45B104F18042013A3C
:1000F00056F8223043F0004346F8223070BD70B508
:100100009DF910401E4623460546FFF761FE38B1B3
:100110002346324629462846BDE87040FFF788BE90
:1001200070BD2DE9F0438BB01446129D15F9046B98
:1001300000961F46804689462B460246214602A865
:10014000FFF7DDFF02A9129A0846FFF7C5FD129BD3
:1001500002AA41464046FFF782FD129B02AA2146B1
:100160002046FFF77CFD2B464A4639463846009626
:10017000FFF7C5FF129A394602A8FFF7ADFD02A9A5
:100180002B46424608460096FFF7B9FF02A92B46C8
:10019000224608460096FFF7B2FF2B46424621460C
:1001A00020460096FFF7ABFF129B22464946484681
:1001B000FFF755FD2B4602AA414620460096FFF761
:1001C0009EFF129B224639463846FFF748FD2B46D4
:1001D0004A46394638460096FFF791FF324602A953
:1001E0002046FFF7BEFD0BB0BDE8F08370B59DF96A
:1001F00010401E4623460546FFF71AFE30B9224638
:1002000029463046FFF798FD012807D0234632469D
:1002100029462846BDE87040FFF7DABD70BD2DE9DC
:10022000F0439BB01646229C14F9045B0095984657
:100230000746894623460246314612A8FFF75FFF6C
:1002400012A9229A0846FFF747FD229B12AA3946B7
:100250003846FFF704FD229B12AA31463046FFF7CD
:10026000FEFC23464A46414612A80095FFF7BEFF12
:1002700023464A46414640460095FFF740FF234645
:100280003A4631460AA80095FFF739FF229B0AAA91
:1002900049464846FFF7E3FC2346324639460AA85A
:1002A0000095FFF7A3FF229A41463046FFF714FD61
:1002B00023460AAA314630460095FFF720FF234621
:1002C0003246394602A80095FFF719FF229B02AA81
:1002D00041464046FFF7C3FC23464A464146404656
:1002E0000095FFF70CFF229A12A902A8FFF7F4FC71
:1002F00002A923460AAA08460095FFF700FF2346F5
:100300003A4602A90AA80095FFF7F9FE0AA9229B1E
:1003100012AA0846FFF7A3FC23464A460AA9484604
:100320000095FFF7ECFE2A4602A93846FFF719FDB3
:100330001BB0BDE8F0832DE9F04115468AB00446B4
:1003400088461C22002103A8FFF7ECF82E1D95F922
:10035000007003232A46414620460293FFF7BCFC67
:10036000334602AA214620460097FFF7C8FE2B46D7
:10037000424621462046FFF772FC0097334605F1BE
:10038000840221462046FFF731FF0AB0BDE8F08124
:100390000C4B1B78062B10D10B4B1B681A070CD18A
:1003A0000A4B186800F0F003302B08D000F0E00092
:1003B000A0F1400358425841704700207047012087
:1003C000704700BFE00F00F0E40F00F0E80F00F00E
:1003D000094B1B78062B0CD1084B1B681A0708D158
:1003E000074B186800F0F000A0F130035842584164
:1003F00070470020704700BFE00F00F0E40F00F0EE
:10040000E80F00F010B50C494A6E042A044611D0DA
:100410000B6E1344032B02F101024A6688BF043BB2
:10042000182202FB031318460021FFF77BF8206017
:10043000012010BD0020FCE738BF002010B50446A5
:1004400086B01422002101A8FFF76CF86088ADF88F
:100450000800FFF771F92378ADF80600092B0CD8D6
:10046000DFE803F005051014161B1D0E1F210723DE
:100470008DF8043008238DF80C3001A8FFF750FAEE
:1004800006B010BD0D238DF80430F6E70E23FAE711
:1004900007238DF804300523EDE70F23F3E710233E
:1004A000F1E70523EFE706238DF80430A3680393F3
:1004B000A388ADF80630E0E708B5134644F2010220
:1004C000904203BF5A6819889868002218F0AAFE63
:1004D00030B50B4B1B68012293F8641021338A421C
:1004E00004DB405CB0FA80F0400930BD13F8014BEA
:1004F000855CA54201D10132F1E70020F5E700BF9C
:1005000018BA002070B5244B0022C3F80025234AF6
:10051000516831B12249C3F8081322490420C1F8B7
:100520008000D3F80C55D3F81445D3F80815D3F848
:1005300010054FF0FF36B542C3F8146518BF05F536
:10054000E075C3F80C65C3F80865C3F810651EBFF5
:100550004FF0A043022643F82560651C1FBF4FF0F3
:10056000A04304F5E074022543F82450441C1FBF47
:1005700000F5E0704FF0A043022443F820404B1CEC
:100580001FBF4FF0A04301F5E071022043F82100A6
:100590000023D376536070BD00200040C4BA002011
:1005A0008402020000E100E02DE9F04F85B08A46A8
:1005B0000390039C2578284626F0FEF80746D8B914
:1005C0002D2D1CD10134012303940193DDF80CB0CF
:1005D000BAF1000F01D0CAF800B00022114603A8FA
:1005E00026F092F88046002835D1614D002420463F
:1005F000294605B0BDE8F08F01340394D9E72B2DCF
:1006000004BF013403940190E0E71846029326F0FA
:1006100066F8B0F10009029B20DBC8451EDD4046AC
:1006200032F00AFB22462B4632F070FB04460D46A0
:10063000484632F001FB22462B4632F0B1F9013632
:1006400004460D460396039E3378002BDDD1B8F1A6
:100650000A0F37D113E000240025F4E7B8F10A0FA0
:1006600030D12E2B0BD10FF20019D9E900890136B8
:100670000396039E30783038C3B2092B39D9039BD7
:100680001A7802F0DF02452A1CD15A1C03925A78CC
:100690002D2A01D02B2A05D12D3A574203F102030E
:1006A000574103934FF000080A20039A1378303B18
:1006B000D9B2092936D9002F39D12E4F0026B8F1E9
:1006C000000F46D1039BBAF1000F01D0CAF80030E9
:1006D0009B458AD09BF800202E2A03D10BF1010BF9
:1006E0005B4582D0019B002B81D005F100431D4664
:1006F0007DE732F0A1FA42464B4632F007FB024654
:100700000B462046294632F04BF9002204460D469E
:1007100040464946174B32F023FC01368046894655
:100720000396A6E7013200FB08380392BDE7114F9C
:10073000C8F100080026B8F1000FC3D020462946B2
:1007400032463B4632F00CFC08F1010804460D46E7
:10075000F1E72046294632463B4632F0D7FA08F107
:10076000FF3804460D46AAE79A9999999999B93F95
:100770000000F87F0000244070B58AB00C460146A6
:1007800068461D4626F050FD0022214605A826F0A9
:100790004BFD684626F03BFC044605A826F037FCD6
:1007A0008442064621D0039850B1C389A3F5007353
:1007B0009BB2C381C38903F4F0530BB92BF09AFDAC
:1007C000089850B1C389A3F500739BB2C381C38954
:1007D00003F4F0530BB92BF08DFD002C01DB002E40
:1007E00000DAF5B9A01B0AB070BD002C1BDA039823
:1007F00050B1C389A3F500739BB2C381C38903F4CD
:10080000F0530BB92BF076FD089850B1C389A3F5CE
:1008100000739BB2C381C48914F4F05401D12BF04E
:1008200069FD0020DFE7684626F082F905A826F07A
:100830007FF9AEE7044A138A9BB223F0410343F0E9
:1008400040031382704700BF582D002010B586B0BA
:1008500000220C46014601A826F0E6FC01A826F07D
:1008600039F901A8217826F0E7F8049850B1C38936
:10087000A3F500739BB2C381C38903F4F0530BB992
:100880002BF038FD06B010BD30B587B00A460146E2
:1008900001A826F0C9FC0025DDE90132934205F1EB
:1008A000010401D2013514D1049850B1C389A3F5D4
:1008B00000739BB2C381C38903F4F0530BB92BF0CF
:1008C00019FD202021F056FC14F1FF340DD207B0A1
:1008D00030BD059810B1C05C0A28E5D021F04AFC73
:1008E00001A8254626F024F9D6E70820EAE730B526
:1008F00087B00D46019009B100230B600021102242
:1009000002A8FEF70FFE02A901982EF041FCE0B10B
:100910000024029B039A23F07F43033323F0030355
:10092000013203F110030AD11C44002202A901A8DC
:100930002EF068FC0028ECD1204607B030BD002D19
:10094000F3D02A6813442B60EFE70446F4E730B590
:1009500087B04FF4D8240021102202A80194FEF79A
:10096000E1FD02A920462EF013FC70B1002202A97D
:1009700001A8DDE901542EF045FC0028F6D124F051
:100980007F4413352C4424F00304C4F5EC2007B055
:1009900030BD2DE9F04F89B0D51C019325F003053A
:1009A000002382468B46174610350393984604ACC5
:1009B000039E86B330462EF0EFFB804603982EF060
:1009C00011FC064678B1039BC21A95420BD9FB1A5B
:1009D0000344984507D9B5F5007F04D221462EF08F
:1009E000D7FB00B90396019B039947EA03671022DE
:1009F0004FF0FF33204605930497CDE906AB18F07E
:100A0000E3FC129B23B194E80F00129C84E80F00D2
:100A1000039E103638E04FF4D8230393B1462146A5
:100A200003982EF0B5FB78B1059B013306D1DDE9C3
:100A300006235B4504BF5245DDF80C900122214698
:100A400003A82EF0DFFBEEE703982EF0A5FB85420E
:100A50001ED903982EF0C6FB012303900398C8B952
:100A6000B9F1000F0BD0214648462EF091FB04222D
:100A7000002309EB020105A8059318F0A5FC0398D3
:100A800078B9B8F1000F11D0304609B0BDE8F08F49
:100A90000023E3E7002BC2D12EF07EFB8542BED8B7
:100AA000DEE72EF079FB8742EBD881E72EF0D0FC11
:100AB00080460028E8D00023039379E72DE9F04F22
:100AC0008DB002AFB3F10009C7E9020192463E6D55
:100AD0004FF0000519DBAE4217DB07F1100110469D
:100AE0003D612CF03CF9804600BB504628F084FF65
:100AF0000446386125F09EFC04F58073834209D9D1
:100B00005A49012026F084FF002528462C37BD468F
:100B1000BDE8F08FE31D23F00703ADEB030D0DF1EE
:100B2000080822464146504628F056FF06B93E695D
:100B300007F1180B5A46D7E902012EF08EFB044646
:100B400020B9B9F1000F2FD04949DAE7B9F1000F08
:100B500035D1BB691A0E05D1B34203D131462EF00F
:100B6000D5FB60BBBD6925F07F439E421CD12D0E95
:100B70001AD1D7F810A0564516D1331F10E062598C
:100B80007A619D428CBFAAEB0502042208EB0501A5
:100B900007F114007B6032F0BFFD28B97B68043593
:100BA000AA45ECD80125B0E7CDF800B000233246C5
:100BB000D7E90201FFF7EDFE04460028C4D03969E9
:100BC000BB6909EB010223F07F439A4201D929490D
:100BD00097E74C4420462EF099FB054620B926495C
:100BE000012026F015FF90E714F003001FD0A4EBBE
:100BF0000009C0F10406D9F800307B613B699E42D0
:100C000028BF1E4607F1140318443246414632F00D
:100C100091FD0422494607F1140018F0D5FB3B6909
:100C2000B3427FF672AFB04434449E1B3E613A69D2
:100C300002F00306921B3A611AB12146404618F0B1
:100C4000C3FB002E3FF461AF39690C443246236880
:100C50007B61414407F1140032F06CFD042221460F
:100C600007F1140018F0B0FB4FE700BFB9380500DA
:100C7000E0380500FE3805001A3905000C4A00234B
:100C800030B41146184640F6CA0401EB0315103281
:100C9000E8819D1C0133A34222F80C5CF5D148F693
:100CA00094430122C852034B1A8030BC2BF0CCB9BC
:100CB000742D0020722D0020F8B5858907460C465A
:100CC00095B31A4B013D03EB05152846EB8903F557
:100CD00000739BB2EB812CF083FDEB89A3F50073CD
:100CE0009BB2EB81EB8903F4F053461C13B9284601
:100CF0002BF000FB30462AF007FF21462CF08CF940
:100D0000044680B1014638462CF054FEE389A3F531
:100D100000739BB2E381E38903F4F05313B92046D7
:100D20002BF0E8FA701CF8BD0126E3E7742D0020D3
:100D300038B5074C25780023EDB2024619462370DA
:100D400029F0E6FA25700348BDE8384020F0CCB918
:100D5000702D002004A7050070B504462BF0AEFAF4
:100D60000546B0B12046002218492DF069F8044626
:100D70002BF0EBF878B900255CB1E389A3F500739B
:100D80009BB2E381E38903F4F05313B920462BF0BF
:100D9000B1FA284670BD00220D4920462DF050F8CA
:100DA00006460028E7D00B4922F07CF8F389A3F52A
:100DB00000739BB2F381F38903F4F0530546002BD3
:100DC000DAD130462BF096FAD6E700BFAA390500F3
:100DD000316E0500B4390500002370B50B6005467F
:100DE0000E462AF007FF044610B90025284670BDBC
:100DF00029462BF0EDFF054668B9E389A3F500739A
:100E00009BB2E381E38903F4F053002BEDD120463C
:100E10002BF070FAEAE720462BF0E1F83060E38926
:100E2000A3F500739BB2E381E38903F4F053002B35
:100E3000DCD1ECE738B5002205462DF001F8044678
:100E400098B100231A460146284622F069FEE3893C
:100E5000A3F500739BB2E381E38903F4F05323B954
:100E60002046BDE838402BF045BA38BDF7B5002222
:100E70000191314907462CF03DFF044600B301467D
:100E800001AB0122384622F04BFE58B92B4826F020
:100E90007DFC2B4A28491378384643F0040313702D
:100EA0002DF006FCE389A3F500739BB2E381E3898F
:100EB00003F4F05313B920462BF01CFA012637E057
:100EC0000246204938462CF0BBFF05462BF0F0F8CF
:100ED000064628B9019A1B4938462CF057FFEDE722
:100EE00028462BF0DFFE074601982BF0DBFE384446
:100EF000B0F5007F05D9124A137843F0020313704E
:100F00002646B7F5007F06D2C7F500730022019987
:100F100028462BF07CFD5DB1EB89A3F500739BB2F5
:100F2000EB81EB8903F4F05313B928462BF0E2F977
:100F3000304603B0F0BD00BFBB390500C339050022
:100F4000712D0020F739050070B5EFF3108672B6E9
:100F50000D4A94680123A4B993600C4B0C4DD3F84F
:100F6000801029401160C3F88050D3F8841051607C
:100F70004FF0FF32C3F88420047006B962B6002037
:100F800070BD0370F9E700BFD4C0002000E100E0AD
:100F9000FC06FFBC10B588B012788DF80C20CDE9A6
:100FA0000001FF22002102918DF80D2001214FF652
:100FB000FF72104C8DF81C10ADF80E208DF810301B
:100FC0001FF060FC70B125F02DFA58B914F1FF3410
:100FD000F6D20949042026F01BFD68461FF062FC8A
:100FE00008B010BD002CF4D025F01CFA0028F0D178
:100FF000F3E700BF80841E00913905002DE9F3411D
:10100000314C637E0546002B5BD123680BB1012375
:10101000637695E80F002D4E86E80F00A27E637F71
:101020002B4E23F00303FF2A63771EBF0123934057
:101030004FF0A0424FF0000118BFC2F80C35254B0D
:1010400021770422C3F808233160316800910099A8
:10105000297939B32A681278C3F81C252A79012A1C
:1010600022D92A685278C3F81C2525680DBB194F70
:10107000DFF85480D7F80831002BFBD03560336897
:10108000019341463846019BFEF776FC0028F1D1DA
:10109000A27EFF2A12D0012393404FF0A042C2F853
:1010A00008350BE0E27ED7E72A7B012ADDD9E27E14
:1010B000D9E7084B0422C3F80423002002B0BDE89E
:1010C000F0811120FAE700BF08BB002010BB002010
:1010D000083100400030004037B50B015BB249B227
:1010E000044643EA01008DF804001A4D50B2034350
:1010F000120152B28DF805302B78114302438DF85E
:1011000006108DF8072013B302AB03EB941302AA69
:1011100013F8040CC4F30113134413F8043C43EA1A
:10112000002018F0C1F82B788BB102AAC4F3810318
:1011300004F003041344144413F8040C14F8043C9E
:1011400043EA002003B0BDE8304018F0ADB803B06A
:1011500030BD00BFE2C00020C30914BF13020B0260
:1011600070B510F0400F0D460CBF294611461943CB
:1011700006461220144618F01DFAB1064CBF230291
:101180002B0216F0100F14BF2146294619431220D6
:1011900018F010FA32074CBF23022B0216F0040F8E
:1011A00014BF214629461943122018F003FAB30749
:1011B0004CBF2102290216F0010F08BF2C46214323
:1011C0001220BDE8704018F0F5B9000010B5074ACC
:1011D000002332F8024B8C4203D1184100F0010089
:1011E00010BD0133082BF4D10020F9E720BA00200C
:1011F000F0B5224B9F7C1C4600221D46D6B2B7425A
:101200000ED895F878701D4C0022D6B2B74216D889
:1012100095F8DE500022D4B2A54220D800200DE07F
:10122000B4F814C0844502F1010204F10A04E5D1C6
:1012300042F64D2301200B808870CE70F0BDB4F8CB
:101240007AC0604502F1010204F10A04DDD142F6E0
:101250004D230B8002238B70CE700120EEE7B3F894
:10126000E060B04202F1010203F10A03D3D142F679
:101270004D230B8003238B70CC70EEE78CBC0020D9
:1012800010B50C4C226886B0034682B104208DF85C
:1012900004000868D989ADF80C10123333F8021C29
:1012A0000290ADF80E10049301A92046904706B0B5
:1012B00010BD00BF8CBC00207FB54B89022B0FD125
:1012C000094A136863B1097B0068029011F0010FAD
:1012D00014BF022103218DF80410104601A998477C
:1012E00007B05DF804FB00BF8CBC002070B50D4D4D
:1012F000002435F8026B964210D10122A240D2B2EE
:10130000D543EDB2014410F8014B2BB11443884290
:1013100000F8014CF7D170BD2C40F8E70134082CDF
:10132000E7D1F8E720BA002070B50023084C1A4630
:1013300041FA02F5ED0706D504EB420600EB430542
:10134000B688AE8001330132082AF1D1036070BD46
:101350001CBA002010B586B004460022684614F07E
:10136000CFFB2046009914F0F9FC204606B010BDD2
:1013700038B501230B7004460D462AF0E6FD88B10E
:1013800000220B4920462CF05BFD10B12DF025FA10
:1013900028702046002207492CF052FDBDE8384055
:1013A0002DF0B4B82046BDE838402CF019BA00BF83
:1013B000AC380500B1380500084B5A6E013A5A6640
:1013C00022B907490A7822F002020A701A6E013225
:1013D000042A08BF00221A66704700BF38BF0020E9
:1013E0007DBC002030B5044685B00D46102200219A
:1013F0006846FEF797F8237A012B0AD0022B0ED00D
:1014000063680193236829469B686846984705B03E
:1014100030BD23690293A38AADF80C30F0E70123B5
:10142000A2898DF80030E389ADF80A20D31AADF80F
:101430000830E5E728DF704729DF704738B51C4BD7
:101440005A6E19465AB31C6E182202FB04331A7ADC
:10145000012A07D0022A23D018460921BDE83840C6
:10146000FFF7C0BF1825D88A9A8A05FB0414D4E96F
:101470000314121AB2F5806F4FEA80000144B4BF22
:1014800092B24FF480622044FFF7D6FF11280BD1AF
:10149000084A137823F0020343F00403137038BDA5
:1014A0009889FFF7C7FFF1E70028F8D0D4E700BF1D
:1014B00038BF00207DBC0020054A137813F0060FCA
:1014C00004D143F002031370FFF7B8BF704700BFA9
:1014D0007DBC00202DE9F3411F4B1B781746DA072E
:1014E000064688462BD51D4D1D4B9D4229D31D4BCD
:1014F0009D4226D239B330B341EA00039B0724D181
:101500002B68984223D36A6800EB87039A421ED364
:10151000FFB101A8FEF776FF78B1019B0024C3E973
:101520000054019B01221A72C3E903869F82FFF7D0
:10153000C3FF204602B0BDE8F0810720FAE7012092
:10154000F8E70220F6E70320F4E70620F2E705209B
:10155000F0E70420EEE700BF7DBC0020202D002036
:10156000202D0020302D002038B5074B074A596840
:10157000948810684A880332032592B200EB8400F5
:101580001D70FFF7A7FF38BD80BC0020DCBF002026
:1015900010B501220C460649FFF79CFF28B9054902
:1015A00001EB041101238B7310BD0E20FCE700BF7B
:1015B000103A050098BE002008B502220149FFF745
:1015C00089FF08BD143A050008B5034B03491868A4
:1015D0000222FFF77FFF08BDDCBF00201C3A050098
:1015E00073B51B4B1B78DB0705462BD5194E1A4BE1
:1015F0009E4229D3194B9E4226D238B3C0F30B0426
:10160000D4B93368984219D3726800F580539A426E
:1016100014D301A8FEF7F6FE90B1019BC3E9006464
:10162000019B02221A722D0B01229D811A82FFF763
:1016300043FF204602B070BD0620FBE70520F9E716
:101640000720F7E70120F5E70220F3E70320F1E7A1
:101650007DBC0020202D0020202D0020302D0020DA
:1016600010B50B4C0B4B628803EB02139A892AB915
:101670005868FFF7B5FF0423237010BD05232370BE
:10168000054B022218689A80FFF7AAFFF5E700BF12
:1016900080BC002098BE0020DCBF002008B5074BAE
:1016A000191D5888FDF796FF18B1BDE80840FFF7EF
:1016B0005BBFBDE80840FFF7D3BF00BF80BC002080
:1016C00060DF704710DF7047002208B5114617F041
:1016D000A9FD00002DE9F347254B1B681BB1984776
:1016E00030B3FFF7F1FF234B1B7803F0FF07FBB18B
:1016F000214D224E2C68DFF88C90B4FA84F46409F2
:10170000B0463378A3B901A8FDF748FF052812D0E9
:101710000028E6D1019B0BB9FEF71CF9184B1B689A
:101720000BB1019898474CB10124EAE7002CFBD09B
:1017300002B0BDE8F087002CFAD13C46DFF848A0A3
:1017400098F80030002BF3D1B9F80030ADF8043030
:10175000DAF8003001A91846FDF71EFF0528E5D08C
:101760000028BED12A6818469047002CE8D1C8E767
:101770006CBC0020D8BF002054BA0020D9BF002084
:10178000E4BF002050BA0020CCC0002010B5084BA8
:101790009A685AB150B9EFF3108172B6054A1C68C5
:1017A00014605C685460986001B962B6002010BD96
:1017B000D4C0002000E100E02DE9F3411D4F7B681B
:1017C00006460D469BB304292FD943697BB3437C5E
:1017D0000024012B0DF107000CBF8846A0468DF8B0
:1017E0000740FFF7B1FB0DF10600FDF781FFD0B117
:1017F00001230370104B4660D3F80435C0E904841C
:10180000C0E902359DF806307B709DF80700FFF7B0
:10181000BDFF24B9094B4FF48012C3F800212046C4
:1018200002B0BDE8F0810424EFE70724F7E70824BD
:10183000F5E700BF14BE00200010014000E100E009
:101840002DE9F341CE0801F007044FF0010808FA32
:1018500004F4855DE4B22540074613D10DF107007D
:101860008DF80750FFF770FBBB5D9DF807001C4229
:1018700002BF1C43BC554546FFF788FF284602B00F
:10188000BDE8F0810025F9E72DE9F34781460027FF
:1018900001261FFA87F84FEAD80A08F0070406FA6B
:1018A00004F419F80A50E4B2254008D00137B7F51E
:1018B000807FEED1B846404602B0BDE8F0870DF11A
:1018C00007008DF80750FFF73FFB19F80A309DF825
:1018D00007001C4202BF1C4309F80A400125FFF71C
:1018E00055FF002DE2D0E6E773B50546B8B1C1F368
:1018F000C70401F0070301269E40035D33420ED06A
:1019000000230DF107008DF80730FFF71DFB2B5D5D
:101910009DF8070023EA06062E55FFF737FF02B0B1
:1019200070BD000038B50A4B1A687AB15D686DB1B8
:10193000FF280BD084B221462846FDF713FF28B1BB
:1019400021462846BDE83840FFF7CEBF38BD00BF6E
:101950001CC000202DE9F74F9846531E072B8146E7
:101960000F46154600F2BB80FF2800F2B880014602
:101970005E48FDF7F7FE0646002800F0B0803946C5
:101980004846FDF741FF044600283ED0C3689D420B
:1019900047D805D25FFA85F9E368207C994543D39F
:1019A00094F81090B9F1FF0F40F09780504B1A68EF
:1019B0009B46002A41D14FF6FF732380A37000237A
:1019C000C4E90133E360238A03F4784343F0FF035F
:1019D0002382112084E0237C1844C0B2FFF7A2FFC9
:1019E000E3685FFA8AF083420AF1010AF3D84FF6FE
:1019F000FF732380A3700023C4E90133E360238ACB
:101A000003F4784343F0FF032382FF214FF6FF7076
:101A1000FDF7FAFE04460028DBD0A0F8009087709E
:101A2000BEE74FF0000ADBE74844C0B209F1010904
:101A3000FFF778FF5FFA89F9AEE75B68002BBAD051
:101A40000023DBF808205FFA83FA924502D34FF0B7
:101A5000FF0912E0DBF8040060B351460193FFF781
:101A6000EFFE019B30B3B9F1FF0F08BFD146AAEBDF
:101A7000090A0AF1010AAA4521D1B9F1FF0F84F838
:101A8000109098D0E560207CFDF77CFE58B305EB04
:101A900085052D01ADB2AD0888F80270C8F80400C4
:101AA000A8F8005026B1082F02D1AD00063D858070
:101AB000002015E0B9F1FF0F0CD14FF0FF09013301
:101AC000BFE74846019309F10109FFF72BFF019B8E
:101AD0005FFA89F9D145F4D3EFE70026D2E7072072
:101AE00003B0BDE8F08F0320FAE700BFF0BE00208E
:101AF0001CC0002038B504460025E368AB420ED870
:101B00004FF6FF732380A3700023C4E90133E36021
:101B1000238A03F4784343F0FF03238238BD207CFB
:101B20002844C0B2FFF7FEFE0135E6E737B5FDF702
:101B30006BFE0546A0B144682CB10A4B01941B789A
:101B40009B0706D403242846FFF7D4FF204603B0A2
:101B500030BD01A8FDF724FD04460028F3D0F1E7CD
:101B60000524F3E77CBC0020FF2810B5044609D803
:101B700001460548FFF7B8FE21460448BDE810407D
:101B8000FFF7B2BE10BD00BFF0BE002010BF0020A6
:101B900013B50DF106010446FDF744FD70B1BDF823
:101BA0000620084B03EB02139A894AB1A17A39B196
:101BB000013A00209A81A07202B010BD0A20FBE712
:101BC0000620F9E798BE002037B50D460DF1060155
:101BD0000446FDF727FD88B1BDF80620084B616873
:101BE00003EB021300209A8901329A81296063680D
:101BF0000C336B600123A37203B030BD0A20FBE7F6
:101C000098BE00202DE9F043DFF88480D8F874E016
:101C1000BEF1030F0F46944635D81C4E756CC1F1CA
:101C200008039D422FD8D8F8704074441C2304F058
:101C30000304814603FB0484B9E80F000FC499E84C
:101C400007000EF1010384E80700C8F87430C7B13B
:101C5000336C2B4403F0070306EBC303002206F1A9
:101C600038040CEBC20103C9A34202F1010283E86C
:101C7000030014BF0833054B9742F2D1736C1F4425
:101C80007764012000E00020BDE8F0834CBB002019
:101C90001CBE00202DE9F0411C46184B1B789B0709
:101CA00006460F46154627D5DFF85880A3880BB1A6
:101CB0000A201FE098F800302BB92146A088FDF7D4
:101CC00089FC20B92060A3880133A380EEE7236854
:101CD0001EB1998832889142EFD11FB119883A8894
:101CE0009142EAD19B682B6023686B60044B1B898F
:101CF0002B810020BDE8F0810220FBE77CBC0020A6
:101D000080BC002098BE002030B587B04CF207039D
:101D100005460C46ADF8043003AA0F4B01A900207C
:101D2000FFF7B8FF10B1002007B030BD01A903A82C
:101D3000FFF74AFF0028F6D10723A370019B5A88BA
:101D40002280029A62609B8803F580432B8003A85F
:101D5000FFF71EFF0120E7E770BC00201FB500233E
:101D6000A0F58040A1F58041CDE90233ADF8040033
:101D7000ADF8061002AB0DF1060101A8FFF78AFFCE
:101D8000002818BF052005B05DF804FB2DE9F041DF
:101D900002230B80164B00251C6800F5805E2F4641
:101DA00008304FF6FF7870450AD305B11C6002B1C8
:101DB0001770BDE8F08101270EE0344601250BE0E5
:101DC00006680136F1D086884645F4D00688002E94
:101DD000F1D08668A642F0D8468806F1030C00EBE5
:101DE0008C00B1F800C00CF1030C66440E80DAE7F9
:101DF00008BE002070B5064D0646002455F8043B89
:101E00000BB1304698470134082CF7D170BD00BFA4
:101E100028BB00202DE9F047AA4C266F1C2707FBA2
:101E200006F586B0635D013B8046052B00F22A81F2
:101E3000DFE813F00600640064001D011D017E014F
:101E400030B1A14A137823F00103137001201FE081
:101E500025442B79032B15D8DFE803F002072C3437
:101E6000FFF7B2FB01232B7109E0984D2B78022B71
:101E700040F03C826868FFF79FFB00232B7000282E
:101E800000F0F080904A137823F0010313700E20C5
:101E90001C237343E218E35C0290023B012B00F227
:101EA00032818B4B907D196C5A6C0144121A196463
:101EB0005A6428E1874F3868FFF792FB0223BB8002
:101EC0000023D0E7834FDFF804823868FFF774FB04
:101ED000814BD7F800E05B88B7F804C01B0108EB22
:101EE00003025168A2F808C0C2F804E00222BA80D6
:101EF0000022396008F803202A71C0E707FB064773
:101F0000724BB7F812A04FEA0A1A03EB0A0299467D
:101F1000118960B1FB8803F103088844C3F57F434E
:101F20005189A2F80880FD330B4453818EE7536832
:101F300003EB81083B7C062B00F29780DFE803F07F
:101F40002D733C4D1F84040041F61D501C2303FBE0
:101F50000643D144DB88B9F80810DA1C0A44A9F812
:101F60000820C3F57F43B9F80A20FD331344A9F8CC
:101F70000A3041F61D53984200F0C38088E7574865
:101F80005749002343601C2303FB06439B690360FE
:101F9000FDF748FB002800F04C81291D0122214457
:101FA0004046FFF797FA1C2303FB064302221A74EC
:101FB000002857D00E20C9E705F10C010122214469
:101FC00008F10800FFF786FA1C2303FB06439A7DFD
:101FD000002A14BF03220122E9E73D4B5A6C002A74
:101FE00000F08C81196C1C2505FB0645481C00F08F
:101FF000070003EBC1071864A88A53F83110013AAF
:102000005A6408EB8000BA88FFF764FAAB8ABA8892
:102010001344AB82AB7D013BDBB2AB75002BC7D168
:1020200001232B74C4E705F108010122214408F1C2
:102030000400FFF74FFA1C237343E25C032A0CBF32
:10204000052206222344B2E7254B1988234B586802
:10205000FFF79EFA1C2303FB064306221A7400288E
:102060007FF474AF06B0BDE8F0870F206EE700285C
:102070007FF4ECAE07FB06473B79012B32D01BB156
:10208000022B3ED00F2003E7CDE90200FB6801934D
:102090000DF1020101A8FDF7C5FA80B10298BDF863
:1020A00002108388FB8003883B81FFF771FA1C23B1
:1020B00003FB064302221A710028D3D059E70A20F5
:1020C000F5E700BF1CBE00207CBC002098BE0020AD
:1020D0004CBB0020DCBF002080BC00204C2D002029
:1020E000E0C00020864FA81D3B4601AA414620447F
:1020F000FFF7D0FDB8B9B9880298FFF749FA0A2866
:10210000DAD1002302931C2303FB06F2A25C013AFE
:10211000052A00F2B580DFE812F08E009200A000E0
:10212000CB00D500E1000A28C7E90088E9D020E704
:1021300000287FF48BAE734BDA7AAAB1D8721A7882
:10214000013A062A9ED801A151F822F0FD21020091
:10215000F72102000D220200132202008520020056
:1021600019220200292202001A78072AE7D801A1C1
:1021700051F822F0952102003F2102003F21020088
:10218000B1210200C5210200E3210200E321020087
:10219000AD2102001A8901321A8100225A80DA72B6
:1021A000594A1278B2FA82F252099A72012207E071
:1021B000564958688A884088033202448A8002223D
:1021C0001A70BCE75D88504A504902EB0512086856
:1021D000556850608888108102228A800D6006222E
:1021E000EEE70722ECE7484900229A728A8942B951
:1021F000897B31B15A80FFF751FA5DE79A7A002A5C
:10220000F1D100221A705A805A607AE7FFF7ACF9D0
:1022100052E7FFF725FA4FE75A883B4B03EB0213CF
:102220005868FFF7C9F947E700225A60FFF7CCF971
:1022300042E70A202CE600238DF8043020E003FB5F
:10224000064301228DF804201A89ADF810209A88DF
:10225000ADF81220DB68039312E003FB0643022271
:102260008DF804201A89ADF810209A88ADF8122054
:10227000DA681B7C03929A1F534253418DF8143045
:1022800001A8FFF7B7FD206F1C22002102FB0040D0
:10229000FDF748F9636F1BB3226F013202F00302AE
:1022A000013B22676367DBB10020FFF7B3FDD9E68E
:1022B00003FB064303228DF80420DA88ADF81020D2
:1022C0001A89C5E703FB06430422DB88ADF810300A
:1022D00000238DF80420ADF81230D1E70523ABE7D9
:1022E0000B4A137823F004031370BBE6084A1378F3
:1022F00043F0020323F00103137002E71368FFDECB
:10230000E8C0002080BC002098BE0020DCBF002078
:102310007CBC00200846FFF77DBD0000054A13780D
:1023200013F0040004D143F004031370FFF772BDEF
:10233000704700BF7CBC0020F0B51C463D4B1B78AD
:102340009E0789B007460D466FD509884FF6FF7383
:1023500099426CD06B88002B69D06968B5F808C0C9
:1023600000239C4503D8BAB9164604310AE051F857
:102370003300800757D10133F3E731F8320030449E
:1023800086B201329445F8D80DF102013046FDF7CE
:1023900091F928B109B0F0BD13885688ADF8023024
:1023A00000238DF81430BDF80230ADF81630032349
:1023B000ADF81830204B8DF804401A6829898DF843
:1023C0001A1001321A602B88ADF80C30032C6B8880
:1023D000ADF8083004BF04238DF81430049208BF10
:1023E0003B686A6808BF0793002401A8ADF80A603B
:1023F000ADF80E40FFF706FC50B9BDF802200F4BB8
:1024000003EB021358890338801B58810820C1E769
:10241000049B3B600A4B7C601B89BC723B81FFF7CD
:102420007DFF2046B6E70320B4E70220B2E7042090
:10243000B0E700BF7CBC002008BE002098BE002092
:1024400080BC002030B58BB0FF28044601921D46A9
:1024500045D88B781846FDF7ADF900283FD04A687B
:1024600002920A88ADF80C20A4F58042ADF81C2039
:10247000A3F58042ADF81E2002AA08920122ADF811
:102480002420194604AA2046FFF768FC0528019A73
:102490000ED1022352B907A904A8FFF74DFF072860
:1024A0001FD010D8B0B103200BB030BD01AAF2E7A5
:1024B00032B10E4B1B789B0702D501A8FDF770F8CF
:1024C00003230022E7E708280DD00E280CBF1120B7
:1024D0000320E9E7002DE7D0049B2B60E4E7072009
:1024E000E2E78620E0E71120DEE700BF7CBC0020A9
:1024F0001F4B204A1B6800BF00BF00BF00BF00BFCA
:1025000000BF00BF00BF93422FD000BF00BF00BF7D
:1025100000BF00BF00BF00BF00BF00BF00BF00BFC3
:1025200000BF00BF00BF00BF00BF00BF00BF00BFB3
:1025300000BF00BF00BF00BF00BF00BF00BF00BFA3
:1025400000BF00BF00BF00BF00BF00BF00BF00BF93
:1025500000BF00BF00BF00BF00BF00BF00BF00BF83
:1025600000BF00BF00BF00BF00BF0138C3D170472C
:10257000A42C00200024F40073B5154E73680546A2
:102580001BB343690BB3002404740DF107008DF8ED
:102590000740FEF7D9FC0DF10600FDF7A9F890B150
:1025A000022303709DF80630456073709DF80700A4
:1025B000FFF7ECF824B9074B4FF48012C3F8002161
:1025C000204602B070BD0424F0E70824F8E700BFFD
:1025D00014BE002000E100E02DE9F8432649274B16
:1025E0000025C1F84051C1F84451C1F84851C1F823
:1025F0004C51C1F80051C1F804511B68002B39D06F
:10260000D1F804451E49DFF88C800968641A24F06B
:102610007F442F461A68A24217D8A41A15441A7C80
:10262000DE6982B1D8F800901F74D3E90521B9F1B1
:10263000000F06D01046C84728B1FFF745F83346CB
:10264000E8E708469047002EF9D10E4A0E4B117864
:102650001B788B4205D10133DBB2022B08BF00236C
:1026600013701278094B43F82250094B4FF4801233
:10267000C3F80021BDE8F88300100140D0C000205D
:10268000F4BF0020F1BF0020F0BF0020E8BF002011
:1026900000E100E068BC00200D4B0E494FF4003211
:1026A00010B5C3F8802001244FF48033C1F84833BB
:1026B0002F20C1F808334C60FFF71AFF064B8C60DF
:1026C0002F2000211960FFF713FF044B197010BD74
:1026D00000E100E000100140F4BF0020D1BF002065
:1026E0002DE9F04FB64AB74913780978B64D85B051
:1026F0009942D5F80080019500F095800133DBB256
:10270000022B08BF002313701278B04B53F82260DD
:10271000019A08EB060323F07F4313600127AC4BBB
:10272000AC4A18680290AC48117890F800904FF0CD
:10273000000CE2465078884278D1BCF1000F02D0FC
:10274000A54981F80090002F40F0BB801F680299D6
:102750007F1A18BF01270020196802919E49039132
:1027600091F800E000244FF00108002840F0AD800F
:1027700092F80190D2F804C092F802A0117849456D
:1027800040F0C1801B68029A9A4201D1002F44D0C8
:10279000002B00F01281D3F80090904C019BD4F8EC
:1027A000046519688E4F751A3B7825F07F4503350F
:1027B000A3B94FF48033C4F84433C4F80433894BCD
:1027C0004FF400324FF00108C3F880212F201A6027
:1027D000C4F80080FFF78CFE87F80080A9452CBF65
:1027E0004944491921F07F41C4F84015D4F8043513
:1027F0009B1B23F07F43891B033321F07F418B42D6
:102800000BD9D4F80435C4F840352F20FFF770FEFB
:10281000744B4FF40032C3F80021039A0023137065
:1028200005B0BDE8F08F0026374678E701EB41049C
:10283000506892F802B000EBC40E013110F8344039
:102840001868C9B28B4508BF0021022C04D0032CA4
:102850007FF470AF002410E0DEF804B00446864632
:10286000002C3FF467AFA34500F0C080A646E469A2
:10287000F6E780F810A0C06901240028F9D1002CE7
:102880003FF458AF186055E7D4F80C90C4F800E056
:10289000761A8C44E1691960B9F1000F07D008EB92
:1028A0000C0121F07F41C4E90119E06120461C6858
:1028B000002C3FF451AF2168B142E5D98E1B266050
:1028C0004AE7002084468646F1E70146C069019D3B
:1028D000D1F804A02E68444DD1F80890AAEB060C5C
:1028E0002CF07F4CAC4535D80CEB09060E60D3F8C4
:1028F00000C081F81080C1E90144CC61BCF1000F37
:1029000033D1196031E701EB410B0131C9B25145B7
:1029100014BF117014701CF83B1001290CEBCB068E
:102920007FF42CAF716891F810B0BBF1000F7FF409
:1029300025AFD6F808C0C1F804C0F5688D603569C8
:10294000CD6076698E61BEF1000F0CBF66465E46B3
:102950004E60BCE7A6EB0A0626F07F464E4502D243
:10296000A9EB0606C2E70C60C1E7D1F80090DCF8DD
:102970000060B1451FD8A6EB0906CCF80060C1F88D
:102980001CC0BEE7A9EB0A09D6F81CA0B446BAF1F0
:10299000000F0AD05646D6F800A0CA45F2D3AAEBDB
:1029A000090AC6F800A0B2466646C1F80090C1F810
:1029B0001CA0F161D9E66646EDE7FFF76DFE2CE756
:1029C000F0BF0020F1BF0020F4BF0020E8BF0020CE
:1029D000D0C0002014BE0020D0BF00200010014055
:1029E000D1BF002000E100E0FEFF7F0074450FD161
:1029F000D0F81CB0C3F800B0BBF1000F08D10A4DED
:102A00000120A86001984FF0010CC0F800B0E14629
:102A10002068E469CEF81C40002C3FF48BAE25689A
:102A20002844206086E600BF0010014037B5074B00
:102A3000054693E803006C46002384E803001A4629
:102A400021462846FFF7FEFC03B030BDD437050011
:102A5000FDF7F4BC10B54FF6FF7304469C420846E0
:102A600009D1FEF711FFB0F5807F044601D14FF682
:102A7000FF74204610BDFF2CF9D82146FEF7E0FE7A
:102A80000028F6D1F3E710B5044601F0EFFC20462C
:102A9000BDE8104000F02EBF1FB5037893B902794E
:102AA000072A0FD1448803932046CDE901338DF8DE
:102AB0000420FCF741FEADF8060001A8ADF808407F
:102AC000FFF7E1FF04B010BD1FB50023CDE90133CE
:102AD0000393ADF80600022301A88DF804308DF8A9
:102AE0000810FFF7D0FF05B05DF804FB86DF7047E4
:102AF00038B504884CB9821C00F10A0512F8013B74
:102B00001BB99542FAD100200AE00B88A342FAD102
:102B100008220231023030F0FFFDB0FA80F04009A7
:102B200038BD08B570B171B103780A78534013F01D
:102B3000FE0F08D106220131013030F0EDFDB0FA70
:102B400080F0400908BD0020FCE710B5044600F005
:102B5000BDFF2046BDE8104000F04ABF43DF70478C
:102B60006FDF7047024B0022C3E90022704700BFAD
:102B700070BC0020F0B5FF2887B004460E4615460D
:102B80001F4629D80846FCF715FE28B303AA20469D
:102B9000FFF7E4F818B10524204607B0F0BD01A9FD
:102BA00003A8FFF711F804460028F4D1019BAE708A
:102BB0005A882A805FB13B6892009A420AD30299F0
:102BC000686830F0B7FD03A8FEF7E2FFE4E7029B78
:102BD0006B60F8E70424DFE70724DDE72DE9F04127
:102BE000CEB020AE502380460CADB8220021304636
:102BF00001930395FCF796FC0DF1970305930DF1F6
:102C0000AE0306930DF1C503079337AB08930DF19F
:102C1000F30309930DF585730A931C4F04960DF287
:102C200021130B930024444507D1E2B2002104A8EC
:102C3000FFF796FF4EB0BDE8F081502200212846F4
:102C4000FCF770FC01AB02AA072137F8020BFFF773
:102C500091FF20F002000528ECD06B7C032B12D8EA
:102C600017230DF1310203FB04630DF1450152F806
:102C7000040B43F8040B8A42F9D111881980927829
:102C80009A700134CFE743F20220D3E7FABF002065
:102C90002DE9F04110220546A6B000212D48FCF791
:102CA00041FC35B929462846FCF75AFD26B0BDE857
:102CB000F0816A0028492748DFF89C8004AE30F094
:102CC00039FD382200213046FCF72CFC002450232B
:102CD000CDE9013412AF0397502200213846FCF7AA
:102CE00021FC01AB02AA072138F8020BFFF742FFD3
:102CF00020F002000528D9D09DF85930032B26D8A2
:102D0000C4EBC402B318DDF85910B1500134BDF85A
:102D10005D209A80A5429DF85F209A71DCD10DF16B
:102D2000170313930DF11E0314930DF1250315934F
:102D30000BAB16930DF1330317930DF13A03189370
:102D40000DF1410312961993E9B23846ACE743F20C
:102D50000220ABE70AC00020FABF00202DE9F043B3
:102D6000037889B00546002B3FD1017907293CD172
:102D700004AA4088FFF7FEFEB8BBFFF7F3FE02A9E6
:102D80000DF10600FEF7C0FF78B36E88BDF806703F
:102D9000BE42F4D0059C631C1846113413F8012B75
:102DA00012B9A342FAD1EAE7DDF80C80102208F14B
:102DB000010130F0B1FC08F1110181462046FFF716
:102DC000B0FEB9F1000F01D00028D8D03046FCF792
:102DD000B3FC0023ADF81A0006A88DF81830ADF842
:102DE0001C60ADF81E70FFF7B0FE09B0BDE8F083BF
:102DF000CA1F012A73B5064654D80025CDE90055EF
:102E00008DF80210FCF700FD044600284CD0437CEE
:102E1000DB074BD4007CFCF7B5FC10B9032002B0F3
:102E200070BDE368019003EB83031B019BB29B0819
:102E30006846ADF80030FCF7C5FC626804F1080391
:102E400069463046FFF7FEFA637C03F00603062B63
:102E500001BF174A136803F1FF33136030B9637C75
:102E600023F0070343F001036374D8E711280BD163
:102E70000F4A136801331360637C23F0060343F0A9
:102E8000040363740020CAE7862809D1084A13683E
:102E900001331360637C23F0060343F00203E3E78E
:102EA0000728BBD10720BAE70520B8E72846B6E7D0
:102EB00010BE00202DE9FF41054610220021684682
:102EC000FCF730FB68882979ADF802008DF8041012
:102ED000FCF79AFC2B78454E092B5ED8DFE803F00F
:102EE0000505684D4D6C7173757D00283FD0437C9E
:102EF000DC073CD5FEF7FEFD2B78581E43424341CC
:102F0000002468468DF800408DF80830FCF76EFC10
:102F100033684BB3364E002537464FF0140808FB94
:102F200005735B7C5A0703D49B0759D5002C57D0F7
:102F3000B1783088FFF75CFF002851D014235D433F
:102F40007B1986289B788DF804307A5B16BF029037
:102F5000082309236846ADF802200CBF8DF8003025
:102F60008DF80030FCF742FC04B0BDE8F08101238D
:102F70008DF80030AB68029316E080B18268AB68D0
:102F80009A420CD1437CD90709D5326823F0050356
:102F9000013243F00403326043740024B8E7022393
:102FA0008DF80030EB6803936846FCF71FFCF4E7EC
:102FB00003238DF80030F7E704238DF80030EB6829
:102FC000D9E70523F5E70623F7E7072368468DF8D9
:102FD00000300124FCF70AFC9AE7EB680293DCE777
:102FE0000135082D06F1140699D1BDE710BE002069
:102FF0002CC0002070B500238CB02D492C4E4FF60C
:10300000FF70CDE90033FCF771FC4FF6FF75044605
:10301000AC420BD0A4F58043ADF8143002AA6B4645
:10302000002105A8FEF736FE0A2822D0214B1A7887
:103030001846E2B94FF6FF718C4218D01E4E367812
:1030400001251D70B607A4F580439BB21DD58B42A8
:103050002CD005218DF8141005A811468DF81850B4
:10306000ADF81A30FEF7CEFD60B1FFF757F90CB09E
:1030700070BD2046FEF778FD20463146FCF736FC51
:103080000446C5E70D4B1D70F1E70223002209211C
:1030900002708DF8141005A8FF21ADF816408DF8C8
:1030A0001810CDE90723FFF705FFE0E70423EDE75C
:1030B00010BF0020A9BE00207CBC0020AABE0020BA
:1030C000F0B5426805783D4C85B0B2FA82F1490905
:1030D0000391691E0346042924D8DFE801F00303A5
:1030E00030496A009989DE8901F5804189B243F649
:1030F000FE77B94204D906F5804080B2B84211D8B3
:10310000012DADF802108DF8046013D1002A14BF10
:10311000032100218DF8001003929B6802936846FA
:10312000FFF7C8FE23781BB100232370FFF762FF6F
:1031300005B0F0BD002A14BF04210121EAE79989F6
:10314000DD8901F5804189B243F6FE76B14204D9AA
:1031500005F5804080B2B042E4D8002A0CBF0222BC
:103160000522ADF802108DF804508DF80020D4E748
:10317000988900F5804080B243F6FE718842D1D82C
:10318000DB89002BCED1FF23ADF802008DF804308F
:103190005AB906238DF80030FEF7E6FC084A0023F2
:1031A00023701370FFF726FFB9E707238DF800306F
:1031B000F4E708238DF80030B1E700BFAABE002075
:1031C000A9BE0020F8B50D490D4DFCF78FFB4FF659
:1031D000FF760446A5F12007B44201D12046F8BD90
:1031E000FF2CFBD821462846FCF7BCFA0028F5D076
:1031F00020463946FCF77AFB0446EDE7F0BE002096
:1032000010BF002073B5104B104C93E803006D46BF
:10321000002385E803001A4629462088FFF712F9A3
:103220004FF6FF762388B34201D0112801D102B0B6
:1032300070BD1846FFF7C6FF00231A4629462080B6
:10324000FFF700F9EEE700BFDC37050058BC0020AF
:103250001FB50378012B044615D10179012912D13C
:10326000002302AA4088FFF785FC60B902238DF88D
:1032700000306388ADF80230039B68461B788DF8F8
:10328000043000F0B5FD054B1A884FF6FF739A42E3
:1032900001D0FFF7B7FF04B010BD00BF58BC00203D
:1032A00070B504468AB0142200216846FCF73AF94A
:1032B0006588ADF804502846FCF73EFA2378ADF84F
:1032C0000200092B15D8DFE803F005163048525EDE
:1032D0008614A1A507238DF8003023798DF80830D6
:1032E0009DF80A3043F001038DF80A306846FCF778
:1032F00017FB0AB070BD07238DF8003023798DF8D5
:1033000008309DF80A30444AA168039143F0010354
:103310008DF80A301368002BE8D09942E6D10023DB
:1033200013603E4A03931580E0E708238DF80030D0
:1033300023798DF80830E3680493374BA1681A6845
:103340000391002AD2D09142D0D1354900221A608F
:103350000B680392013B0B60C8E707238DF8003030
:1033600023798DF8083001238DF80930BEE7082352
:103370008DF8003023798DF8083001238DF809305D
:10338000A3680493B2E7274D09238DF800302B780A
:10339000002BABD04FF6FF70FFF714FF4FF6FF7313
:1033A00098420646A2D12049FCF7A0FAB042044652
:1033B0009CD1142200210DEB02002970FCF7B2F819
:1033C0000B238DF81430ADF81840ADF8164005A861
:1033D000FCF7A6FA8AE70A238DF80030114BA4689F
:1033E0001A780294002A81D0142200210DEB0200E9
:1033F0001970FCF797F80C238DF814304FF6FF7313
:10340000ADF81830ADF816300794E0E705238DF8D5
:1034100000306BE70623FAE7ECBE002004BE002074
:1034200054BC00205ABC002010BF00202DE9F047FA
:10343000474B1B788AB00546002B00F08780454B30
:10344000454F93E803003C7803AE86E80300BCB91F
:103450004FF6FF70FFF7B6FE0123ADF8143001AB55
:1034600006930423029305AA02AB06218046019429
:10347000ADF81640FFF77EFB07284AD101233B70C9
:10348000364B1C689846002C5AD1354A354F128865
:103490003B68AA4241D1002B3FD0142221460DEBBC
:1034A0000200FCF73FF8072328468DF81430FCF79C
:1034B00043F90623ADF8160005A8ADF818508DF8AD
:1034C0001C30FCF72DFA20460AB0BDE8F087CDF895
:1034D00004A0019B4046A34224BFC1461C46FFF7FF
:1034E00071FEBDF814309B00029305AA02AB0621C1
:1034F0008046FFF73FFB0028EBD00528E7D04FF6CA
:10350000FF7398451CD1164BA3F80090154B1C6017
:10351000B4E74FF6FF79A246EDE701333B600022A6
:103520000E4B31462846FEF78DFF0028CCD00023F5
:10353000C8F800303B68112803F1FF333B6001D12C
:103540001120C1E7862818BF0320BDE70820BBE78C
:103550000CBE0020E4370500EBBE0020ECBE0020CE
:1035600004BE002054BC002063DF7047A6DF704714
:10357000A2DF70472DE9F04391B0984611238DF8F2
:10358000043013788DF805300024164601254FF0DD
:10359000000365F34203074689461C22214609A819
:1035A0008DF80630FBF7BEFFB3788DF80930C3F312
:1035B0000302A24214BF1A2212228DF8242001AA6B
:1035C0000E9203AB72788DF808200493224602AB6A
:1035D00065F34202059308238DF80A20CDE90644DD
:1035E00004AAADF81C3009A9434638888DF80E505E
:1035F000ADF80C900894FFF7BBFF11B0BDE8F08365
:10360000A0DF7047044A0123116883400B401ABFB2
:103610001218507E184670471CBA002070B4094D2D
:10362000134601262A6806FA01F4144207D001F174
:10363000190402463146281970BCFDF757BE70BC0C
:10364000704700BF1CBA00201FB50023CDE901332D
:1036500003938DF80A201A46074BADF8081006248C
:103660001978ADF806008DF80440FFF7D7FF01A8E0
:10367000FFF709FA04B010BDAF2C002010B4084ABF
:10368000012314688B40234006D00A445DF8044BA4
:103690000146507EFDF79ABD18465DF8044B704711
:1036A0001CBA002010B50A4B19780446FFF7E6FF54
:1036B00058B1084B00205A88A24201D1C0B210BDB7
:1036C0000130082803F10C03F5D1FF20F7E700BF14
:1036D000E8BB0020EABB00202DE9F8430546FCF7D3
:1036E0002BF8234B074600221420984600FB02F1DA
:1036F000CC5AAC422AD10B44002634464FF0140970
:103700005BB199782846FEF711FA10B1052818BF69
:10371000032401363246072A1DD9A4B9FF2D24D827
:10372000144928464FF6FF75FFF794F9FFF762FC3E
:10373000AF4208D03846FFF7B5FFFF2803D00C236F
:1037400043430D4AD5522046BDE8F8830132082A8A
:10375000CCD10023D0E709FB02F338F80310A942CB
:1037600001D14344CCE70132D5E70724EBE700BFA2
:103770002CC0002010BF0020EABB00202DE9F04142
:103780001F46154B9DF818400E4690461978054681
:10379000FFF744FFB8F1000F17D0104B3A461978E5
:1037A0002846FFF73BFF0E4B224619782846FFF7C5
:1037B00035FF44B12846FFF775FFFF2803D00C23DF
:1037C0004343084AD652BDE8F081002CFBD0304676
:1037D000BDE8F041FFF780BFAF2C0020B12C0020E6
:1037E000B02C0020EABB002008B5FFF75BFFFF28E4
:1037F0001DBF0C234343034A4FF6FF7018BFD05A36
:1038000008BD00BFEABB00202DE9F04385B00546A6
:10381000FFF7EAFF4FF6FF739842074641D00122B7
:103820004FF0030901AB0821384602F10108FEF709
:1038300091F81FFA88F8064648BB02990A46032306
:1038400042F8049B06312846FBF76AFF044660B93C
:1038500008213846FFF7CCFA0446112C3FD01AD87D
:103860000CB30C2C2FD107231EE00C280DD00528FB
:1038700000D1344608213846FEF758F9002818BF11
:1038800003244246002ECDD1E7E70126F2E70728C0
:10389000E9D00446E1E7862C13D043F202039C42B0
:1038A00011D100221CE0012328468DF80430ADF828
:1038B0000850FFF799FFADF8060001A8FFF7C8F818
:1038C000EFE70823F0E7092328468DF80430FFF7D7
:1038D0008BFFADF80850ADF806000394EDE7012228
:1038E000034B28461978FFF799FE05B0BDE8F08331
:1038F00079BC00200378072B02D14088FFF784BFF2
:10390000704700002DE9F0434FF6FF75A84285B0DF
:10391000044668D0FFF768FFA84227D10026032796
:10392000B0464FF001093B46324641462046FBF780
:10393000F9FE042805464DD0082847D00B282DD184
:1039400017F002031FD1B8F1000F20D11EBB0323D3
:1039500020468DF80430FFF747FFADF80840ADF87A
:10396000060001A8FFF774F8002237E0002301AA3F
:103970000821FFF7FFF80028D0D1029B03F10608C9
:103980009E881F68CDE701274FF00009CBE703278A
:103990001E469846F8E703274646F5E7B9F1000FBB
:1039A000D5D0112819D043F202039842DCD008B9CF
:1039B0000223CDE7092320468DF80430FFF714FFDA
:1039C000ADF80840ADF806000395CAE7B9F1000F5D
:1039D000EED1BCE7B9F1000FB9D00122034B20466C
:1039E0001978FFF71BFE05B0BDE8F08378BC002016
:1039F00037B50578012D044614D14088FFF782FFC2
:103A00006088FFF7F1FE00236A462946FFF7B2F807
:103A100040B9019B1B782BB1034B608819782A466B
:103A2000FFF7FCFD03B030BD7ABC0020F0B587B0D5
:103A300004460E461746FFF7D7FE4FF6FF7398422F
:103A4000054624D01E4B20461978FFF717FE80B399
:103A50000023CDE90033029304238DF80030194B85
:103A6000ADF802401978ADF8046020468DF8067074
:103A7000FFF704FE68B12846FFF72EFE124B2046E2
:103A800000221978FFF7CAFD6846FEF7FCFF07B071
:103A9000F0BD07212846FEF749F80528EED1092395
:103AA000049003A88DF80C30ADF80E40FEF7EBFF44
:103AB000E4E73A4631462046FFF7C6FDE7E700BF98
:103AC000B12C0020B02C0020AF2C002010B50278C3
:103AD00086B004461AB1012A09D006B010BD0E4BBB
:103AE0001B78002BF9D0C088FFF7F6FDF5E70B4BEC
:103AF00040881978FFF792FD1422002101A8FBF7F6
:103B000011FD6088ADF80600FFF76EFEADF8080005
:103B100001A8FBF705FFE0E70CBE002058BA002023
:103B200070B5044686B01422002101A8FBF7FAFC08
:103B300023786088ADF80600013B0B2B00F29080E3
:103B4000DFE803F02106233A4E585C68747A7C8CD7
:103B50002679444B321C19784FF0010518BF012219
:103B60008DF80450FFF75AFD731B5A425A413E4BE1
:103B700060881978FFF752FD6088FFF735FEADF8D1
:103B80000800002D42D106B070BD02238DF804302C
:103B90002379002B14BF012302238DF80C30314B05
:103BA00001221978FFF73AFD2F4B227919786088A6
:103BB000FFF734FD0125DFE703238DF804302A4B9E
:103BC0001978FFF75BFD002814BF012302238DF84D
:103BD0000C30A3798DF81030A388ADF80E30E9E7EA
:103BE000204B1978FFF74AFD0028CCD102238DF82D
:103BF0000430DFE703238DF80430EAE70723A288C7
:103C00008DF80430ADF808208DF80C3001A8FBF7D2
:103C100087FEB8E708238DF80430A388ADF8083094
:103C200007238DF80C30A3680593EFE706238DF882
:103C3000043063680393BDE70523D8E703238DF8B9
:103C40000430094B1978FFF719FD002814BF012330
:103C500002238DF80C3041F20113BEE70423C6E7BE
:103C6000002589E7A8BE002058BA00201FB50D29FD
:103C70004FF0000301930393ADF80600029108D1C1
:103C80000B2301A88DF80430FFF74AFF05B05DF85B
:103C900004FB86290CBF0A230923F2E730B5084943
:103CA0000A680023012505FA03F42242D8B202D1A2
:103CB00022430A6030BD0133182BF4D11846F9E7CE
:103CC0001CBA002010B50378182B044602D1FFF768
:103CD000E5FF207010BD000010B5024B197DFDF707
:103CE00023FB10BD1CBA00202DE9F04F3D4D89B0DB
:103CF0002878FFF787FC60B103A8FFF7EDFFDFF836
:103D0000E8A0DFF8E8B00DF110090027039B9F42FF
:103D100002D309B0BDE8F08F39F8024B297820466C
:103D2000FFF7ACFC064678B39AF800102046FFF780
:103D3000A5FC804640BBBBF800304FF6FF72194629
:103D40002046FBF7F1FC43F20302904229D10133F4
:103D5000ABF80030EFE7052320468DF80030FFF781
:103D600043FDADF802006846ADF80440FEF770FE72
:103D7000B046324629782046FFF750FC42469AF872
:103D800000102046FFF74AFC0137BFE72046FFF747
:103D90002BFDFEF74BFE0026EBE72046FFF7B2FDBA
:103DA000E7E70828F2D012D80028D4D00628EDD0B2
:103DB0000923029020468DF80030ADF80440FFF74B
:103DC00013FDADF802006846FEF742FED1E743F26C
:103DD00002039842CDD043F201439842DDD011282E
:103DE000E6D1C6E77ABC00207BBC0020E4C00020FE
:103DF0001FB5044640882378ADF80600012B10D08B
:103E00005AB21AB1022B15D004B010BD01A88DF81A
:103E10000420FEF71DFE6088FBF78EFCFFF772FDA5
:103E2000F2E78DF8043001A8A388ADF80830FEF75A
:103E30000FFEE9E72379002BE6D0FBF77DFC4FF678
:103E4000FF739842E0D0044B01221978FFF7E6FB9C
:103E5000FFF74AFFD8E700BF7ABC002038B5074C0F
:103E60000146207DFDF7B2F930B1A07DFDF7AEF936
:103E7000002814BF0220012038BD00BF1CBA00205A
:103E80002DE9F0478CB0894616468046FFF7E6FFDD
:103E900020228246002104A8FBF744FBBAF1000F60
:103EA00046D0B9F1000F17D099F8005015F0010570
:103EB0004FF6FF7415D04046FFF796FCA042074628
:103EC00039D14048FDF7E0FCB0F5807F01D0B84221
:103ED00075D10025032470E04D4685264FF6FF7707
:103EE0005FE02E4627465CE04A4631464046FBF7F7
:103EF0001FFC0446B9F1000F5DD000285DD199F890
:103F0000003013F0010F14BF012102214046FEF7DB
:103F1000DBFDB6F1850218BF0122002400950123C4
:103F200039464046FFF72AFC20460CB0BDE8F08732
:103F300043F20204F8E7002502AB012207213846CC
:103F4000FDF708FD0446002837D12146502203988A
:103F5000FBF7E8FA039B83F800A0039C079604F1A3
:103F60003403049304F118030893631C0993404637
:103F7000154B0B93FFF796FBFF280CD0134A0C212F
:103F800001FB002050F8042FC4F811208288A4F807
:103F900015208279E2753846FBF75CFC044660B96F
:103FA0000646BAF1020F04AB9ED1002231464046CC
:103FB000FBF7BEFB0446002CABD00022AEE7074661
:103FC0000125B9E7F0BE0020ABBE0020EABB00200F
:103FD000F0B585B00446FFF741FF324F0128064691
:103FE0003D7831D12046FFF7FFFB4FF6FF73984233
:103FF0002AD0204632462946FFF710FB0023CDE9A0
:104000000133039301A80C238DF80430ADF806406A
:10401000FFF786FD244B1B78E3B139782046FFF784
:104020002DFBB8B9214B22491A682046FFF728FF1B
:104030008628054632D011280FD070B12946204677
:10404000FFF714FE05B0F0BD002229462046FFF719
:10405000E5FADFE700221146E7E7A5F111035E422A
:104060005E410022134B20461978FFF7D7FA124B16
:10407000324619782046FFF7D1FA104B0022197802
:104080002046FFF7CBFA0E4B002219782046FFF7A7
:10409000C5FA002DD6D0112DD4D0CFE700260122AD
:1040A000E0E700BFAE2C0020D7BF002094BE002068
:1040B000D2BF0020AD2C0020AC2C0020AB2C002067
:1040C000AA2C0020F0B587B0074601A8FFF704FE30
:1040D00002AD0024019B9C4201D307B0F0BD35F82E
:1040E000026B39463046FFF7C9FA10B13046FFF788
:1040F0006FFF0134EEE700002DE9F04F054687B071
:10410000904699460F4639B9A14B1B78F3B905245F
:10411000204607B0BDE8F08FFFF7A0FE0138C0B21F
:10412000012800F22D8100212846FBF703FB0446FD
:10413000862C00F0B080112C00F09980002C00F04B
:104140009680B9F1000F00F0BF80B9E0FFF786FE5E
:10415000012800F09E80022840F012818D490B78E2
:10416000284613F001048B4614BF4FF0010A4FF0AC
:10417000020AFFF739FB4FF6FF739842064659468D
:104180003AD03B4602AA0721FEF7F4FC0446F0B9F8
:10419000039B93F84420D10740F1C780B8F1000F8A
:1041A00040F0D68003F1340202F112012846FBF7F9
:1041B000BDFA4FF0000A044600230093BAEB030354
:1041C00018BF0123B4FA84F25209314645E00528AC
:1041D000F2D1BDE004AB012207213046FDF7BAFB66
:1041E0000446002840F0C1803046FBF733FB04460C
:1041F000002800F0B280B8E0002C41D06648FDF7FE
:1042000043FBB0F5807F834637D0B04236D004AB55
:1042100001220721FDF79EFB044650B95846FBF7E3
:1042200019FB044628B95B492846FBF783FA044684
:1042300038B107215846FDF779FC10B1052818BFA1
:1042400003244FF6FF73BBEB030318BF0123B4FA3B
:1042500084F200935209012359462846FFF78EFA4B
:10426000002C7FF465AF51462846FEF72DFCA4F1E3
:1042700011035E425E4100220FE0B3460324E0E7F3
:104280002846FBF757FA009704460123B0FA80F25C
:104290009AE7404948E700260122404B2846197812
:1042A000FFF7BCF93E4B324619782846FFF7B6F9BE
:1042B000B9F1000F08D0002C3FF42AAF112C17D011
:1042C00021462846FFF7D2FC0D2C3FF421AF06D83B
:1042D000002C3FF41DAF082C18BF032418E7862CD0
:1042E00014D043F202039C423FF412AF112C1AD1B6
:1042F0002C4B3A4619782846FFF790F92A4B42464C
:1043000019782846FFF78AF9002401E7254B3A4639
:1043100019782846FFF782F9234B42461978284638
:10432000FFF77CF9F4E60324F2E6B8F1000F0FD1B1
:10433000598D03F1180200297FF436AF03F12C01E7
:10434000343311F8010B00287FF42EAF8B42F8D1E3
:104350009BF80030DA073FF53DAF0E492846FBF7E2
:10436000E9F9044600283FF427AF07213046FDF75E
:10437000DDFB00283FF420AF052818BF03241BE70E
:1043800043F20204B9F1000F3FF4C2AE98E700BF58
:10439000D7BF0020D2BF0020F0BE0020AB2C0020F1
:1043A000AA2C0020A92C0020A82C00202DE9F047E1
:1043B00086B00746FFF726F958B101A8FFF78CFC35
:1043C000DFF84880DFF8489002AE0025019B9D424F
:1043D00002D306B0BDE8F08736F8024B39462046D6
:1043E000FFF74CF980B198F800102046FFF746F926
:1043F00099F8001082462046FFF740F90123014654
:1044000052462046FFF778FE0135DFE7A82C002052
:10441000A92C002010B50378062B0ED9072B1BD131
:104420000E4B1C782046FFF7EDF810B12046FFF741
:1044300049FE0B4B1878FFF7B9FF0A4B1C78204652
:10444000FFF7E0F810B12046FFF73CFE064BBDE851
:1044500010401878FFF7AABF10BD00BFAD2C002098
:10446000AB2C0020AC2C0020AA2C00201FB5037818
:104470000446092B09D8DFE803F0050A2020202094
:10448000202020204088FFF7A3FD04B010BD144B6E
:10449000197819B3134B00791B7803F0010290428D
:1044A00006D86179C3F34003994294BF00210121EA
:1044B000012300226088FFF71FFE23788DF8043067
:1044C000043434F8023CADF8063094E8030004AB41
:1044D00003E9030001A8FFF723FBD6E70121E7E783
:1044E000D7BF0020D2BF002037B5174B174A5B88D3
:1044F0001188174C174D994208D852889A4205D313
:104500006369FBB900232B7003B030BD2B783BB13E
:104510006369002BF6D000228DF8042001A80FE07B
:104520000D490E480978D4E9012300290CBF114632
:104530001946FDF741F90028E4D0A369002BE1D02A
:104540009847DFE70122E7E74ABC002030BF0020A0
:10455000ACBB002048BB0020F8BF0020C8BB002037
:104560007BDF70477ADF704776DF704775DF704713
:1045700037B5164B18884FF6FF73984210D0144A7F
:10458000144D1378297B0133DBB2994213702C460A
:1045900008D31149FFF7EAFF10B1AB6903B198479F
:1045A00003B030BD002313702B7C33B13B21FFF7E8
:1045B000DBFF10B1AB6903B198476369002BEFD003
:1045C00000228DF8042001A8E9E700BFA8BB002065
:1045D000F8BF0020ACBB002030BF002065DF704773
:1045E0002DE9F74F0C9CBDF834B027880025804694
:1045F0008A4691462E46B8F80020B2420BDC35B10F
:104600002288013AD21B92B2FF2A39D8DA5500200B
:1046100003B0BDE8F08FD8F8042052F826000190CE
:1046200000220DF1030101A8FFF7D8FF0028EFD108
:104630009DF803204A4521D12288002D14BF002077
:10464000022002EB09010144594519DC3DB9013250
:1046500092B2228003F802A02288013222802288AE
:104660000DF103011A4401A8FFF7B8FF0028CFD1CC
:1046700021889DF803200A44228001250136BAE7EB
:104680000C20C5E72DE9F341089CBDF824501746DE
:10469000CDE9004502220646FFF7A2FF48B91022E5
:1046A00039463046CDE9084502B0BDE8F041FFF794
:1046B00097BF02B0BDE8F0812DE9FF4700231380CA
:1046C00090F82D3006460D4614463BB302A8FBF782
:1046D0003FF9002840F0FB8013880822CA54238841
:1046E00001339BB21B222380CA54238801339BB21F
:1046F000CA18DDF809102380E950BDF80D30938009
:1047000023889DF8082006339BB212F0FE0218BFE2
:1047100001222380EA54238801332380B378FBB13C
:10472000238804331F2B21D802A8FBF70FF9002898
:1047300040F0CD8023880322EA54238801339BB2C2
:1047400019222380EA542388BDF8082001339BB244
:10475000E9182380EA54120A4A702388023323801E
:10476000F278AAB12388D91C1F2901D90C20AEE008
:104770000221E954238801339BB201212380E954AB
:1047800023880B449BB22380EA5423880B44238064
:104790007268AAB12388D91C1F29E7D8022192F98F
:1047A0000020E954238801339BB20A212380E95475
:1047B000238801339BB22380EA542388013323806A
:1047C0003389002B76D1338A5BB11F23CDE90043B7
:1047D00007222B46032106F11000FFF753FF0028A4
:1047E00075D1338B5BB11F23CDE9004315222B46D6
:1047F000142106F11800FFF745FF002867D1326A3F
:10480000002A67D1776A4FB3BB882188981C8A1C1D
:1048100002441F2AAAD8FE28A8D803336B54238841
:1048200001339BB2FF222380EA54238801339BB2D9
:1048300023803A88EA54E918120A4A702088023024
:1048400080B22080BA884AB1B96800294AD0284489
:104850002EF070FF2388BA881344238096F82C30FA
:10486000002B79D1307890B33388012B3AD023884C
:104870009F1C1F2F3FF67AAF012805D172780232B4
:104880001A441F2A3FF672AFC3F11D039BB202A95F
:10489000E819ADF80830FBF757F8C0B93278022AAA
:1048A00040F09880BDF808209A4240F2AE80ADF802
:1048B000083098E01F23CDE9004306222B46022151
:1048C00006F10800FFF7DEFE00283FF47CAF04B0DD
:1048D000BDE8F0872788BB1D1F2B3FF647AF118827
:1048E000052901D80720F2E76FF4486C01EB0C03AF
:1048F0009BB24FF27D3C6345F4D95388052BF1D927
:104900006FF44860181880B26045EBD94FF6FF701D
:10491000814203D0834201D09942E3D80523EB556D
:10492000238801339BB212212380E9542388013369
:104930009BB223801188E954E818090A4170238842
:1049400002339BB223805288EA54E918120A4A7053
:1049500023880233238055E7B36A002BC2D04FF07F
:1049600000084FF00C094FF0160A96F82C305FFA49
:1049700088F293427FF676AFB16A09FB02F28F1894
:10498000BB88981CFE283FF6F1AE208803332B54D9
:10499000238801339BB2238005F803A023880133C9
:1049A0009BB223808A5AEA54E918120A4A70208876
:1049B000023080B22080BA884AB1B968002991D00B
:1049C00028442EF0B7FE2388BA881344238008F1C8
:1049D0000108CAE7012A7FF46AAF72789342FFF4B4
:1049E00066AFADF808200821BDF80830FE2B3FF671
:1049F000BDAE22880133AB542288013292B22280AC
:104A0000A95422881344238061E70921ECE70000C0
:104A100007B5144B1A686AB1002018601B68009330
:104A20004FF08042009B0123C2F808330E4A5370B6
:104A3000FAF790FF0D4B1A688AB100221A601B68C2
:104A40000193019B4FF080430222C3F80823064BD9
:104A50000120987003B05DF804EBFAF77BBF03B058
:104A60005DF804FB0001004094BB002004010040FD
:104A700013B5104B104C114800221A601B680193AB
:104A80002146019BFAF778FF88B9A27E0C48FF2ADD
:104A90001FBF012393404FF0A042C2F80835002306
:104AA00063762371236802B0BDE81040184702B056
:104AB00010BD00BF0831004008BB0020003000409E
:104AC0000CBB002070B52D4C86B094F821300193BA
:104AD00094F820300093E36904F1260204F12301E5
:104AE0004FF04020FAF779FF2346E0B994F82360AD
:104AF000A56906BB217B8A1E012A1CD8E0692269B0
:104B0000904218D16269E37BE261C5F34015032945
:104B100084F8203084F8215007D100954FF04021CF
:104B20002046FBF731F806B070BD4FF0402120461B
:104B3000FAF7CDFFF7E7124A07CA06AC04E9070007
:104B4000C6B14FF04021D1F8C424C1F8C424900765
:104B50000CD501228DF80820002283F824206A0752
:104B6000E1D4D3E9002102A89047DCE75107F3D54F
:104B70000222EFE78DF80860EEE700BFE0BA002000
:104B8000ECBA0020F7B515464FF0FF32C1F8082304
:104B900090F8242004460F4602F0FF0E2AB18368E5
:104BA000C1F80433112003B0F0BD012680F8246061
:104BB000836100F10C0C95E807008CE80700AA78E7
:104BC00084F820206A68E2616A78C7F888252A7824
:104BD000B24212D012B91E1C18BF012684F82160FF
:104BE0000096AB786A6839462046FAF7CDFF23680D
:104BF000002BD8D184F82430D5E784F821E0AB78B5
:104C00006A6839462046FAF762FFF0E7002343500E
:104C100082B043580193019B02B07047064A08B521
:104C20004FF492711046FFF7F1FF4FF48471FFF7D4
:104C3000EDFF0123136008BD0020004010B5CB7DBF
:104C40000A464FF4847123B9FFF7E0FFD0F8183516
:104C500010BDFFF7DBFF537ED168D0F81805C854AC
:104C6000537E0133DBB25376F2E70000F8B52C4CEB
:104C7000626822B12B4B4FF40171C3F80813E37D36
:104C80004BB1237E7BB322B1264B4FF40172C3F8A4
:104C90000423112026E00122E275E0606376A27E03
:104CA000237612B90BB9FFF7B9FF636873BB4FF4F2
:104CB000A2711C481B4E1A4FFFF7A8FFD6F82431EB
:104CC000D6F80821D6F8445182B90DB9002BF5D099
:104CD0000022E27503BB0DBBA17E124B012299B1EC
:104CE0001A600020F8BD20610123D8E7002BEFD126
:104CF000002DEDD139463046FFF7A0FF637EE27DFF
:104D00009A42DBD82B46E3E75A60EAE7054B4FF4BB
:104D10000172C3F80423E4E70320E3E70F20E1E78F
:104D2000C4BA0020002000400A4610B54FF48E712E
:104D3000FFF76CFF938A91689BB2C95C938A013339
:104D40009BB29382C0F81C1510BD000030B54A4AD2
:104D5000D2F8043313F4007F85B015464AD0D2F858
:104D60002431002B46D04FF492711046FFF74EFFCE
:104D70004FF40173C2F80833404B997E09B9012101
:104D800051603D4902228DF80020D1F88024C1F8FD
:104D900080240392DA7D8DF80820DA6801920022DF
:104DA000DA751A766846D3E9001290473248D0F88F
:104DB0001C313BB1314A938A917D994247D91146C2
:104DC000FFF7B2FF2C4AD2F844318BB14FF4A271F5
:104DD0001046FFF71BFF294B997E09B10121116095
:104DE000DA7D2AB10022DA75587ED968FAF7C2FB5B
:104DF00005B030BDD5F804335B07D7D5D5F80831F9
:104E0000002BD3D01D4C1C482146FFF717FF637EB3
:104E1000E27D9A422346C9D1227E52B12369E168DC
:104E2000E3600023607EE27523766376FAF7A2FBE7
:104E3000BCE7A27E0AB901226A600F4A4FF40171F1
:104E4000C2F808130022DA75587ED968EEE74FF4ED
:104E50008E71FFF7DBFE917D0029B3D000238DF822
:104E6000081091688DF80030019193756846D2E979
:104E700000139847A6E700BF00200040C4BA0020F6
:104E8000800000F1A040D0F8003723F44033C0F890
:104E90000037D0F8003743EA0141C0F800177047E7
:104EA00000F1804000F5C040002382B00360036839
:104EB0000193019B02B070472DE9F04F85B00024AB
:104EC000594D01944FF48072012102F1804303F5A2
:104ED000C04390B21B68012B06D1D5F804330B42B6
:104EE00002D0FFF7DDFF0C430432B2F5907F4FEAAA
:104EF0004101EAD14D4B1B68012B0AD14FF4BE7022
:104F0000FFF7CEFF4FF0A04344F00044D3F8103534
:104F1000019314F0FF0F1AD0454F012600253442AB
:104F200010D0AB0003F1804303F5C043D3F8100564
:104F3000D3F8101557F8253023B1C1F30141C0F360
:104F4000042098470135082D4FEA4606E7D1002C8A
:104F500063DA4FF0FF330022CDE90232344D354E93
:104F60000024A24601274FF0A04816F9012B531C3C
:104F700046D0D2B222F0C0094FEAD90104A80844B1
:104F800002F0070310F808CC07FA03F31CEA030F3A
:104F900036D005EB090C92099CF930C055F82CB0BD
:104FA000BBF1000F0AD1032A2AD10DF10C0E1EF815
:104FB00001C04CEA030C0EF801C001E0032AF4D052
:104FC00009F5E07110F80C0C58F821101842C1F3E3
:104FD000014105D0022913D1032A0BD1114604E067
:104FE00003290DD1032A05D102214846FFF748FFC6
:104FF0000134E4B2BBF1000F02D011464846D84755
:105000000AF1010ABAF1040FAFD134B14FF0A04355
:10501000019AD3F81035934202D105B0BDE8F08F64
:105020000193039B02939AE7006000407C6100407B
:105030006CBA0020BCBA00200028C3B2A8BF00F19F
:1050400060424FEA501010B5BABF0D4A03F00F048A
:1050500002F561424FEA41114FEA8000C9B200F106
:105060006040B4BF115582F8001300F5614003F0B1
:105070001F0201239340C0F88031036010BD00BFC0
:1050800014ED00E02DE9F8430446C279C17A0E2000
:105090001CF0EAF9237B644A0BB3537843F0100306
:1050A00053702568EB175906604B41EAD511680625
:1050B0004FF0FF328B4208BF82420AD35C4A002382
:1050C0002EF06CF900F5006020F47F6626F00F06E4
:1050D0004EB929465748BDE8F84322F057BB5378EC
:1050E00003F0EF03DCE720791CF032F940B9607976
:1050F0001CF02EF920B95048BDE8F84322F046BB19
:105100004E4F3B781BB100233B70FBF7FBF9257931
:105110004B4B002228461A701CF01AF920B14FF4AC
:105120004071284614F036FE657928461CF010F9C7
:1051300020B14FF49851284614F02CFE637A25795B
:10514000002B284614BF4FF00E094FF000091CF049
:10515000FFF800285AD03B4B05EB45051D4495F858
:105160000180647920461CF0F3F8002851D0354BBB
:1051700004EB44041C446378334CE27E002A4BD198
:105180005A1C0AD04FF0A04101229A40C1F80825CC
:1051900003F5E072032041F82200B8F1FF3F2B4DE8
:1051A0001FBF4FF0A04108F5E072002041F8220037
:1051B000C5F82465C5F86C950026C5F81485C5F8B2
:1051C0000C35234B636028464FF48E712660FFF741
:1051D0001DFD4FF4A271FFF719FD1E4BC5F80433F6
:1051E00002210846FFF728FF0423C5F80035B8F16F
:1051F000FF3F4FF48073E6822676638310D0FFF77B
:105200000DFD0123A37614F019FA09E04FF0FF38E1
:10521000A7E74FF0FF33AFE708210F4822F096FAD7
:1052200001233B70BDE8F88314BA002047E8010071
:1052300048E801004339050058390500F1C0002055
:10524000F2C00020243A0500C4BA0020002000402B
:1052500075960300800002006E390500F8B50E4611
:10526000D11C48BF911D144641F387010546671EB6
:10527000FAF7A3FD00214AB2A24201F1010100DBCD
:10528000F8BDBB1A23F00300B25C03F00303DB009C
:1052900002FA03F32A581A432A50ECE7F0B5002526
:1052A0004F1E6CB28C4205F1010500DBF0BD3B1BCB
:1052B00023F0030603F003039659DB0026FA03F3F9
:1052C0000355EEE72DE9F041B3F9024014F11F0553
:1052D00048BF04F13E050F4603F1240645F3471588
:1052E000904601462B4632463846FAF7A1FDB8B93A
:1052F000B4EB451F16DA6211012304F01F0403FA10
:1053000004F457F822301C4214BF012400242B4619
:10531000324639464046FAF78BFD2046BDE8F0811B
:105320000124F4E70446F2E710B500231A465CB204
:10533000A14203DCB2FA82F0400910BD50F82340CC
:1053400001332243F3E700002DE9F04F8A46234F53
:105350008BB00646114650461446FAF70EFD3B68E0
:10536000FBB10425C0EB441014FB05FB00B205FBA8
:1053700004654FF0FF38043D28FA00F84FF040096B
:105380003B6859463046984758B12B6803EA0803F2
:105390002B6021463046FFF7C7FF20B1B9F1010964
:1053A000EED1002017E023463246514602A8FAF714
:1053B0000FFD2146019002A8FFF7B6FF019B0033C5
:1053C00018BF01235B00002814BF5842C3F101003D
:1053D000C0B20128E2D10BB0BDE8F08F6C2D0020E7
:1053E0002DE9F04FD1B0CDE905015B9D95F9004065
:1053F00048A8914622461F46FAF7B3FCA30007933C
:10540000069BA20013441946224638A80293FAF7D5
:10541000A8FC95F90060002F00F08C8032463946D8
:1054200028A8FAF79EFC0DF5807A324630AF48A9DD
:105430005046FAF796FC38A93846FAF792FC2B4604
:1054400028AA38A948A8FAF74BFC2B4628AA38A95D
:1054500048A8D5F8A460B0472B4628AA394650463C
:10546000FAF73EFCBDF968310497023B1BB2002BF2
:1054700067DCD9F80030009503F001084FEA4818BE
:1054800040AADB4302EB080A03F0010330AA904470
:105490005B0140AA1A44039230AAD3184146039AEA
:1054A0000493504605F10409FAF7B9FE4B4640AAA9
:1054B00048A908A80094FAF722FE08A908462B4636
:1054C0004246FAF7CCFB08A908462B46069AFAF79B
:1054D000C6FB214608A8FFF727FF00285DD008A8D3
:1054E000FAF76BFC08A92B46029A0846FAF7B7FBB5
:1054F00008A92B4652460846FAF7B1FBDDE903013D
:10550000434652460095FAF70CFE2B4608AA30A9EE
:1055100040A8FAF7E5FB224640A90598FAF721FCD6
:10552000059B079C234430A91846FAF71AFC51B092
:10553000BDE8F08F314628A8FAF73FFC01232893F5
:1055400071E71FFA83F85B1108F01F0259F8233046
:105550000095012101FA02F21A42049B13BF202791
:105560000027202600260AEB070B1F440AEB060340
:105570000393049B039A1E44334639465846FAF770
:105580004EFE08F1FF383B4600955A4631460398D7
:10559000FAF7C7FD0FFA88F369E710AF224608A9AA
:1055A00038460DF1600BFAF7DCFB20AE4946584651
:1055B000FAF7D7FB30462146FAF7FFFB012328A86C
:1055C0002093FAF7FAFB224659463846FAF7B4FB1D
:1055D00028B9224620A908A8FAF7C3FB82E73B684E
:1055E000DA0709D421463846FAF799FB224649469C
:1055F0003046FAF768FDE6E7189BDB0707D421463B
:105600005846FAF78CFB2246494628A8F1E70028BD
:1056100023461CDD5A4639463846FAF7D9FB21465F
:105620003846FAF77CFB224628A93046FAF784FB75
:10563000002805DA23464A4631463046FAF7F8FB99
:10564000234628AA31463046FAF7C2FBCEE73A464F
:1056500059465846FAF7BCFB21465846FAF75FFB15
:105660002246314628A8FAF767FB002805DA28A960
:1056700023464A460846FAF7DBFB28A9234632466A
:105680000846FAF7A5FBBEE72DE9F04793F900605D
:1056900092B0044689461046314615469846FFF7B3
:1056A00043FE002840F09180424649460AA8FAF796
:1056B00013FB43460AAA214602A8FAF7D0FA0AA920
:1056C00008464246FAF708FB43462A4649464846FA
:1056D000FAF7C5FA08F10407424629462846FAF7C0
:1056E000FBFA3B462A46214620460096FAF77EFD05
:1056F0003B462A46294628460096FAF777FD3B4660
:105700002A46214628460096FAF7F9FC43462A46DF
:1057100021462046FAF7A3FA3B4622462146284670
:105720000096FAF763FD3B4600962A46214620463E
:10573000FAF75CFD2368DB074AD533463A46214633
:105740002046FAF775FB314682462046FAF7E7FA1B
:1057500006F18043013B54F8230040EACA7044F844
:105760002300424621462846FAF7B6FA3B4602AAEB
:10577000294628460096FAF7C2FC3B4602AA29466B
:1057800028460096FAF7BBFC02A908463B462A4683
:105790000096FAF7B4FC434602AA21462046FAF7DF
:1057A0005EFA0AAA3B46104621460096FAF7A7FC85
:1057B000324629462046FAF7D4FA49462846FAF7EF
:1057C000D0FA0AA94846FAF7CCFA12B0BDE8F08739
:1057D00031462046FAF7A3FAC3E7000073B5002369
:1057E0000DF102008DF80230FBF7AEFB264B1B7863
:1057F00003F0FF04002B41D1244B1A68002A3DD04E
:10580000234AD2F80813C90738D51C601B68214DFC
:1058100001930DF10300019BD2F808658DF8034058
:10582000FBF792FB6A6829681F2A98BF541CA142A3
:10583000F6B26C6004D1202C14BF611C00212960D9
:1058400015499DF803008E542A6894423ABFC2F16C
:1058500021021319A31AAA689A4238BFAB60FBF75A
:1058600095FF6B682A681F2B94BF013300239A426F
:1058700001BF074A0123C2F8083353609DF80200B4
:10588000FBF784FF02B070BDD8BF002000D10040FC
:1058900000D00040C4BF0020A0BF002030DF704710
:1058A0002DE9F74F3B4F06468846B8F1000F03D16C
:1058B000012003B0BDE8F08F4546202D28BF2025EC
:1058C0005FFA85FB002400230DF102008DF8023001
:1058D000FBF73AFB304B1B7803F0FF0993BB0DF14C
:1058E00003008DF80390FBF72FFBD7E900148C42DF
:1058F00004D3641AA54207D9052414E02134641A9C
:10590000A542F9D8C1F12104244BA542194431D84C
:105910002A4630462DF00EFF3B682B44212B28BF32
:1059200000233B6000249DF80300FBF72FFF1C4B76
:1059300000221A601B680193019B1A4B0122C3F8D5
:1059400004231A609DF80200FBF720FFB9F1000F55
:1059500008D059463046FFF7A1FF42F207039842AC
:105960000446ADD0022CAED0002CA9D1A8EB05087E
:105970002E449AE7224630462DF0DCFE074BA5EB7D
:10598000040A5246194630192DF0D4FEC7F800A07B
:10599000C8E700BFC4BF0020D8BF0020A0BF0020C0
:1059A00000D1004000D0004017B4314A314B11689B
:1059B00089B90021304A106820BB00205A79D407E9
:1059C00040D408B9002949D01C68DA88234603B0BE
:1059D0005DF8044B1847002111601268D9680092E5
:1059E000009A0029E5D0254AD2F84005814204BF3B
:1059F000D88801EB8001C2F840155A7942F00402C0
:105A00005A71D7E700201060126898680192019AD5
:105A10000028D2D0194AD2F83845A04204BFDC8809
:105A200000EB8400C2F838055A7942F002021407EC
:105A30005A71C3D512F0010402BF64F3C3025A7154
:105A40002046BBE702F00601062907D122F0060234
:105A500011075A7106D56FF3C3025A7103B05DF88E
:105A6000044B7047054AD2F83805D2F84015ABE729
:105A7000145102405CBA0020045102400050024020
:105A8000A5DF7047A4DF7047A3DF70472DE9F0471B
:105A90000E4690B016F01005814692469846189C26
:105AA0000CD011238DF8083023788DF809300122AD
:105AB0004FF0000362F342038DF80A301C220021EC
:105AC00009A8F9F72FFD8DF8246005B102AD42F663
:105AD0004D23ADF80C3063789DF864108DF80430D8
:105AE0000022A3788DF80530134661F3C303DBB2BF
:105AF00043F00303CDE906220E95012701AD8DF891
:105B00000630089203AE1A9BB9F800008DF80E70AB
:105B100004AA09A9CDE90465ADF81CA0FDF728FD8C
:105B200058BB42F60813ADF80C3063788DF804309A
:105B3000A3788DF80530034667F342038DF80630ED
:105B40001A9A98F800308DF8003098F80130CDF8A6
:105B50001A00ADF81E008DF8013032F8080B8DF8F0
:105B60000E70022304A9CDE90465ADF81830ADF834
:105B70001C30CDF820D0FFF787FF10B0BDE8F087CC
:105B8000A1DF704708B5FAF723FC10B1774B784ACC
:105B90001A60FAF7FDFB28B1764B774A1B68C3F30E
:105BA00042331360FAF714FC20B1744AD36823F02F
:105BB0008073D360FAF7ECFB40B14FF080430022D2
:105BC000C3F80C21C3F81021C3F83825FAF700FCFC
:105BD00010B16B4B03221A60FAF7FAFB40B1694B24
:105BE00005221A6001229A6700229A603F225A60B9
:105BF000654B1B78062B50D1644B1B6819074CD1A1
:105C0000634B1B6803F0F003502B46D14FF08052DA
:105C1000604BD2F80414C3F82015D2F80814C3F866
:105C20002415D2F80C14C3F82815D2F81014C3F8B0
:105C30002C15D2F81414C3F83015D2F81814C3F880
:105C40003415D2F81C14C3F84015D2F82014C3F848
:105C50004415D2F82414C3F84815D2F82814C3F810
:105C60004C15D2F82C14C3F85015D2F83014C3F8E0
:105C70005415D2F83414C3F86015D2F83814C3F8A8
:105C80006415D2F83C14C3F86815D2F84014C3F870
:105C90006C15D2F84424C3F87025FAF779FB28B1C3
:105CA0003D4B3E4A1B6803F04F0313603C4AD2F859
:105CB000883043F47003C2F88830BFF34F8FBFF3CE
:105CC0006F8F4FF01023D3F80C22D2071ED5354B1F
:105CD0000122C3F80425D3F80024002AFBD04FF09A
:105CE0001022D2F80C3223F00103C2F80C322D4BF3
:105CF0001A46D3F800140029FBD00021C3F804157C
:105D0000D2F80034002BFBD004F0CCFAD3F80022F8
:105D1000002A03DBD3F80432002B23DA214B0122C3
:105D2000C3F80425D3F80024002AFBD04FF010223A
:105D30001521C2F80012D3F80024002AFBD04FF03E
:105D400010231522C3F80422164B1A46D3F8001468
:105D50000029FBD00021C3F80415D2F80034002B31
:105D6000FBD0D1E7104B114A1A6008BD74C0074040
:105D70000DF0ADBA440200103C050040F0ED00E02B
:105D8000A005004010560040E00F00F0E40F00F0C6
:105D9000E80F00F000C0004058020010E40E004080
:105DA00000ED00E000E00140A42C00200090D003B2
:105DB0007047704700207047704770478DDF70470D
:105DC00077DF704701381F289DBF034B23FA00F08F
:105DD00000F00100002070478B80808030B551ECCE
:105DE000100B85B053EC112B8DED000B55EC124BC5
:105DF0008DED021B2DF0FCF99DED000B28B19DED02
:105E0000021BB0EE410AF0EE610A53EC102B204663
:105E100029468DED000B2DF0EBF99DED000B08B13F
:105E200045EC104B05B030BD38B555EC104B002299
:105E3000002310EE100A29462DF0DAF910B105F111
:105E400000431D4645EC104B38BD436833B1013B60
:105E5000436003685A1C0260187870474FF0FF30A7
:105E600070470B685A1C0A60187070472DE9F04F94
:105E700089B00E4600AF0023044607F114013046F6
:105E80007B6126F06CFF054618BB304623F0B4FD5D
:105E90008046786120F0CEFA08F5807383420CD9F1
:105EA000A649012021F0B4FD3246A549012021F088
:105EB000AFFD2437BD46BDE8F08F08F1070323F09E
:105EC0000703ADEB030D6D4642462946304623F0ED
:105ED00083FD7E6926B99B49012021F099FDE8E701
:105EE0004FF00308B6FBF8F303EB43039E4201D0E7
:105EF0009549F1E720461BF02BFA08B99349EBE7E7
:105F0000934BC7F808D004EB44041C446178914CCF
:105F10002079002840F009818F4A0123C2F8040546
:105F2000FF29C2F82405C2F82005C2F81C35C2F8C2
:105F30002805C2F818054FF0C050C2F81405C2F881
:105F4000103518BF01F5E0704FF0A04308BF4FF0C7
:105F5000FF31C3F85887C3F8FC8A18BF43F8208084
:105F60001623C2F86435FF23C2F868354FF0FF33BB
:105F7000C2F860352520C2F87015C2F86C350221D0
:105F8000764B2360FFF758F8012323710323B6FBF8
:105F9000F3F39BB203EB430808F1010828F0010278
:105FA0009100ADEB010D6846FA606D4A3A60411808
:105FB0004FF0000C796082F800C0E91C4FF0EE0948
:105FC000851C4FF0880A4FF08E0B63455FDC0C2276
:105FD00002FB030300227968994200F29E80267931
:105FE000012E40F0A28000F06043B3F1005F40F06A
:105FF000A280FB68C3F34E02574B0021C3F8502523
:10600000C3F83815C3F80815C3F84005C3F80C6584
:106010006579E28025F0090545F008056571C4E958
:106020000210C3F80065022323710D46002977D0C2
:106030004FF6FE7208EA0202F9F774FA494B0022A1
:106040001A601B68FB61FB69474B1A601B68BB61E8
:10605000BB69414B2222C3F8042301221A603A682B
:106060001278042AFBD94149002222250120C3F8D5
:1060700008530860C3F80025C3F808530860C3F844
:1060800000253B4B2021C3F88410227150E011F809
:10609000026C11F8032C360246EA024611F8012C74
:1060A00005F10C0E164306F44012B2F5001F1ED087
:1060B000B2F5401F20D0B2F5801F20D105F802BCF8
:1060C00006F44002B2F5000F1CD0B2F5400F1ED00E
:1060D000B2F5800F1ED105F801BC0235AE454FEA7E
:1060E0000616E0D10CF1010C033175466DE76FF037
:1060F000170205F8022CE3E705F8029CE0E705F833
:1061000002ACDDE76FF0170205F8012CE5E705F8B2
:10611000019CE2E705F801ACDFE703F8012B5AE741
:10612000014623682846984788E70820FBF7CCFA01
:10613000D7F808D0BDE61020F8E700BFB938050051
:106140002B4505005745050077450500A24505008C
:10615000243A05005CBA002000500240811B030075
:1061600005C1002004510240145102400450024075
:1061700000E100E0024B03495868002227F060BEAE
:10618000582D00202C76050070B5002216490546D2
:1061900027F056FE28F0BAF9144B1549064603229B
:1061A000586827F04DFE044678B10022B1B227F0BE
:1061B00079FDE389A3F500739BB2E381E38903F4DE
:1061C000F05313B9204626F095F80A4B1C6824B109
:1061D000E38903F500739BB2E3812846002110F0A8
:1061E00033FA204670BD00BF193C0500582D002031
:1061F000263C0500F4C0002008B540B2FFF7E0FDE2
:10620000BDE8084012F0ACBE38B5054608460C465D
:1062100025F0B3FE002808BF002422460E49284678
:1062200027F0B4FD0D4B4FF6FF72198874B18A4206
:1062300004D10020BDE8384012F092BE0022188838
:10624000114613F027F80828F4D1F2E78A42F0D07B
:10625000188813F01DF8F6E7F43B0500B42C002075
:10626000014B188810F0FABAB42C0020014B1888A2
:1062700010F0F4BAB62C002008B5074B1A884FF678
:10628000FF71914207D018881321FEF76DF9BDE820
:10629000084012F065BE08BDB62C002007B50023EB
:1062A0000846072269460093CDF8033028F0C6FB64
:1062B000094B1A884FF6FF71914209D018886A4637
:1062C000012112F0E9FF12F04BFE03B05DF804FB70
:1062D00043F20200F7E700BFB42C002038B50022DB
:1062E0000E49054627F0ACFD0446A8B90C491CF040
:1062F00031FE0A4904460246284627F047FD2A4651
:106300000849204627F042FD002025F0F5FB06490C
:106310000246204627F05BFD204638BDCE3B0500F7
:10632000D33B0500ED3B05000F3C050010B50446CE
:1063300025F00BFE224630B92CB107490320BDE8F9
:10634000104021F065BB054B0549586828F0CAF993
:10635000BDE8104012F01EBE80400500582D002000
:10636000A9400500F8B5044628B9214A136823F46A
:1063700080431360F8BD1F4926F070FA0028F4D15D
:10638000204625F00AFE054690B1194A13682046BA
:1063900043F48043136028F0E5FB53EC102B10EE20
:1063A000100A194617F0FCFDBDE8F84012F0D8BD00
:1063B000204625F0CAFD0028DCD00D4A0E4913689E
:1063C00043F48043136020462A4627F039FD28F025
:1063D0003BFC2A4606460F462046084927F030FD7A
:1063E00028F032FC02460B4630463946DAE700BF59
:1063F000F8C00020473F05004C3F0500583F05000E
:10640000084B1A6818B142F400521A60704722F41F
:1064100000521A60044B1860044B01221A7010F0ED
:10642000D7B800BFF8C0002008C1002007C1002075
:1064300010B5044625F0A1FD084B0949002808BF06
:1064400000242246186827F0A1FC201C18BF012058
:1064500010F07AFCBDE8104012F082BD582D0020EB
:10646000F43B05002DE9F74F504B514905460322F7
:10647000586827F0E5FC0646002845D000224D4923
:10648000DFF83081284627F0DBFC3146814668463C
:1064900020F0CBFA009CECB1204627F071F90022E5
:1064A0004146074627F0CCFC01230022494682469C
:1064B000FAF762F958BBFB8903F500739BB2FB81C5
:1064C0003C465046394627F07FF8684620F098FA57
:1064D000002CDFD0009850B1C389A3F500739BB2A4
:1064E000C381C38903F4F0530BB925F003FF294698
:1064F000002C57D001A820F098FA019D4DB93246E2
:106500004946204627F034F803B0BDE8F08F002458
:10651000D7E7EB8903F500739BB2EB81284627F0A0
:106520002FF9012229460746204627F0FDFD224982
:106530008046284626F092F920498246284626F0D1
:106540008DF9BAF1000F00D1D0B1404627F018F90B
:10655000834610B3BAF1000F1BD00122394627F051
:1065600014FBBBF80E20A2F5007292B2ABF80E201D
:10657000BBF80E2002F4F05212B9584625F0BAFECC
:1065800040463A46294626F0F3FF01A820F038FAA3
:10659000B3E7394627F025FEE3E73946404626F0C3
:1065A00019FFEDE7304627F0B3FAA8E7582D002091
:1065B000FB3C0500553E0500023D05000B3D050076
:1065C000F8B5064608460C4625F0BFFC074620B342
:1065D00000223949204627F033FC28F0FEF800223B
:1065E00007463649204627F02BFC0446E0B125F04B
:1065F000A4FCC8B9E389A3F500739BB2E381E389E6
:1066000003F4F05313B9204625F074FE22462C49BA
:106610000320BDE8F84021F0FBB92CB122462949FE
:10662000032021F0F5F93C46304625F0A6FC002871
:106630003AD0002E38D048F24801234825F0ABFA72
:106640000546D0B12246002127F094FE32461F496C
:10665000284627F09BFB1E4B1E4918682A4627F048
:1066600095FBEB89A3F500739BB2EB81EB8903F4F7
:10667000F05313B9284625F03DFE301C18BF012009
:10668000394610F08BFB12F06BFCA4B1E389A3F543
:1066900000739BB2E381E38903F4F0535BB92046B6
:1066A000BDE8F84025F026BE094B0A49186827F0D6
:1066B000FFFF0026E1E7F8BD6E3F0500173E05002D
:1066C000753F0500A93F0500DD680200C23F0500D7
:1066D000582D0020C73F05002DE9F84380460C46A1
:1066E00025F04BFC30B9384942460120BDE8F8435B
:1066F00021F08EB9204625F050FC05462046C5B154
:1067000028F030FA57EC106B002432463B463046F6
:1067100039462CF095FD30B900222C4B30463946D5
:106720002CF066FDC8B12A490120BDE8F84321F0EC
:106730006FB925F00AFC50B12A462649204627F0B9
:106740007FFB40B128F080FA06460F46DDE714B122
:1067500022462149C9E7214F0026214DD5F8049052
:1067600025F023FA1F490246484627F030FB4246EF
:106770001D49686827F00AFB08211C4825F00BFA20
:10678000054670B12146FFF71BFFEB89A3F50073A7
:106790009BB2EB81EB8903F4F05313B9284625F043
:1067A000A9FD0021124825F0F6F9044648B1002160
:1067B00047EC106B0CF010F82146BDE8F84326F0CA
:1067C00003BFBDE8F88300BF913C050000002440F2
:1067D000E23C0500EA3C0500BF3C050000409F404C
:1067E000582D0020FB3C0500F23C050065640200CA
:1067F000F567020037B5144C00210846FFF7E0FEAC
:1068000003221249606827F01BFB00220190104907
:10681000606827F015FB0D490546606827F048FFC2
:106820000B49606827F044FF019B33B12DB1012370
:1068300001AA294600201AF0CBFB2946019826F030
:10684000C3FE03B030BD00BF582D0020FB3C050047
:10685000F23C05001FB54FF08052D2F8A430D2F8B8
:10686000A820D8B20290C3F307200190C2F30721F9
:10687000C3F3074000901B0ED2B241F0C0010348A1
:1068800026F018F905B05DF804FB00BF173D0500C0
:1068900038B5044625F059FBD8B100220E492046F0
:1068A00027F0CEFA054625F003FC10B1284626F065
:1068B000F9F904465DB1EB89A3F500739BB2EB8156
:1068C000EB8903F4F05313B9284625F013FD204655
:1068D00038BD0446FBE700BFF73905002DE9F04F4E
:1068E0008BB000AFC7E902011446002A76D09E495A
:1068F00000201CF02FFB0022054638619B492046F2
:1069000027F09EFA99490246284627F060FA0022AD
:1069100097493D69204627F093FA95490246284653
:1069200027F055FA25F041F9804605F043FB002297
:1069300083469049204627F083FA8146E8B1024613
:106940008C49386927F022FA002307F124014846D0
:106950007B6226F004FA044600284ED1484623F014
:106960004BF8054678621FF065FD05F5807383429C
:1069700038D98149012021F04BF8B8F1000F07D038
:10698000D8F8003023B142467C49386927F0FEF937
:10699000584626F0BBF920B15A467949386927F0A4
:1069A000F5F95A464146484626F0E2FDFB68002BC1
:1069B00040F0C08007F1100301220021B8681CF0EC
:1069C000F7F9386950B1C389A3F500739BB2C3814D
:1069D000C38903F4F0530BB925F08CFC2C37BD466A
:1069E000BDE8F08FEB1D23F00703ADEB030D6C4604
:1069F0002A462146484622F0EFFF7B6A002BBCD096
:106A0000B8F1000FC4D0BBF1000FB6D0002514E0E0
:106A1000092A09D1A91C2144701ED7F810A026F01C
:106A200007FC5849024619E0911E012927D89A46C9
:106A300002239E4216DA013635447B6AAB429CD96A
:106A40006319665D5A78082AE2D1A91C2144701E98
:106A5000D7F810A026F0ECFB4B490246504627F031
:106A6000B6F9E8E73AF8021F48487B6026F022F8BA
:106A70000146404627F0BEF87B680233D9E7911FF4
:106A8000012908D8A81C204413F0CCFE014640463A
:106A900027F0B0F8CFE7162A33D159883B4826F0C3
:106AA00009F828F026FB82460028C4D001220146BE
:106AB000584627F039FB291D78602144F01E23F049
:106AC00021FA7B6802463BB130B101463860184676
:106AD00026F080FCD7E900231846114626F074FD05
:106AE000BAF80E30A3F500739BB2AAF80E30BAF8CC
:106AF0000E3003F4F053002B9DD1504625F0FAFBE5
:106B000099E7FF2A97D1D8789B78D7F810A043EA65
:106B1000002024F0F9FF1E490246504627F057F99D
:106B2000291D2144F01ED7F810A023F0EBF91949D4
:106B3000024693E7D7E9031607F114001FF075FF2B
:106B4000786948BB0446786950B1C389A3F50073DE
:106B50009BB2C381C38903F4F0530BB925F0CAFB80
:106B6000002C7FF427AF2CE738400500553E050088
:106B7000FA3B0500DB380500B9380500023D050089
:106B80000B3D05005240050048400500CE7405004D
:106B9000574005006440050026F0F2FD0022BA4986
:106BA000054627F04DF98046002800F00F810022AD
:106BB000B549304627F044F94146814607F11800AF
:106BC0001FF033FF0124B869002840F0CC8049460B
:106BD000404626F0F9FC0022AC49284627F030F95F
:106BE0008046E0B10022A949304627F029F98146C4
:106BF000404625F0A4FA002800F0EA80484625F037
:106C00009EFA002800F0E4804946404626F062F9EA
:106C100000284946404608BF002426F0D5FC002243
:106C20009B49284627F00CF9804610B3002297496B
:106C3000304627F005F98146404625F039FA98B1EB
:106C4000484625F035FA78B1404626F02BF88246C2
:106C5000484626F027F8824506D8012300224946F7
:106C60004046F9F789FD00B100244946404626F028
:106C7000ABFC00228749284627F0E2F8804680B125
:106C800000228449304627F0DBF801468146404621
:106C900026F020F949460028404608BF002426F087
:106CA00093FC00227C49284627F0CAF88046F0B1C0
:106CB00025F04BF960B1414607F124001FF0B5FE05
:106CC000DFF8D4A1D7F824B0BBF1000F40F09480D6
:106CD000B8F80E30A3F500739BB2A8F80E30B8F8E0
:106CE0000E3003F4F05313B9404625F003FB0022A5
:106CF0006A49284627F0A4F88046F0B125F025F926
:106D000060B1414607F124001FF08FFEDFF894A127
:106D1000D7F82490B9F1000F40F09980B8F80E3000
:106D2000A3F500739BB2A8F80E30B8F80E3003F448
:106D3000F05313B9404625F0DDFA5DB1EB89A3F5B8
:106D400000739BB2EB81EB8903F4F05313B928462F
:106D500025F0D0FA07F114001FF052FE002C3FF48A
:106D6000EFAE0124EFE6B9F1000F12D026F008FDD6
:106D7000014607F11C0013F0D1FC494607F1200041
:106D80001FF053FE4FF0000A386A40B9BAF1000F05
:106D900000D1002407F118001FF032FE13E726F09F
:106DA000EFFC014607F1240013F0B8FCBA7F97F816
:106DB00026309A4205D1BA8BBB8C9A4208BF4FF05D
:106DC000010A07F120001FF01BFEDDE7012402E7A6
:106DD000334BA8EB03000011013082B2B9F1000F70
:106DE00008D0A9EB03000011013080B2131A5842F9
:106DF00058410DE74846F9E7BBF80E3003F500733C
:106E00009BB2ABF80E3000225146304627F018F8FE
:106E1000814648B900245846494626F0D5FB07F17B
:106E200024001FF0EDFD4DE70022594627F07CF9C4
:106E30000028EFD0C389A3F500739BB2C381C38937
:106E400003F4F053002BE6D125F054FAE3E7B9F848
:106E50000E3003F500739BB2A9F80E3000225146A4
:106E6000304626F0EDFF83460146484626F032F8CC
:106E700059460028484608BF002426F0A5FB07F124
:106E800024001FF0BDFD43E7023D05005240050010
:106E900075400500553E05000B3D050064400500AA
:106EA000742D0020574005002DE9F04186B000AF59
:106EB00000238846391D06467B6025F050FF0546B5
:106EC000E0B9304622F098FD044678601FF0B2FA2F
:106ED00004F58073834206D93F49012020F098FDD4
:106EE00032463E4938E0E31D23F00703ADEB030DC6
:106EF0006D4622462946304622F06EFD7B68002B07
:106F0000EED0404625F039F828B1354B35491868A0
:106F1000424626F03BFF344B1A6812F0400F1E46E3
:106F200007D13249012020F073FD1837BD46BDE876
:106F3000F0812F4A12884FF6FF71914201D12D49FD
:106F4000F0E71A6812F0800201D02B49EAE77C686A
:106F5000102C05DD29491022012020F059FDE4E71D
:106F6000274B93F800C0274BA4B2BCF1000F23D1EC
:106F70009A7C62B3B3F8760188422AD09B8A7C80DF
:106F8000C7F80AC0A7F80EC03B810123BB7207F106
:106F90000801BB1CC7E90435FCF7E8FA18B97B887F
:106FA000A34218BF0C2011F0DBFF0028BDD13368CD
:106FB00043F080033360B8E7B3F87601884208D025
:106FC0007C80C7F80A20FA81B3F84E31DCE707204D
:106FD000E9E70820E7E700BFB9380500BE3E050035
:106FE000582D00204E3E0500F8C00020583E0500F8
:106FF000B62C00206C3E05007B3E0500933E05004C
:1070000006C100208CBC00202DE9F04FB04B91B0A0
:107010001B681B0700AF044607D5AE49012020F0CE
:10702000F7FC4437BD46BDE8F08F17F033F8204633
:1070300024F08BFF8046002800F05E81214607F196
:1070400014001FF0F2FCDFF8ACA2796981B10023D3
:10705000BB61CB8903F500739BB2CB8107F11800AC
:1070600013F05CFB024698B19B49012020F0D0FC54
:1070700078690028D5D0C389A3F500739BB2C3817A
:10708000C38903F4F053002BCBD125F033F9C8E7C3
:107090007D691DB1284626F073FB0546294607F198
:1070A0001C001FF0C2FCF969B8F1000F0FD071B1DC
:1070B000CB8903F500739BB2CB8107F1200013F05D
:1070C0002DFB024610B38549012020F0A1FCF86990
:1070D00050B1C389A3F500739BB2C381C38903F484
:1070E000F0530BB925F006F95DB1EB89A3F50073F8
:1070F0009BB2EB81EB8903F4F05313B9284625F0DA
:10710000F9F807F114001FF07BFC9EE707F1280057
:107110003C8C97F8226013F0C5FB08B1FAF7D4FA5B
:107120004FF00009002207F13001388DC7F8309088
:1071300013F0B6FB052810D043F2030290420CD0A6
:10714000A8B93B8EA34214D197F83230B34210D184
:10715000B7F82890B9F1000F0FD1386A13F078FB17
:107160005F4904460246012020F052FC48E0FAF74D
:10717000ABFA3B8D01333B85D4E7FC691CB120465B
:1071800026F0FEFA044600225649204626F058FE14
:10719000002255490646204626F052FE27F01DFBE8
:1071A0000022B8605149204626F04AFE27F015FB20
:1071B000F8602EB3002307F1240130467B6225F0EE
:1071C000CEFD8346002837D1304622F015FC786288
:1071D00078601FF02FF97A6802F58073834221D915
:1071E0004349012020F014FCF389A3F500739BB2FE
:1071F000F381F38903F4F05313B9304625F07AF89C
:107200005CB1E389A3F500739BB2E381E38903F4E6
:10721000F05313B9204625F06DF807F11C001FF05C
:10722000EFFB40E7D31D23F00703ADEB030DEB4667
:107230005946304622F0D0FB7A6A002AD4D0002189
:1072400079853A85494607F12802BAF80000C7F85F
:107250002CB0FEF717FC11F083FEBB6880F0010034
:107260005FFA80F813B9FB68002BBDD0BAF8002094
:107270004FF6FF719142B7D0FB68BAF80000A7F84B
:1072800030900022002BC7F83220FA867A6A7A8280
:1072900014BF0222012287F8322007F1300107F1E2
:1072A0001202C7E90E2BFCF761F930F008029BD0FF
:1072B00043F20402904297D043F20142904293D0AD
:1072C00011F04EFE002818BF4FF000088CE700BFF9
:1072D000F8C00020164105003E4105005741050059
:1072E00087410500C2450500774105007E41050044
:1072F000B9380500B62C0020002C3FF492AE22468F
:107300000249032020F084FB8BE600BFAB4105005F
:107310002DE9F04F9BB000AF0D4604463C22002102
:1073200007F12C00F8F7FEF8022387F82C302846E6
:10733000062387F82F3024F008FE002800F08D8007
:1073400000228E49284626F07BFD38B127F045FA09
:10735000002814BF0223002387F82C30002288491C
:10736000284626F06DFD38B127F037FA002814BF03
:107370000623052387F82F3000228249284626F06D
:107380005FFD064618B3002307F10C01FB6025F0F2
:10739000E6FC804600284ED1304622F02DFB814687
:1073A000F8601FF047F809F58073834237D97649B2
:1073B000012020F02DFBF389A3F500739BB2F3812C
:1073C000F38903F4F05313B9304624F093FF2846B1
:1073D00000226E4926F034FD054690B13B6D002B2E
:1073E00036D026F0FDF93B6D1880EB89A3F50073CC
:1073F0009BB2EB81EB8903F4F05313B9284624F0D8
:1074000079FF204624F099FD80B3E38903F50073EA
:107410009BB2E38120466C37BD46BDE8F08F09F191
:10742000070323F00703ADEB030DE8464A46414648
:10743000304622F0D1FAFA68002ABCD084B06B46FC
:107440004FF6FF713B6519809A80C3F80880B2E758
:107450004F49032020F0DCFAC7E7002DD1D04D4979
:107460002A46032020F0D4FA0024D3E7204624F053
:1074700048FD06460028C8D1204624F066FD0028B5
:1074800076D0204625F03CF90C235843073020F0F5
:107490000700ADEB000D214607F108001FF0C5FA0B
:1074A000E946DFF8E4B04D46B246B868C0B987F89F
:1074B0005860C7F854901F2307F1080207F10C0128
:1074C00007F12C003B81FDF7F7F811F049FD00288A
:1074D000CAD107F10C01388922F014FD044699E75E
:1074E00026F04EF907F10C010446C7F80CA025F070
:1074F00036FC804678B9204622F07EFAF860786043
:107500001EF098FF7A6802F58073834225D95946A8
:10751000012020F07DFA5CB1E389A3F500739BB2F2
:10752000E381E38903F4F05313B9204624F0E2FE2B
:10753000B86820B1C38903F500739BB2C38126F0FC
:10754000E5FFFB682880AB80C5F8088007F10800DC
:107550001FF056FA01360C35A7E7D31D23F00703B9
:10756000ADEB030DE8464146204622F035FAD2E75E
:10757000002CA0D02246084973E700BF353D050026
:107580003E3D050064400500B93805005740050040
:107590004B3D05007F3D0500B53D050008B5054A9A
:1075A000136823F4007313600FF030FCBDE808404B
:1075B00011F0D6BCF8C0002008B5054A136843F4A2
:1075C000007313600FF014FCBDE80840FEF754BED2
:1075D000F8C0002008B511F083FE41EC100B08BD87
:1075E00008B50C4B1B884FF6FF729BB2934203D138
:1075F000094A1288934208D0084819F075FD084AD4
:10760000136843F00803136008BDBDE8084010F09C
:10761000B3B900BFB42C0020B62C00201F3E0500DB
:10762000F8C0002038B50F4C0F49002205466068AD
:1076300026F006FC26F06AFFC3B27DB143F00100DC
:1076400098420ED0646824F05FFA0749024620464B
:1076500026F0BDFBBDE83840FFF7C2BF03F0FE00D7
:10766000EEE738BD582D0020643F05002DE9F041BC
:107670008CB006460F4624F068FC40B93EB1324655
:107680005249032020F0C4F90CB0BDE8F08100237A
:10769000029301934E4B039302AB05934D4B06931C
:1076A0004FF003080B23ADF81C300DEB080301224B
:1076B0000893494B8DF803200993424601AB03A977
:1076C0003846ADF81080ADF828800B9322F09AFC74
:1076D0000028D9D00298414D414C24F014FD48B106
:1076E000029A4049686826F051FB236843F008037A
:1076F000236009E0029B002B4AD13A49686826F0D2
:10770000D7FF23685906F0D4029850B1C389A3F576
:1077100000739BB2C381C38903F4F0530BB924F007
:10772000E9FD9DF80330002B37D023682E496868A7
:107730009A065EBF236843F00803236026F0B8FF73
:1077400032462A49686826F0CDFF3A4628496868DB
:1077500026F0C8FF019A1AB1236843F0080323609A
:107760002449686826F0BEFF019850B1C389A3F58B
:1077700000739BB2C381C38903F4F0530BB924F0A7
:10778000B9FD236813F0180F1BD0FFF729FF7BE723
:107790001949404620F03CF9B6E72368D5F8048043
:1077A0009B0648BF23684FF0000044BF43F0080326
:1077B000236024F0A1F90C490246404626F007FB5D
:1077C000BEE730460FF0C2F85EE700BFAB410500F0
:1077D000543E0500B1400500B6400500582D00207C
:1077E000F8C00020C0400500EF400500F84005004B
:1077F000024105000C410500CA40050013B5694669
:10780000044612F09FFF28B90749012020F000F933
:1078100002B010BD054B06495868224626F0B6FA5C
:10782000FFF7DEFEF4E700BFD63E0500582D00202E
:107830000C3F050070B50D4D2A7806460C462AB15E
:1078400001200B4920F0E4F8002070BD08F084FD11
:10785000084B2E70186024B1E38903F500739BB2C6
:10786000E381054B01201C60EFE700BFFCC0002056
:10787000AB3B0500F4C0002000C1002037B5054631
:10788000002105208DF80610FFF7D4FF70B1084BDA
:107890001C6824B1E38903F500739BB2E38101996D
:1078A00028460EF053FF204603B030BD0446FAE7E9
:1078B000F4C0002037B505460C4605200021FFF72F
:1078C000B9FFD0B1214601A812F068FE024638B1D6
:1078D0000B49012020F09CF80024204603B030BD65
:1078E000084B1C6824B1E38903F500739BB2E38164
:1078F000019928460EF02AFFEFE70446EDE700BFA6
:1079000074410500F4C0002013B5002104208DF857
:107910000610FFF78FFF68B1074B1C6824B1E3899D
:1079200003F500739BB2E38101980EF05FFF2046E0
:1079300002B010BD0446FAE7F4C0002013B50C46AF
:1079400004200021FFF776FFC8B1214601A812F0FC
:1079500025FE024638B10B49012020F059F80024D9
:10796000204602B010BD084B1C6824B1E38903F522
:1079700000739BB2E38101980EF038FFF0E70446F4
:10798000EEE700BF74410500F4C0002038B5124D89
:107990002A8801464FF6FF70904215D00320FFF76A
:1079A00049FF78B10D4B1C6824B1E38903F50073DE
:1079B0009BB2E38113212888FCF7D6FD11F0D0FAA1
:1079C000204638BD0446F5E7FEF7F8F9BDE8384033
:1079D000084608F035BD00BFB42C0020F4C00020DC
:1079E0002DE9FF4100220F463149804626F028FA52
:1079F00000223049064626F023FA6946054612F071
:107A0000A1FE044658B92946304625F0DDFD2A4935
:107A100003201FF0FDFF204604B0BDE8F0815EB1F9
:107A2000F389A3F500739BB2F381F38903F4F05358
:107A300013B9304624F05EFC41460220FFF7FAFEFF
:107A400080B90024002DE6D0EB89A3F500739BB22A
:107A5000EB81EB8903F4F053002BDCD1284624F0B2
:107A600049FCD8E74821154824F095F80446002839
:107A7000E7D00223014602AA0020CDE9025719F0FF
:107A8000A7FAE389A3F500739BB2E381E38903F4CA
:107A9000F05313B9204624F02DFC094B1C68002C30
:107AA000D0D0E38903F500739BB2E381CAE700BF3E
:107AB000ED3B0500553E05004D3C050081A7020049
:107AC000F4C0002070B504460E46002018491BF093
:107AD00041FA054610B90025284670BD22461549D1
:107AE00026F054F92846FEF7F9FBEB89A3F500735D
:107AF0009BB2EB81EB8903F4F053044613B928469B
:107B000024F0F8FB002CE6D031462046FFF768FF52
:107B1000E389A3F500739BB2E381E38903F4F05397
:107B20000546002BD8D1204624F0E4FBD4E700BF63
:107B300038400500553E05002DE97043064658B112
:107B400024F003FA044638B932464E4903201FF0A8
:107B50005FFF2046BDE8708300224B49304626F087
:107B60006FF9044624F0E9F998B95CB1E389A3F50B
:107B700000739BB2E381E38903F4F05313B9204609
:107B800024F0B8FB2246414903201FF041FF0024A6
:107B9000DFE75CB1E389A3F500739BB2E381E3897E
:107BA00003F4F05313B9204624F0A4FB0022384913
:107BB000304626F045F927F047F802460B46804646
:107BC00089462BF03DFB30B9002200234046494650
:107BD0002BF018FB18B1DFF8C8904FF00008002117
:107BE0002C4823F0D8FF0446002846D0002149EC59
:107BF000108B0AF0F1FDE389A3F500739BB2E381DA
:107C0000E38903F4F053054613B9204624F072FBD0
:107C100029460120FFF70EFE002830D008211E481B
:107C200023F0B9FF044670B13146FEF7C9FCE38981
:107C3000A3F500739BB2E381E38903F4F05313B916
:107C4000204624F057FB154B1C6824B1E38903F54B
:107C500000739BB2E381002D3FF47BAFEB89A3F56A
:107C600000739BB2EB81EB8903F4F053002B7FF49C
:107C700070AF284624F03EFB6BE70546C8E7044694
:107C8000E9E700BFE23D0500173E0500753F05002E
:107C9000EA3C050095A30200EDA80200F4C0002014
:107CA00000409F402DE9F04F91B0014602A813F02B
:107CB000FDF828B94FF00009484611B0BDE8F08F33
:107CC0009DF81370012F06D0182F04D046490120CB
:107CD0001FF09EFEEEE7BDF80F50BDF811607D432A
:107CE0001F35012F4FEA65150CBF4FF0200A4FF0EA
:107CF0001A0AAD0005FB06A6304623F07BFF81463D
:107D00000028D7D024F06BF9422303704D23437031
:107D100086700C233612C67080F80AA08373BDF8F3
:107D20000F3083741B0AC374BDF8113003751B0A2E
:107D300043750123012F83759DF81330037608BF27
:107D4000FF23044602BF8376C37603770022BDF883
:107D500011609642B0DD9DF8133002F1010BA6EBE5
:107D60000B06012B05FB06A638D04FF0000817B212
:107D7000BDF80F3043452FDD3A460FFA88F102A8CF
:107D800013F026F89DF81330DB0808FB0363020AA2
:107D9000E0542344000C5A70987008F10108E7E79A
:107DA00000235B0039B2009A019302A813F010F887
:107DB0000137019B00F00100B84543EA0003F0D110
:107DC00006EBE80208F1080802F8013CBDF80F30A4
:107DD000A8F10807BB42E3DC5A46B8E713B24FF0FC
:107DE000080800932644F1E7D141050038B5FFF7B4
:107DF00059FF054610B90025284638BD0AF0FEFF98
:107E0000EB89A3F500739BB2EB81EB8903F4F0538C
:107E1000044613B9284624F06DFA002CEBD0214615
:107E2000084824F047FEE389A3F500739BB2E38181
:107E3000E38903F4F0530546002BDDD1204624F0FE
:107E400059FAD9E7FF41050010B5FFF7CFFF044607
:107E500068B11AF02BFFE389A3F500739BB2E381AD
:107E6000E38903F4F05313B9204624F043FA02489F
:107E7000BDE810401AF086B904A7050030B58FB0F0
:107E80000C4601466846154613F010F820B12AB298
:107E900021B2684612F09CFF0FB030BD30B58FB0F4
:107EA0000D460146684613F001F800284CD0BDF994
:107EB0001B20BDF91F309A4244DC04F07BF80446D5
:107EC00018B3BDF91B0023F01FFE204902462046CF
:107ED00025F07DFFBDF91D0023F016FE1C4902466A
:107EE000204625F074FFBDF91F0023F00DFE19494F
:107EF0000246204625F06BFFBDF9210023F004FE69
:107F000015490246204625F062FFC5B100226FF0F8
:107F10007F038DF81F208DF820308DF821208DF8FB
:107F200022304FF0FF327F2368468DF81B208DF8FA
:107F30001C308DF81D208DF81E3012F07DFF20467C
:107F40000FB030BD0024E0E70446F8E71844050010
:107F50001B4405001E4405002144050070B58EB089
:107F600004460D4601466846164612F09FFF50B380
:107F7000BDF80530022D23F070039BB21DD0032DF8
:107F80001ED0012D08BF43F03003ADF805304EB1CF
:107F9000BDF80530DA064CBF83F0400383F02003C0
:107FA000ADF80530684612F047FFE38903F500732A
:107FB0009BB2E38120460EB070BD43F06003E4E75E
:107FC00043F05003E1E70446F4E770B58EB0044691
:107FD0000E4601466846154612F068FF70B16846C5
:107FE000ADF81660ADF8185012F026FFE38903F5DE
:107FF00000739BB2E38120460EB070BD0446FAE7E1
:10800000F0B58FB004460E460146684615461F4639
:1080100012F04CFF00B3012E9DF81A10A8BF0126E4
:10802000012DA8BF012546EAE67666F3010145EA7F
:10803000E57565F3830187F3020767F30511684669
:108040008DF81A1012F0F8FEE38903F500739BB265
:10805000E38120460FB0F0BD0446FAE72DE9F04376
:1080600017461D46421E47F6FE739A428FB0814660
:10807000884602D84A1E9A4208D93D4901201FF07D
:10808000C7FC002420460FB0BDE8F0833846FDF75A
:1080900099FE044620B9374901201FF0B9FCF1E7E9
:1080A000284623F052FFD8B100223349284625F054
:1080B000C7FE002204463149284625F0C1FE254668
:1080C0000646284623F059FF044680B92A462C4923
:1080D00001201FF09DFC3146284625F075FAD1E7B6
:1080E000EB8903F500739BB2EB810646E9E736B1F5
:1080F000304623F042FF044608B93246E7E72149FB
:1081000000201AF027FF04460028BBD000234FF0C0
:10811000FF32CDE903238DF805308DF806304FF698
:10812000FF730593069B1849009003F4400343F046
:108130007F4343F470230693144B07938023ADF8D9
:1081400020308DF822302A4601238DF80430ADF816
:108150000790ADF809808DF80B7025F017FE3246B8
:108160000B49009825F012FE684612F065FEB2E752
:10817000EB420500F8420500044305000D430500ED
:1081800016430500F64105004A4305007FFF7F00C6
:10819000544305002DE9F04192B006460D460146D4
:1081A00004A8144612F082FE4FF00008002869D09F
:1081B0000DF10A0202A904A8ADF80C50ADF80E406A
:1081C000ADF80880ADF80A8012F060FC0DF10E02E7
:1081D00003A904A812F05AFCBDF90830BDF90A2021
:1081E000BDF90C50BDF90E40ED1AA41A119B2246A0
:1081F000294604A89847DDE907734545079326DD1E
:10820000BDF81920013A12B26B1E00921BB2424611
:10821000414604A80F9DA847002C26DDBDF8173065
:10822000013C013B24B200941BB20022002104A8AF
:108230000F9CA04704A8079712F0FEFDF38903F5F1
:1082400000739BB2F381304612B0BDE8F081E3D0F9
:10825000BDF81920BDF81710013A4B1E12B229447F
:1082600000921BB2424609B2D3E7E3D0BDF8191021
:10827000BDF817300A190139013B09B200911BB250
:1082800012B2D3E70646DEE7F0B58FB004460E46DD
:108290000146684615461F4612F008FEE0B1B7B920
:1082A000039B36B22DB22A463146684612F0B0FD25
:1082B0006846ADF81660ADF8185012F0BDFDE389C0
:1082C00003F500739BB2E38120460FB0F0BD384642
:1082D00025F086FA0346E4E70446F5E72DE9F04F7A
:1082E0009DB004460D4601460EA8CDE9052312F0C7
:1082F000DDFD20B9002420461DB0BDE8F08F2846E2
:1083000023F023FE20B9764901201FF081FBF1E71D
:1083100000227449284625F093FD26F0F7F8002244
:1083200071490290284625F08BFD26F0EFF80022D7
:108330006E490090284625F083FD26F0E7F80022DC
:1083400001906B49284625F07BFD804625F048FAD0
:108350000390B8F1000F0ED0B8F80E30A3F50073FB
:108360009BB2A8F80E30B8F80E3003F4F05313B9EE
:10837000404623F0BFFF284600225E4925F060FDFD
:10838000054623F0BEFDA8B1029B002B18DC5A491C
:1083900001201FF03DFB002DACD0EB89A3F500734D
:1083A0009BB2EB81EC8914F4F054A3D1284623F05E
:1083B000A1FFA0E7284623F07BFE0028E4D1E6E7F2
:1083C000009B002BE3DD019B202BE0DC284624F002
:1083D0004FFA07465DB1EB89A3F500739BB2EB81C1
:1083E000EB8903F4F05313B9284623F083FF019B74
:1083F000012BB8BF01239B4609AB00221846394622
:108400001EF012FF012202FA0BF2531E0025049304
:1084100009AB2E46A946AA4607935E455BDADDE91D
:1084200009239A4202D2009B994522DB0C9850B155
:10843000C389A3F500739BB2C381C38903F4F053CE
:108440000BB923F057FF5FB1FB89A3F500739BB213
:10845000FB81FB8903F4F05313B9384623F04AFF3C
:108460000EA812F0E9FCE38903F500739BB2E381E7
:1084700041E72B020D9D0DB1099AAD5C07980836B6
:108480001D431EF055FBB345F3DCA6EB0B06049A27
:1084900025FA06F31340B8F1000F02D0039A9A426E
:1084A0000DD0019A012A01DC9BB1119B069A059916
:1084B0004A44514412B209B20EA812F0A9FC029B20
:1084C0000AF1010A5345DCBF09F101094FF0000A26
:1084D000A3E7129BEAE7009B9945D6DBA6E700BF1E
:1084E000714305009A43050090440500A043050030
:1084F000A4430500645D0500B0430500F0B5DBB0A2
:1085000004460D4601460CA812F0D0FC18B9002410
:1085100020465BB0F0BD284623F0F5FD0028F6D0DC
:108520002946012201A821F086F81AAE0025374617
:1085300001A81EF02AFA08B1802D16D101A81EF05C
:10854000E5F9802D03D140210D481FF0FFF83A4690
:1085500069100CA812F0BAFA0CA812F06DFCE389AD
:1085600003F500739BB2E381D2E701A81EF005FC7E
:1085700026F8020B01A801351EF03AFBD8E700BF30
:10858000E44305002DE9F04F9FB004460E46014636
:1085900010A8039212F08AFC20B9002420461FB0D4
:1085A000BDE8F08F304623F0AEFD0028F5D031460F
:1085B000012205A821F03FF8002605A81EF0E5F9E4
:1085C000C0B905A81EF0A2F9039B53B12DB20095C6
:1085D0000FFA8AF3BDF95820BDF9561010A812F011
:1085E0007BFB10A812F028FCE38903F500739BB213
:1085F000E381D3E705A81EF0C0FBF307834616D539
:10860000012E0FFA87F90FFA80F816D0CDF8008006
:108610004B46BDF95820BDF9561010A812F05CFB6E
:10862000AB465D46ADF85690ADF85880BB4605A800
:1086300001361EF0DDFA5F46BFE7BA46F1E770B5D6
:1086400090B004460E46014602A8154612F02EFCD4
:10865000C8B136B22DB23346BDF92020BDF91E1087
:10866000009502A812F038FB02A8ADF81E60ADF824
:10867000205012F0E1FBE38903F500739BB2E38124
:10868000204610B070BD0446FAE7F0B591B004463C
:108690000D46014602A816461F4612F007FC98B187
:1086A000BDF95830009332B23BB229B202A812F0A1
:1086B00013FB02A812F0C0FBE38903F500739BB221
:1086C000E381204611B0F0BD0446FAE708B524F076
:1086D0007DF908BD2DE9F04F95B004460D460146E1
:1086E00006A812F0E3FB002839D0BDF92C30023384
:1086F00038D100223749204625F0A2FB0022364916
:108700000646204625F09CFB25F000FF80462846C3
:1087100026F0BEF800220146814601A81EF084FD25
:108720000027DFF8B8A03C464FF0C00BDDE901326E
:1087300093421BD3049850B1C389A3F500739BB235
:10874000C381C38903F4F0530BB923F0D3FD48462A
:10875000314624F039FFBC422046B8BF384615B038
:10876000BDE8F08F4FF000084646D0E7059D35B1D3
:10877000ED5C0A2D03D1A742B8BF27460024BDF9FE
:108780002C20002A0FDD203DEBB25E2B97BF1AF89C
:108790001530002313FB02F3B3FBFBF31C4401A8C9
:1087A0001EF0C6F9C2E7531C01D10434F7E70232C8
:1087B000F5D1304623F07CFC40B14545EFDBA5EB1D
:1087C0000801304624F002F90444E8E7304625F079
:1087D00007F8F9E7974405009C440500505B050045
:1087E000F8B506460F46144623F062FC0546E8B18C
:1087F000204623F0D2FBD8B1204624F0F1FF0546F5
:10880000384626F045F8044624F04CFA2D1A13D5C4
:1088100000255CB1E389A3F500739BB2E381E38992
:1088200003F4F05313B9204623F064FD2846F8BD45
:10883000304624F037FAE2E7204624F033FA2F18C6
:10884000304624F02FFA8742E2D82A4601232146F7
:108850003046F7F791FFB0FA80F56D09D9E7F8B522
:1088600007460D46164623F023FC044698B12846D9
:1088700026F00EF8002E05460FDA00245DB1EB89D4
:10888000A3F500739BB2EB81EB8903F4F05313B9AA
:10889000284623F02FFD2046F8BD24F003FA841962
:1088A000384624F0FFF98442E7D8012332462946AE
:1088B0003846F7F761FFB0FA80F46409DEE700009C
:1088C0002DE9F04FA5B000AF0D46F862014607F163
:1088D0005800BA621C4612F0E9FA002800F06082E3
:1088E000B7F96C30002B05DD7B624FF0000BC7E958
:1088F00007BB21E05E1C00F08380023340F08580DE
:108900000022A049F86A25F09BFA0022F8619E49EE
:10891000F86A25F095FA00229C493862F86A25F039
:108920008FFA25F0F3FD002278629949F86A25F064
:1089300087FA25F0EBFD834697F87220B7F85D3093
:108940003B8102F0300110299BB263D183F03003E8
:10895000A7F85D30BB6AB7F85F10BC620133CC1A70
:1089600002F00302012A0FD82946F86AFFF7B2FE87
:1089700097F8723003F0030303FB0000BB6A00EBBF
:10898000D070A3EB6003BB6297F87230C3F381022F
:10899000012A08D87A6A03F0030303FB022303EBDE
:1089A000D373A4EB6304B7F85F307B61B7F8613031
:1089B000BB61B7F85D30D80648BFD7E90523284624
:1089C00048BFC7E9053225F063FF0022F860014681
:1089D00007F130001EF028FCBE6AD7E90C239A424A
:1089E00080F0A3803B6C9BB313F80290B9F10A0F9F
:1089F0002FD17B6A07F130001C441EF099F8EBE799
:108A000006234FF0000B7B6271E74FF0000BC7F8B5
:108A100024B06CE720290ED183F06003A7F85D3005
:108A2000BB6AB7F85F100133CB1ABB62B7F861308D
:108A300001341C1B94E7302992D183F05003B7F81E
:108A40006110A7F85D30631CCB1ABC6ABB6287E774
:108A50009946B7F96C80B8F1000F40F38C80A9F10A
:108A600020095FFA89F25E2A9BBF4A4B13F819303E
:108A7000002313FB08F39CBFC021B3FBF1F33B6160
:108A80003B695B42B34249DA7B699E4246DAC8F1F0
:108A90000003A34242DABB699C423FDA5E2A3DD81A
:108AA00000233C4A1D4699455BDC02EB4902C7F8AE
:108AB00000D053787B60384B88B000201D44EA46D4
:108AC000814660237A68914526DA2A7895F801C0B4
:108AD0004FF0300E02F07F0218FB02E2B2FBF3F21D
:108AE00032442AF810200AEB40010CF07F0218FBF8
:108AF00002E21CF0800FB2FBF3F222444A8000F144
:108B0000020034D04110524607F1580011F0DEFF48
:108B10001DF088FC602350B3D7F800D03B691E4499
:108B20001DF080FC002800F02881F86B002840F040
:108B30002981D7E90712F86824F01AFD3B89A7F8C4
:108B40005D3007F1580012F077F9FB6AFA6ADB89A9
:108B500003F500739BB2D381F86A9437BD46BDE834
:108B6000F08F02EB4301013349780D449BE709F193
:108B700002090235A6E7B8F1FF3F5FD1F11C0DDA1B
:108B80000436CDE7DA43050097440500DF430500CE
:108B90009C440500505B0500344705007B699E42FC
:108BA000EEDA621DECDBBB699C42E9DAA9F121092E
:108BB000B9F15E0FE4D8052399FBF3F303EB8302CD
:108BC000A9EB020909EB49023A614FF00609754A1F
:108BD00009FB03F302EB430906F1010A33B2002556
:108BE0007B600FFA8AFA39F8028B3B6948FA03F87E
:108BF00018F0040F07D062197B6E796812B207F182
:108C0000580012F005F918F0020F07D02A197B6EF0
:108C100012B2514607F1580012F0FAF818F0010F9D
:108C200008D02A19B11C7B6E12B209B207F15800A4
:108C300012F0EEF80135062DD5D1A1E718F1020F9B
:108C40007FF46EAF386A23F033FA00285DD0CB454D
:108C500000F3918007F144050022396A28461EF08E
:108C6000E3FA4FF00008A9EB0B09796CBB6C7A6D45
:108C7000994203D2FB6C0B444B453DDB002A42D0AA
:108C8000555C386D50B1C389A3F500739BB2C381A5
:108C9000C38903F4F0530BB923F02CFB6B42B342AE
:108CA0003DDA7B699E423ADA7B6A5B42A34236DA5E
:108CB000BB699C4233DA7B6AF96908FB03F807F168
:108CC000440A4FEAD80250461EF0AEFA08F00708F0
:108CD0004FF00009C7F804A0A94545DB386DF0B195
:108CE000C389A3F500739BB2C381C38903F4F05316
:108CF000ABB923F0FFFA12E002B1525C284690446F
:108D00001DF016FFB1E71546BBE7386A24F068FD91
:108D1000A9EB0B08CB45054600FB08F8BEDD2E4449
:108D2000FEE67B6D73B17A6C9B5C03FA08F31B065D
:108D300008D504EB0A027B6E396912B207F15800BC
:108D400012F066F808F10108B8F1080F04D178684C
:108D50001DF0EEFE4FF000080AF1010A7B6A534550
:108D6000DFDC09F10109B7E706EB09031BB24FF09D
:108D7000000A3B61F2E70025D1E707F130001DF062
:108D8000D7FE2AE6C389A3F500739BB2C381C389CA
:108D900003F4F053002B7FF4CCAE23F0ABFAC8E61B
:108DA000F862D9E68C3A05002DE9F0438FB004460D
:108DB00088460146684616461D46169F12F076F80C
:108DC000002846D0404623F073F940B922490120DB
:108DD0001EF01EFE002420460FB0BDE8F083FF2EDB
:108DE00001D91E49F3E7284623F062F928B928463D
:108DF00023F01DFA08B91A49E9E77B1EFE2B01D9B9
:108E00001849E4E742461849204624F0BFFF2A46A5
:108E10001649204624F0BAFF384622F075FE144960
:108E20000246204624F0D3FF304622F06DFE114961
:108E30000246204624F0CBFF4FF6FE736846ADF89D
:108E4000143011F0F9FFE38903F500739BB2E3815D
:108E5000C1E70446BFE700BF2444050041440500C4
:108E60005E44050088440500DA4305009744050088
:108E7000DF4305009C4405002DE9F04F99B00AAC92
:108E800081460F460146204616461D4612F00EF852
:108E9000002800F08980229BADF826300DF12202D7
:108EA00008A92046ADF82070ADF82260ADF8245036
:108EB00011F0ECFD0DF1260209A9204611F0E6FDA6
:108EC000BDF92000BDF92420BDF92210BDF92630DE
:108ED0008518121ACE1802EBD27A5B1A4FEA6A0A88
:108EE000013203EBD378B8BFCAF1000A4FEA680831
:108EF0000133B8BFC8F1000808FB08F30393039AD5
:108F00000AFB0AF305EBD57506EBD6766D107610E5
:108F1000049353430793009605EB0A033246A5EBEF
:108F20000A01204611F0C0FC0023CDE905340127D9
:108F3000B8450DDA0AA811F07FFFB9F80E3003F535
:108F400000739BB2A9F80E30484619B0BDE8F08F07
:108F5000059B049A5C1E07FB07F3AAEB040453432A
:108F6000002C17DCF21BAAEB040305EB040BA5EBAA
:108F7000040A5146059300925B46069811F094FC52
:108F8000F219514600925B46069811F08DFC0137AC
:108F9000A246CDE7039904FB04F201FB02320799D4
:108FA0009142DFDA013CDBE78146CDE737B5054684
:108FB0001C4613440093121B0B19091BFFF75CFF9F
:108FC000EB8903F500739BB22846EB8103B030BDFB
:108FD000F0B593B004460F46014604A816461D4658
:108FE00011F064FF002849D0189BADF80E300DF148
:108FF0000A0202A904A8ADF80870ADF80A60ADF83D
:109000000C5011F043FD0DF10E0203A904A811F05C
:109010003DFDBDF90A200092BDF90C30BDF90810E4
:1090200004A811F041FCBDF90C30BDF90E200092EE
:109030001946BDF90A2004A811F036FCBDF90E202E
:109040000092BDF90C30BDF9081004A811F02CFCF9
:10905000BDF90830BDF90A2000921946BDF90E206D
:1090600004A811F021FC04A811F0E6FEE38903F541
:1090700000739BB2E381204613B0F0BD0446FAE7CB
:10908000F0B593B004460F46014604A816461D46A7
:1090900011F00CFF58B3189BADF80E300DF10A0219
:1090A00002A904A8ADF80870ADF80A60ADF80C503C
:1090B00011F0ECFC0DF10E0203A904A811F0E6FC7E
:1090C000BDF90E300093BDF90A20BDF90C30BDF991
:1090D000081004A811F0E8FB04A811F0ADFEE38924
:1090E00003F500739BB2E381204613B0F0BD044644
:1090F000FAE730B591B004460D46014602A811F0DA
:10910000D5FE78B38DB100234FF0FF32CDE90523B2
:10911000ADF820309DF8223023F03F034FF6FF7268
:1091200043F00F0307928DF82230DDE90553BDF8B7
:1091300011200593013ABDF80F3012B20092013BA5
:1091400000221BB2114602A811F0AEFB02A8059541
:1091500011F072FEE38903F500739BB2E3812046B0
:1091600011B030BD0446FAE72DE9F04F9DB00EADC9
:1091700003900F460146284616461C4611F096FEFF
:10918000002800F0C680269BADF836300DF1320283
:109190000CA92846ADF83070ADF83440ADF8326017
:1091A00011F074FC0DF136020DA9284611F06EFC89
:1091B000BDF93040BDF93420BDF93200A31803EBEE
:1091C000D3734FEA630ABDF93630C118121B01EBA5
:1091D000D1711B1A491002EBD27464100491013250
:1091E00003EBD371B8BF64424FEA610B0133B8BFE0
:1091F000CBF1000B0BFB0BF30793079A04FB04F373
:10920000089353430B93049A119BAAEB040128463D
:1092100011F097FB119B049A0AEB0401284611F008
:1092200090FB002301270993BB450DDA0EA811F02E
:1092300003FE039B039ADB8903F500739BB2D38182
:1092400003981DB0BDE8F08F099B089A5E1E07FBCE
:1092500007F3A61B5343002E2BDCA31B0993AAEB99
:1092600006030593049BA3EB07090AEB0603069389
:10927000049B03EB0708A31B012B24DC119B05991E
:109280004A46284611F05DFB119B06994A4628463E
:1092900011F057FB119B05994246284611F051FBEE
:1092A000119B06994246284611F04BFB0137344684
:1092B000BAE7079906FB06F201FB02320B999142CD
:1092C000CBDA013EC7E7AAEB0403544401334A4614
:1092D0000599CDF800902846013C0A9311F0E4FA74
:1092E00023464A460699CDF80090284611F0DCFA4C
:1092F0000A9B0599CDF800804246284611F0D4FA21
:10930000CDF80080234642460699284611F0CCFA53
:10931000CCE7039094E737B505461C461344009309
:10932000121B0B19091BFFF71FFFEB8903F50073D5
:109330009BB22846EB8103B030BD00002DE9F04719
:109340008AB0804622F0B4FE044638B96149032051
:109350001EF05EFB20460AB0BDE8F08700224146C1
:1093600068461DF061FF00273C463E46B9463D4633
:10937000DDE90032934212D3039850B1C389A3F5BB
:1093800000739BB2C381C38903F4F0530BB922F07D
:10939000B1FF02F00FFE0546D8B90024DAE7049ABF
:1093A0006AB1D35C0A2B0AD155EA090308BF012729
:1093B00009F10109002568461DF0BAFBD8E7A1456F
:1093C00005F10105A8BF09F10104AE42B8BF2E4660
:1093D000F1E7304622F098FB3F490246284624F048
:1093E000F6FC204622F090FB3C490246284624F039
:1093F000EEFC04FB06F007300021C01023F018FF3C
:10940000044668B9EB89A3F500739BB2EB81EB8945
:1094100003F4F053002BC0D1284622F06BFF99E7EC
:109420003A46414668461DF0FFFE4FF000084746A9
:109430004FF08009DDE90032934213D3039850B115
:10944000C389A3F500739BB2C381C38903F4F053AE
:109450000BB922F04FFF22462149284624F0B7FCE1
:109460002C4677E7049A5AB1D35C0A2B06D108F14F
:109470000108002768461DF05BFBDBE7202B26D0A8
:10948000204622F015FE10B306FB087A21464FEA6B
:10949000DA0205A81DF0C8FE099909B1059BC95C4F
:1094A0000AF0070A49FA0AFA41EA0A0105A8C9B20C
:1094B0001DF01CFD089850B1C389A3F500739BB241
:1094C000C381C38903F4F0530BB922F013FF0137B2
:1094D000D0E700BF5E4305009A43050090440500B5
:1094E000645D05002DE9F04316461D46421E47F611
:1094F000FE739A428FB080460F4602D84A1E9A42A7
:1095000005D9774901201EF083FA002408E030468F
:10951000FCF758FC044638B9724901201EF078FA6D
:1095200020460FB0BDE8F0836F49002019F012FD0E
:1095300004460028F4D04FF000094FF0FF33CDE986
:1095400003394FF6FF730593069B009003F4400325
:1095500043F07F4343F470230693644B07932846FC
:1095600080238DF805908DF80690ADF820308DF8A9
:1095700022308DF80490ADF80780ADF809708DF8B1
:109580000B6022F0E2FC002865D04A465849284684
:1095900024F056FC25F021F928B1BDF8053043F040
:1095A0000103ADF8053000225249284624F048FC5A
:1095B00025F013F928B1BDF8053043F00403ADF8E8
:1095C000053000224C49284624F03AFC25F005F9E4
:1095D00028B1BDF8053043F00803ADF8053000228E
:1095E0004649284624F02CFC25F0F7F888B19DF870
:1095F0000B0001280BD1BDF8053043F00203ADF894
:109600000530BDF809305B0703D03D497BE73D4994
:1096100078E7284600223C4924F012FC0546D0B1E8
:109620003A4923F01BF950B93949284623F016F975
:1096300050BBBDF8053043F08003ADF80530EB8931
:10964000A3F500739BB2EB81EB8903F4F05313B9DC
:10965000284622F04FFEBDF80900BDF8073043430D
:109660009DF80B0058430730C0100AF0ADFB294AA3
:1096700005460146009824F00FFC294623F0A4FF7C
:10968000684611F0D9FB4BE72349284623F0E6F85A
:1096900020B9BDF8053043F48073CEE71F49284652
:1096A00023F0DCF820B9BDF8053043F4C073C4E7FB
:1096B0001B49284623F0D2F820B9BDF8053043F401
:1096C0000073BAE71749284623F0C8F820B9BDF857
:1096D000053043F42073B0E713481EF037F8AEE7C7
:1096E000EB420500F8420500F64105007FFF7F00D0
:1096F000184205001F420500234205002F420500C5
:109700006D4205003D420500A6420500B24205003B
:10971000B6420500645D0500BA420500BE42050080
:10972000C2420500C6420500CA4205000000000012
:1097300008B500222DED028BB0EE408AF0EE608A73
:10974000002351EC100B29F067FD98B1B0EE480AE8
:10975000F0EE680A27F028FB0B4B51EC100B0022AF
:1097600029F0D4FABDEC028B41EC100BBDE80840A7
:1097700027F096BABDEC028B9FED010B08BD00BF30
:10978000000000000000F87F0000E03F0000000043
:10979000F8B555EC104B25F000474FF0FF32284B41
:1097A0002046394629F04CFD60B94FF0FF32244B7A
:1097B0002046394629F03AFD20B9B5F1004F08BFDF
:1097C000002C05D145EC104BBDE8F84022F08AB9D9
:1097D000002200232046294629F00AFDC8B912A11B
:1097E000D1E900012B46224629F0DAF806460F4659
:1097F00029F0ECFD04460D4654EA05030DD1002284
:1098000000233046394629F0F3FC30B19FED080BB8
:10981000DAE709A1D1E90001E4E720462946BDE8DD
:10982000F84022F0D1B900BF2083E4FFFFFFDF3F03
:1098300000000000000000802083E4FFFFFFDFBF86
:10984000FFFFEF7F27F028BA26F00ABF27F0C4B940
:10985000F0B585B000AF0023391D06467B6023F0CC
:109860007EFA0446F0B9304620F0C6F80546786026
:109870001CF0E0FD05F58073834208D919490120E9
:109880001EF0C6F8254628461437BD46F0BDEB1D30
:1098900023F00703ADEB030D6C462A462146304604
:1098A00020F09AF87B681048FB60002207F108015D
:1098B000BC6011F0ABFB002339463B60F7F78CFA34
:1098C0003E68054626B909481DF060FF3546DAE7CF
:1098D0007B680548BC60324607F10801FB6011F067
:1098E00095FBD0E7B93805004B5E0200A1440500A6
:1098F000F0B583B000AF0023391D06467B6023F02E
:109900002EFA0446F0B9304620F076F80546786025
:109910001CF090FD05F58073834208D9164901209B
:109920001EF076F8254628460C37BD46F0BDEB1DE7
:1099300023F00703ADEB030D6C462A462146304663
:1099400020F04AF800231A467968204611F051FCAD
:10995000002339463B60F7F73FFA3E68054626B9D3
:1099600006481DF013FF3546DDE73B46044A79689B
:10997000204611F03EFCD6E7B9380500A1440500A9
:10998000635E0200F8B5051E0C4606DC294901207D
:109990001EF03EF800242046F8BD084622F0D5FA15
:1099A0000646A8B100222449204624F049FA24F0B2
:1099B00014FF002221490646204624F041FA24F0F3
:1099C000A5FD30F0080309D0102809D01C49DEE7B6
:1099D00024B122461B4901201EF01AF8012400E0A0
:1099E00002242946204620F0EEFA07469EB1294679
:1099F000204620F0E8FA05461349002019F0AAFA9B
:109A0000044610B10FB146B13DB92A463946204649
:109A100023F0AEFDBEE73546EEE73A460B49204659
:109A200024F0D5F9002DB6D02A460949204624F065
:109A3000CEF9B0E7DE450500FD4505001C460500F2
:109A40000A4605002146050058460500645D0500EC
:109A50006146050070B50D1E064606DA0B49012069
:109A60001DF0D6FF0024204670BD1B2021F0E4FF2E
:109A7000044615F1FF35F6D31CF0D4FC0028F2D1D2
:109A80003146204623F001F8F3E700BFB445050056
:109A9000F8B507460E4622F058FA00283CD00022BE
:109AA0001E49384624F0CCF9044622F001FB70B37D
:109AB000204623F0F7F8002E01DD864206D3174931
:109AC000384624F0F5FD25462846F8BD32460021EB
:109AD000204622F0DFFF6FF0004231460546204667
:109AE00022F0D8FF0D490246384624F070F9002CC8
:109AF000EAD0E389A3F500739BB2E381E38903F421
:109B0000F053002BE0D1204622F0F4FBDCE71B20D1
:109B100021F092FF0546EAE70546D5E7F73905004B
:109B2000F0B587B024F0B4FE0546002842D00146C7
:109B3000002201A81DF078FB4FF0FF340027DDE97B
:109B400001639E4225D3049850B1C389A3F50073E5
:109B50009BB2C381C38903F4F0530BB922F0CAFB53
:109B6000A742DABFE21B013200223946284622F022
:109B700091FFEB89A3F500739BB2EB81EB8903F4B2
:109B8000F053044613B9284622F0B4FB204607B030
:109B9000F0BD059800B1805D1CF00EFE30B9039B4E
:109BA0001E4437EA240728BF3746344601A81CF074
:109BB000BFFFC4E70446E9E72DE9F84F05460E4626
:109BC00022F076FA20B94FF000084046BDE8F88F41
:109BD00021F0EBFF80460028F5D01EB9294623F07E
:109BE00097FFF2E73046F7F7B7F8002800F08180DA
:109BF000002021F089FF6A490246304624F0E7F848
:109C00002946304606F076FA0027044684B12046FD
:109C100022F058F9814618B3E389A3F500739BB28B
:109C2000E381E38903F4F05313B9204622F062FB89
:109C3000002021F069FF5A490246304624F0C7F857
:109C4000284623F02FF8B842BFD339466FF00042C0
:109C5000284622F01FFF0146404623F0CBFFB4E721
:109C60004946204623F0B4FD4A464E4982462046E6
:109C700024F0E6F824F04AFC8146504623F012F81E
:109C80008346BAF1000F0ED0BAF80E20A2F500728A
:109C900092B2AAF80E20BAF80E2002F4F05212B9CD
:109CA000504622F027FBA9EB07023946284622F04E
:109CB000F1FE0146404623F09DFFE389A3F50073C2
:109CC0009BB2E381E38903F4F05309EB0B0713B96B
:109CD000204622F00FFB384621F016FF304902469D
:109CE000304624F074F82946304606F003FA04465C
:109CF0008CE7304624F0CCFD064698B122F0D2FF26
:109D00008146284622F0CEFF002700F1010BABEB85
:109D1000090A3C46544531DCB9F1000F1CD1C4B9E5
:109D20000134F7E78146ECE75C461FE00146404618
:109D300023F0EEFEFB89A3F500739BB2FB81FB8948
:109D400003F4F05313B9384622F0D4FA04EB0907B0
:109D5000E6E754450AD111E05445E5D001232246F7
:109D600031462846F6F708FD0028D9D1E21B3946CE
:109D7000284622F08FFE07460028D7D1002E3FF458
:109D800024AFF389A3F500739BB2F381F38903F445
:109D9000F053002B7FF419AF304622F0ABFA14E7F2
:109DA000CE450500D8450500F8B506460D460AB370
:109DB000104623F015FD002D044603DA304622F04C
:109DC00071FF0544002C03DA304622F06BFF044497
:109DD0001B2021F031FE25EAE57524EAE4740746EC
:109DE00030B1A54204DA631B2A46314622F00FFE49
:109DF0003846F8BD00296FF00044E9DADEE7F8B52F
:109E000005460C46C2B1104623F0EAFC20EAE07693
:109E1000002C05DA284622F045FF044424EAE474C5
:109E20001B2021F009FE074620B133462246294671
:109E300022F0EDFD3846F8BD6FF00046E8E7F8B5D2
:109E400007460C46CAB1104623F0CAFC20EAE0756A
:109E500024EAE474A542B8BF23464FF01B00BCBF00
:109E60002C461D4621F0E8FD064620B12B1B22465C
:109E7000394622F0CCFD3046F8BD6FF00040E5E7F2
:109E800008B508B1036823B91B20BDE8084021F0DC
:109E9000D3BD002123F09CFCBDE8084024F0BABDEE
:109EA00070B5054686B01B200E4621F0C5FD044660
:109EB00028B3284622F0FCF808B3002E1FDB3246F8
:109EC000294601A81DF0B0F9DDE901239A4209D223
:109ED000059B03B19B5C8DF803300DF10301204617
:109EE000F6F7B4FC049850B1C389A3F500739BB294
:109EF000C381C38903F4F0530BB922F0FBF9204668
:109F000006B070BD37B505461B2021F095FD04460F
:109F100028B1294601A81CF088FD019810B92046F7
:109F200003B030BD23F02CFC24F0F0FA0DF1030156
:109F30008DF803002046F6F789FC01A81CF060FDAF
:109F4000EBE700002DE9F04F89B000AF0D469246D7
:109F5000804617F0F1F84FF0010BF91D0446284632
:109F600087F807B0F7F704FA0023064607F108015F
:109F70005046BB6022F0F3FE0546F0B950461FF094
:109F80003BFD8146B8601CF055FA09F580738342A9
:109F900007D9454958461DF03BFD2437BD46BDE86D
:109FA000F08F09F1070323F00703ADEB030D6D46B6
:109FB0004A46294650461FF00FFDBB68002BECD0E7
:109FC000132C1DD1394A1278002AE6D0F979384885
:109FD000BD61002291427A61FA61BB754FF0402168
:109FE00014BF1346202307F114027E75FAF7CAFD49
:109FF00002460028D1D02F4904201DF009FDCCE7EE
:10A00000002CCAD12C492246404623F019FF814634
:10A01000014607F10C0016F061FB90B32246274978
:10A02000404623F00DFF24F0D8FB3B7CB874FF2B97
:10A0300027D07A7CFF2A24D07A753B75B875FA68E8
:10A040001F4B93FBF2F307F11400012BD8BF2346FB
:10A05000D7F808B097F807A0BB6116F005FB7100B0
:10A0600001F4FF7107F1140016F0B6FAA34514DCF1
:10A07000BAF1000F03D007F1140016F0C1FABB7D4E
:10A08000BB74B87C21F038FD0C490246404623F0F1
:10A090007DFE494623F098FA7FE7295D07F1140019
:10A0A00016F09AFA0134E1E7B9380500F0C0002053
:10A0B000E0BA0020064505001A45050023450500C5
:10A0C00090D003002DE9F04F93B000AF0E46154637
:10A0D000814617F031F84FF0010A044607F11701E5
:10A0E000304687F817A0F7F743F9002D804606DCC5
:10A0F0004FF0000840464C37BD46BDE8F08F1CF0DD
:10A1000099F905F58073834204D95F4950461DF0E3
:10A110007FFCEDE7EB1D23F00703ADEB030D132CE4
:10A120006E463BD1594B1B78CBB1002307F120027F
:10A130004FF040215648C7F82230C7F826307B85BB
:10A1400087F820A087F8218087F822507E62FAF7EE
:10A1500019FD024618B14F4904201DF059FC29464B
:10A1600001201FF030FF80460028C1D001460022A8
:10A1700007F120001FF01CFA354416F8011B07F107
:10A1800020001CF0BAFE07F120001CF017FDB542BC
:10A19000F3D107F120001CF0A9FBABE7002CA7D1FD
:10A1A0003D492246484623F04BFE8246014607F1D0
:10A1B000180016F093FA002859D02246374948462D
:10A1C00023F03EFE24F009FB3B7FB877FF2B4ED0F7
:10A1D0007A7FFF2A4BD0F97D87F8212087F820303D
:10A1E000BA6987F822002E4B93FBF2F307F12000A7
:10A1F000012BD8BF2346F9607B6216F035FA4FEA8F
:10A20000480101F4FF7141F0010107F1200016F04F
:10A21000E3F905F1FF38A8EB04035942594108223C
:10A220004FF0000B07F12000C7E9011216F07CF98E
:10A23000BA6879684FEA4B0B013A40EA0B0BF1D14F
:10A2400007F1200016F09EF9012197F821000FF088
:10A2500087FB06F804B00134A542DCD1FB681BB1D2
:10A2600007F1200016F0CCF997F82230BB77B87FC1
:10A2700021F042FC09490246484623F087FD514639
:10A2800023F0A2F96BE700BFBE440500F0C0002038
:10A29000E0BA0020F34405001A45050023450500F7
:10A2A00090D00300BFF34F8F0549064BCA6802F4F4
:10A2B000E0621343CB60BFF34F8F00BFFDE700BFE9
:10A2C00000ED00E00400FA05024B03495868002243
:10A2D00023F0B6BD582D0020A13B050010B51D4C44
:10A2E0002378834206D002461B490420BDE8104073
:10A2F0001DF08EBB00232370184C206890B129B349
:10A30000114603F0A5F9206850B1C389A3F5007385
:10A310009BB2C381C38903F4F0530BB921F0EAFF68
:10A32000002323600E4C206850B1C389A3F500734D
:10A330009BB2C381C38903F4F0530BB921F0DAFF58
:10A3400000232360074B01221A7010BD114603F051
:10A35000DFF9D8E7FCC00020703B0500F4C0002006
:10A3600000C1002004C1002010B50A460C4600219F
:10A37000FFF7B4FF6CB1E389A3F500739BB2E381EF
:10A38000E38903F4F05323B92046BDE8104021F0DF
:10A39000B1BF10BD10B5094B1C78012C0CD10021A8
:10A3A0000846FCF70DF9064822F0A8FF01462046B2
:10A3B000BDE81040FFF7D8BF10BD00BFFCC00020B3
:10A3C000FE3D05000A460021FFF788BF73B5002255
:10A3D0004149054623F034FD24F098F83F4B4049AD
:10A3E00006460322586823F02BFD044678B12A461E
:10A3F000B1B223F057FCE389A3F500739BB2E3816C
:10A40000E38903F4F05313B9204621F073FF0022CF
:10A410003449284623F014FD24F078F880B200284F
:10A4200046D129460820FDF705FA18B90024204630
:10A4300002B070BD2C4B1C6824B1E38903F5007396
:10A440009BB2E381294E33884FF6FF729A4207D1BF
:10A45000274822F053FF01460820FFF785FFE6E773
:10A4600000221D49284623F0EBFC24F04FF8013070
:10A4700080B2ADF80400ADF8060001A930880EF0F6
:10A48000FBFE0EF00FFD05460028D0D00146082047
:10A49000FFF798FFEB89A3F500739BB2EB81EB8983
:10A4A00003F4F053002BC2D1284621F023FFBEE76E
:10A4B00000210920FDF7BEF90028B7D00A4B1C681F
:10A4C00024B1E38903F500739BB2E381012128469F
:10A4D0000CF0BAF8ABE700BF193C0500582D00207E
:10A4E000263C0500FF3B0500F4C00020B42C0020F2
:10A4F0000B3C050070B5014606460720FDF79AF9AA
:10A5000000283AD01E4B1C6824B1E38903F5007380
:10A510009BB2E3811B4D2B884FF6FF729A4208D104
:10A52000194822F0EBFE01460720FFF71DFF2046E9
:10A5300070BD00221549304623F082FC23F0E6FF6F
:10A540002B8881B2002218460EF094FE0EF0AAFC71
:10A5500005460028EBD001460720FFF733FFEB89C3
:10A56000A3F500739BB2EB81EB8903F4F053002B4E
:10A57000DDD1284621F0BEFED9E70446D7E700BF6B
:10A58000F4C00020B42C00200B3C0500193C050051
:10A590002DE9F04F85B0884600AF002306463946C6
:10A5A00040463B6022F0DBFB0546F8B940461FF011
:10A5B00023FA044638601BF03DFF04F580738342A4
:10A5C00009D9424901201DF023FA2C4620461437B0
:10A5D000BD46BDE8F08FE31D23F00703ADEB030D8F
:10A5E0006D462246294640461FF0F6F90021062016
:10A5F000FDF720F908B90446E8E7354B1C6824B19B
:10A60000E38903F500739BB2E381324B1A884FF65E
:10A61000FF719142984607D12F4822F06FFE014604
:10A620000620FFF7A1FED1E700222C49D7F80090C1
:10A63000304623F005FC23F069FF00221FFA80FA60
:10A640002749304623F0FCFB064600283CD0002278
:10A65000244923F0F5FB24F0C0F8F389A3F5007337
:10A660009BB2F381F38903F4F053834613B9304668
:10A6700021F040FE00239B453B8114BF02230123B0
:10A680003B71391D0123B8F800007B71FD60A7F80C
:10A6900006A0A7F80A900EF0EBFD0EF003FC0546AD
:10A6A000002893D001460620FFF78CFEEB89A3F526
:10A6B00000739BB2EB81EB8903F4F053002B85D13F
:10A6C000284621F017FE81E78346D3E7B938050015
:10A6D000F4C00020B42C00200B3C0500193C050000
:10A6E0002D3C0500383C050038B50D4601460A20D2
:10A6F000FDF7A0F8002839D01D4B1C6824B1E38970
:10A7000003F500739BB2E3811A4B1A884FF6FF7171
:10A71000914208D1184822F0F1FD01460A20FFF7C6
:10A7200023FE204638BD1888144B1B7880B2DBB15D
:10A7300000232A461946F9F7DFFC0EF0B3FB054665
:10A740000028EED001460A20FFF73CFEEB89A3F576
:10A7500000739BB2EB81EB8903F4F053002BE0D143
:10A76000284621F0C7FDDCE70820E6E70446D8E7E5
:10A77000F4C00020B42C00200B3C05000CBE0020CF
:10A78000F0B58BB06D460C4629460FF0DBFF002874
:10A7900000F08D800022012395E80300ADF8182019
:10A7A0008DF81830A023ADF81A30454BADF80C10D9
:10A7B000CDE90732434B0290090C58688DF80E1012
:10A7C0004149099223F03CFB23F0A0FEC3074CBF94
:10A7D0003E4B3F4B089320464FF0C873099321F03E
:10A7E000B4FB002841D000223A49204623F028FB40
:10A7F00024F02AFA02460B4606460F4628F020FDB2
:10A8000090B90022344B3046394628F07FFA2AA30B
:10A81000D3E9002328F0A4FB0022304B28F0C0F835
:10A8200028F04CFDADF8200000222D49204623F0F1
:10A8300007FB24F009FA02460B4604460D4628F0B1
:10A84000FFFC90B90022244B2046294628F05EFAEE
:10A8500019A3D3E9002328F083FB00221F4B28F023
:10A860009FF828F02BFDADF8220002AB93E803001F
:10A87000ADF81410090C04908DF8161008AA06A95A
:10A8800004A80EF0FFFC0EF00DFB044678B1014663
:10A890000220FFF797FDE389A3F500739BB2E381E4
:10A8A000E38903F4F05313B9204621F023FD0BB0E4
:10A8B000F0BD00BFAFF300800000000000889340AF
:10A8C00090000400582D0020643F050090012003F3
:10A8D0001000A0004C3F050000408F400000E03F0A
:10A8E000583F05000A460121FFF7F8BC38B5124B66
:10A8F0001C78012C05461DD100210846FBF760FE9F
:10A9000021460E4823F0BBF9044607F0B1FE5CB1C6
:10A91000E389A3F500739BB2E381E38903F4F05369
:10A9200013B9204621F0E6FC29460120BDE8384055
:10A93000FFF7D8BF38BD00BFFCC0002000C1002019
:10A940007CDF70472DE9F04FAC4D85B02B6800AF30
:10A95000044603F0040308460E463B6021F0F5FA76
:10A96000002800F0BC800022A549304623F068FA98
:10A97000B0B123F0CBFD4FF47A73584340F271230A
:10A9800090FBF3F080B2B0F5804F9E4B28BF4FF4A0
:10A99000804020281A8838BF2020824218BF1880A3
:10A9A00000229949304623F04BFA38B123F015FFC5
:10A9B0002B68002875D023F400632B600022934994
:10A9C000304623F03DFA38B123F007FF2B6800280A
:10A9D0006AD023F480532B6000228D49304623F047
:10A9E0002FFA8146002800F08480002307F10C0133
:10A9F000FB6022F0B4F98046002864D148461EF07E
:10AA0000FBFF8246F8601BF015FD0AF58073834258
:10AA10004DD9804901201CF0FBFFB9F80E30A3F599
:10AA200000739BB2A9F80E30B9F80E3003F4F0535E
:10AA300013B9484621F05EFC204621F086FA824692
:10AA400008B9002C58D131462046FCF761FC002C97
:10AA500040F0D2800024704D70496868224623F08F
:10AA600041FE32466E49686823F03CFE5CB1E389E2
:10AA7000A3F500739BB2E381E38903F4F05313B9A8
:10AA8000204621F037FC3B680BB10CF0B1F9404691
:10AA90000EF066FA3B6843B30CF0B8F90EF060FABA
:10AAA00023E043F4006388E743F4805393E70AF11B
:10AAB000070323F00703ADEB030DE846524641467A
:10AAC00048461EF089FF11234146BA893B7207F1BF
:10AAD0000800FFF735FF80460EF042FA9DE746B1C9
:10AAE0003246504903201CF093FF1437BD46BDE8A1
:10AAF000F08F4FF000089FE7204621F01EFA7860A3
:10AB0000002868D0E38903F500739BB2E3812B68CA
:10AB100023F47F0323F40043214607F10C002B604C
:10AB20001BF083FFD346F86850B9BAF1000F92D0FA
:10AB3000BBF1010F8FDD2B6843F400432B608AE7E4
:10AB400022F01EFE814621F000FA10B9B9F1000F83
:10AB50001ED131464846FCF7DBFB8246F86810B14F
:10AB6000514622F037FCBAF1000F0ED0BAF80E3081
:10AB7000A3F500739BB2AAF80E30BAF80E3003F4B6
:10AB8000F05313B9504621F0B5FBD7F804A009E003
:10AB9000484621F0D2F90028F7D1484621F0B1F912
:10ABA0000028F2D10BF1010BB9F1000F0ED0B9F86A
:10ABB0000E30A3F500739BB2A9F80E30B9F80E3031
:10ABC00003F4F05313B9484621F094FB07F10C004D
:10ABD0001BF016FFA7E7204621F093F900283FF469
:10ABE00039AFE38903F500739BB2E3812B6823F44B
:10ABF0007F0323F40043A1E704462CE7F8C00020BC
:10AC0000143F0500B22C00201D3F0500293F050020
:10AC100052400500B9380500582D0020333F05008B
:10AC20003D3F05007F3D050072DF7047F0B5264BC4
:10AC3000264983B0044600AF0246586823F052FD0F
:10AC4000204621F07AF9E8B10023391D20467B60C7
:10AC500022F085F8054668BB20461EF0CDFE06466C
:10AC600078601BF0E7FB06F58073834217D918491B
:10AC700001201CF0CDFE174903201CF0C9FE0C3743
:10AC8000BD46F0BD204621F03CF90028DCD1002C67
:10AC9000F5D02246104903201CF0BAFEEFE7F31D61
:10ACA00023F00703ADEB030D6D46324629462046DF
:10ACB0001EF092FE00213B792A460846FFF7B4FFBA
:10ACC0000EF04EF9DBE700BF582D0020D23F050003
:10ACD000B9380500DB3F05000740050070B5384C6A
:10ACE00038492068002223F0ABF8054678B10021EE
:10ACF00001200CF053F8EB89A3F500739BB2EB81B4
:10AD0000EB8903F4F05313B9284621F0F3FA00223B
:10AD10002D49206823F094F8054670B101200CF00D
:10AD200013F8EB89A3F500739BB2EB81EB8903F475
:10AD3000F05313B9284621F0DDFA00222349606858
:10AD400023F07EF8002205462149606823F078F858
:10AD5000064605B918B131462846FFF7F3FD2846E7
:10AD6000314622F031FC00221A49606823F068F86D
:10AD7000054668B10BF0EAFDEB89A3F500739BB2C1
:10AD8000EB81EB8903F4F05313B9284621F0B2FAB2
:10AD900060681149002223F053F8044678B1FFF7A8
:10ADA00045FFE389A3F500739BB2E381E38903F4D4
:10ADB000F05323B92046BDE8704021F09BBA70BD26
:10ADC000582D0020C73F0500F43B0500333F050028
:10ADD0003D3F0500F8400500D23F050070B58EB03C
:10ADE00004460D4601466846164610F05FF848B323
:10ADF0003EB140F2FF339D42A8BF1D46012DB8BFB2
:10AE00000125BDF9143002330FD10F49204623F03C
:10AE10004FFC0E49204623F04BFC0D49204623F001
:10AE200047FC0C49204623F043FC6846ADF814501B
:10AE300010F002F8E38903F500739BB2E38120462A
:10AE40000EB070BD0446FAE7DA43050097440500EA
:10AE5000DF4305009C4405002DE9F04D2DED028BEC
:10AE600090B004460E46014602A890461F469DF843
:10AE7000685010F01BF8002800F09980304623F04D
:10AE800071FE4046B0EE408AF0EE608A23F06AFE22
:10AE900038465BEC10AB23F065FE8DED000BB8F18E
:10AEA000000F7ED0002F7CD00022424B51EC180BBB
:10AEB00027F02CFF28F0DAF900223E4B07465946CE
:10AEC000504627F023FF28F0D1F99DED000B00221A
:10AED000384B064651EC100B27F018FF28F0C6F946
:10AEE000BDF80D2012F4607287F3080386F308069C
:10AEF00080F3080008D0B2F5C07F29D020D8802A7E
:10AF00002AD0B2F5807F2CD09DF81320102A2FD1A3
:10AF1000D910B210C90241EA421141EAE000002D05
:10AF200043D0059002A80FF087FFE38903F5007373
:10AF30009BB2E381204610B0BDEC028BBDE8F08DE2
:10AF4000B2F5007F11D0B2F5207FDDD1324601E0AD
:10AF50001A463346064606E01A460346304616466B
:10AF6000D2E71A4603461046CEE71A463346F6E7BE
:10AF7000202A06D11A0442EA0622104340F07F40FC
:10AF8000CDE7182A04D1190441EA06210843C6E78F
:10AF900033441844B0F5C07F4FF0FF30B8BF0020F5
:10AFA000BDE7304622F01CFCB9E70690BAE704463C
:10AFB000C0E700BF0000704010B58EB00C460146DF
:10AFC00068460FF073FF40B1BDF80530DB0648BF9F
:10AFD00084F001041CB1BDF809000EB010BDBDF82D
:10AFE0000700FAE72DE9F04F97B00546014608A89B
:10AFF0000FF05CFF28B94FF00009484617B0BDE8D4
:10B00000F08F00F0D7FF04460028F4D00021284636
:10B01000FFF7D2FF012107462846FFF7CDFF05467F
:10B0200038469DF82B6020F06FFD3D4902462046D2
:10B0300022F0CDFE284620F067FD3A490246204620
:10B0400022F0C5FE012E07D0304620F05DFD3649C6
:10B050000246204622F0BBFE05FB07F07043073096
:10B060000021C01022F0E4F8814668B9E389A3F515
:10B0700000739BB2E381E38903F4F053002BBAD150
:10B08000204621F037F9B8E70146002203A81CF05A
:10B09000CBF80025A846AB46AA46DDE9031291424B
:10B0A00013D3069850B1C389A3F500739BB2C38133
:10B0B000C38903F4F0530BB921F01CF94A461B492C
:10B0C000204622F084FEA14697E70FFA8BF20FFA92
:10B0D0008AF108A80FF07CFE0AF1010A08FA06F8C6
:10B0E000574548EA000806EB050203DC0BF1010BAB
:10B0F0004FF0000A15460AE0083D28FA05F1C9B2EA
:10B1000003A801921BF0A6FE019A4FEA1828072D0A
:10B11000F2D8D5086FF0070303FB0525BDE700BF94
:10B120009A43050090440500A0430500645D0500B6
:10B130002DE9F74F21F00045894616461F464FF08E
:10B14000FF32414B29468046044628F079F8002812
:10B1500076D14FF0FF323C4B4046294628F066F846
:10B1600000286DD132463B463046394628F068F813
:10B17000002865D1002200234046494628F038F8CF
:10B1800028B309F10045002200233046394628F053
:10B190002FF810B107F100431F460022002330466C
:10B1A000394628F01BF878B94FF0FF32264B30466D
:10B1B000394628F027F838B14FF0FF32224B2046AD
:10B1C000294628F01FF8E8B90024002522E04D4662
:10B1D000D9E700221D4B2046294627F097FDCDE9EF
:10B1E0000001B246BB4652465B46DDE9000128F04D
:10B1F00013F852465B46E0B92046294627F0CEFBBD
:10B2000004460D4622462B463046394627F0FAFFC3
:10B210000028DED1002200234046494627F0E8FFFF
:10B2200010B105F100431D462046294603B0BDE894
:10B23000F08F1046194627F0B3FB82468B46D2E7C3
:10B240000024034DF0E700BFFFFFEF7F0000E03F69
:10B250000000F87F2DE9F84355EC114B11EE100A70
:10B26000294657EC106B28F001F80928804619D8B8
:10B2700027F0E2FC22462B4627F0B0FF90B1B8F150
:10B28000000F63D030463946B8F1010F03D141ECCD
:10B29000100BBDE8F88332463B4627F037FD08F136
:10B2A000FF38F1E7002200233046394627F0A0FF9F
:10B2B0000022D8B3284B20462946FFF739FF002249
:10B2C000002327F08BFFF0B300224FF0804320468D
:10B2D0002946FFF72DFF0022002327F07FFFB0460D
:10B2E00007F1004949EC108B68B125F05DFD22465D
:10B2F0002B4651EC100B27F009FDBDE8F84341EC5B
:10B30000100B25F0CDBC25F04FFD22462B4651EC0D
:10B31000100B27F0FBFC41EC100B25F0C1FC53ECAB
:10B32000102B10EE100A03F10041B0E70023304665
:10B33000394627F053FF30B100220023204629462A
:10B3400027F060FF28B147EC106BCEE700200249E0
:10B350009DE7002000219AE70000F03F38B5164C29
:10B36000164B1546002291420CBF2146194622F089
:10B3700067FD0446F0B15DB100232B7020F0C1FDE4
:10B3800030B1A38803F00F03022B04BF01232B70FD
:10B39000204621F06DFAE389A3F500739BB2E381A7
:10B3A000E38903F4F053054613B9204620F0A2FFC9
:10B3B000284638BD0546FBE7645D0500614605008B
:10B3C0002DE9F04F8FB0CDE900230D4600229C49B6
:10B3D000DDF860A09DF864B0044622F031FD23F052
:10B3E000FCF930B1974901201CF012FB0FB0BDE809
:10B3F000F08F284615F0ACFF08B99349F3E7DDE973
:10B40000006323F000474FF0FF32904B304639463F
:10B4100027F016FF80B94FF0FF328C4B304639468B
:10B4200027F004FF40B984A3D3E90023DDE900013C
:10B4300027F0DEFE074608B18549D4E70EF02EFB63
:10B44000CDE90201504620F080FD0646002800F0BC
:10B4500087803A467F49504622F0F2FC23F0F4FB05
:10B4600021F000490F464FF0FF32784B494606461F
:10B4700027F0E6FE00BB4FF0FF32744B30464946E2
:10B4800027F0D4FEC0B9002200233046394627F009
:10B49000CDFE88B10022704B3046394627F036FC8D
:10B4A00000226E4B27F032FC00226B4B27F058FD38
:10B4B00027F08CFFCDE9020100226949504622F0B5
:10B4C000BFFC23F08AF906464FF0000841460DF113
:10B4D000170220468DF81780FFF740FF42460746C7
:10B4E00001212046FFF73AFF9DF817308046002BD8
:10B4F0003FD0BBF1000F14BF4FF005094FF0060914
:10B50000DDE900230020544927F02AFD0022534B97
:10B5100027F0FCFB0022504B27F022FD27F056FFBE
:10B5200026B1B8F1000F14BF46463E46029B089074
:10B530001818039B8DF8349043EB0101B9F1030F08
:10B54000CDE9060102D0B9F1050F1AD1454B33F808
:10B550001530ADF8323013BB43481CF0F7F837E034
:10B56000BAF1000FB0D05246404901201CF050FA09
:10B57000AAE7BBF1000F14BF4FF003094FF0040915
:10B58000BEE709F00509B9F1040FE5D1384B05EB29
:10B59000450213449B78002BDED08DF83250002FEB
:10B5A00047D0344BFB1A1B1101339BB2ADF8283046
:10B5B00026B1304BF61A36110136B6B206A8ADF8F0
:10B5C0002A6015F043FB06A815F06CF90028C3D0DB
:10B5D0004146384621F0F8FF012020F08DFA184945
:10B5E0000246204622F0F3FB9DED000B20F07AFA94
:10B5F00021490246204622F0EAFB204B20495868A8
:10B60000032222F01DFC054600283FF4EFAE214640
:10B6100022F07EFAEB89A3F500739BB2EB81EB89F4
:10B6200003F4F053002B7FF4E1AE284620F062FED5
:10B63000DCE63B46BAE700BFFCA9F1D24D62503FC1
:10B640000F4705008B460500A7460500FFFFEF7F6B
:10B65000B34605009E66050000408F400000304163
:10B66000D34605000CC10020DA460500214605003E
:10B67000243A0500742D0020F5460500582D0020C1
:10B68000FA4605002DE9F341054608460C4690466A
:10B6900057EC106B0EF012FD0022002351EC100B42
:10B6A00027F0A6FD38B9CDE9008032463B46214659
:10B6B0002846FFF785FE02B0BDE8F08107B50123FB
:10B6C000CDE9002353EC102BFFF77AFE03B05DF8B1
:10B6D00004FB00002DE9F04F684B694958688DB0B4
:10B6E000002222F0ADFB0746A8B1014602A81BF0DC
:10B6F0009CF9DFF8A8A1DFF8A8B1029878B9FB8916
:10B70000A3F500739BB2FB81FB8903F4F05313B9DB
:10B71000384620F0EFFD00200DB0BDE8F08F22F09C
:10B720002FF800225146044622F08AFB23F055F8F8
:10B730008046002800F09F80002211462046FFF737
:10B740000DFE0646002851D04E4D451B2D110135EA
:10B75000ADB204AA03A94C48ADF80C5014F0FAFF9E
:10B760008046002844D102464849204622F068FB22
:10B770000123039003AA2046454915F077FC03985E
:10B7800050B1C389A3F500739BB2C381C38903F48D
:10B79000F0530BB920F0AEFD002020F0ADF951467A
:10B7A0000246204622F013FB5EB1F389A3F5007335
:10B7B0009BB2F381F38903F4F05313B9304620F0C0
:10B7C00099FD5CB1E389A3F500739BB2E381E38942
:10B7D00003F4F05313B9204620F08CFDB8F1000FAC
:10B7E00045D1394602A81BF0F1F886E70546B0E7D7
:10B7F000BDF82230002BD7D0BDF820904B45D3D0D8
:10B80000B9EB050318BF01230922594620460193CD
:10B8100022F016FB22F07AFE019B8342C4D0184628
:10B8200020F072F959460246204622F0D0FA174B12
:10B8300018490022A94518BF1946204622F000FBEE
:10B840000123039003AA2046134915F00FFC039827
:10B850000028A9D0C389A3F500739BB2C381C38913
:10B8600003F4F053002B9FD120F044FD9CE702A885
:10B870001BF0C6F841E7002CA4D1B2E7582D0020F8
:10B88000FA460500742D0020B7F90300645D050039
:10B890006946050061460500814605000F47050021
:10B8A0007346050013B500221B49044622F0C8FA6E
:10B8B00022F093FF28B9194901201CF0A9F802B021
:10B8C00010BD002220461146FFF748FD044600B394
:10B8D000134BC31A1B1101339BB20DF10601114822
:10B8E000ADF8063014F07AFF18B90F4901201CF0AA
:10B8F0008FF85CB1E389A3F500739BB2E381E38920
:10B9000003F4F05313B9204620F0F4FCFFF7E2FEF5
:10B91000D5E70346E1E700BF0F470500FF460500F6
:10B92000742D0020B7F903001747050070B50446D1
:10B930008AB01B200E4620F07FF80546002838D03C
:10B94000204622F0A5FF00220146044605A81BF070
:10B950006BFC0022294668461BF066FCDDE90532D7
:10B96000934229D3089850B1C389A3F500739BB2C1
:10B97000C381C38903F4F0530BB920F0BBFC0398D7
:10B9800050B1C389A3F500739BB2C381C38903F48B
:10B99000F0530BB920F0AEFC5CB1E389A3F5007362
:10B9A0009BB2E381E38903F4F05313B9204620F0FE
:10B9B000A1FC28460AB070BD099939B1C95C66B1CD
:10B9C000A1F16103192B01D82039C9B268461BF0D7
:10B9D00033F805A81BF0ACF8C0E7A1F14103192B1F
:10B9E000F4D82031F1E72DE9F84380460C4617469C
:10B9F000994620F05DFB18B900242046BDE8F88385
:10BA0000204622F045FF05460028F5D0404621F0AB
:10BA100049F90446284621F045F984420EDAEB89BB
:10BA2000A3F500739BB2EB81EB8903F4F05313B9D8
:10BA3000284620F05FFC4FF0FF34DEE7241AB9F10E
:10BA4000000F0DD13846661C20F0A7FA88B338469F
:10BA500021F0C6FE041E2CDBA642E0DB012710E02D
:10BA6000384620F09AFA38B1384621F0B9FE00285D
:10BA700022DB8442A8BF04464FF0FF36374600E081
:10BA80003C44B442CBD00123224629464046F4F739
:10BA900073FE0028F4D1EB89A3F500739BB2EB8110
:10BAA000EB8903F4F053002BA7D1284620F022FCA9
:10BAB000A3E701270024E4E74FF0FF363746F9E714
:10BAC0002DE9F04F9BB08A461546074622F0E0FE6E
:10BAD00006465046F5F740F980462846B8F1000F73
:10BAE00000F06A8120F049FA002846D0EB8903F57E
:10BAF00000739BB2EB81002020F006F8AB490246B0
:10BB0000504622F064F96721504604F0B1FA3146FC
:10BB10000490504604F0EEFA04469CB1204620F012
:10BB2000D1F918B91AF07EFC804680B3E389A3F5F9
:10BB300000739BB2E381E38903F4F05313B9204609
:10BB400020F0D8FB37465DB1EB89A3F500739BB2BB
:10BB5000EB81EB8903F4F05313B9284620F0CAFBBC
:10BB6000049B002B00F0D58000201FF0CDFF8F49F3
:10BB70000246504622F02BF9CBE0284620F098FAF6
:10BB80000028B3D1284622F083FE0546B3E741469C
:10BB9000204621F01DFE424685490390204622F0B2
:10BBA0004FF922F0B3FC0590039821F07BF8414651
:10BBB0000690059A304620F06DFF42460146074642
:10BBC00008A81BF031FB08A81AF084FF284620F0D3
:10BBD000D4F90DF134080246002856D0039B039A8D
:10BBE000DB8903F500739BB2D3814FF001090D92FD
:10BBF0004946204621F0ECFD09F101038346002867
:10BC00003FD102466A490793204622F019F91AAB40
:10BC100003EB8902674942F8340C5A46204622F069
:10BC20000FF9079B1AAA02EB830309F1020943F8F3
:10BC3000340C0DAB5A465946CDE9009328465B4675
:10BC40001CF07EFF22F0E6FE0DA98046484621F05A
:10BC50003DFC5A46414608A81DF03BFDB8F1000FD7
:10BC600027D0B8F80E20A2F5007292B2A8F80E20E4
:10BC7000B8F80E2002F4F052DAB9404620F03AFB50
:10BC800017E048F829B09946B2E7294640461BF02C
:10BC9000CBFADDE90D3293423FD3109848B1C38906
:10BCA000A3F500739BB2C381C38903F4F053002B47
:10BCB000E4D0089A0A9B134403F10108DDE9053139
:10BCC0000B4408A81A4631461DF003FD0B9850B1ED
:10BCD000C389A3F500739BB2C381C38903F4F053F6
:10BCE0000BB920F007FB0399304621F06DFCE38986
:10BCF000A3F500739BB2E381E38903F4F05313B916
:10BD0000204620F0F7FA049B002B40D1002D7FF451
:10BD10001BAF38461BB0BDE8F08F119999B3C95CD1
:10BD2000242930D140461AF003FF119B2BB30D9A02
:10BD300013F802B0ABF13103082B1FD8ABF130017F
:10BD4000204621F045FD8146C0B10146002208A8E9
:10BD50001DF0BFFCB9F80E30A3F500739BB2A9F833
:10BD60000E30B9F80E3003F4F05313B9484620F002
:10BD7000C1FA40461AF0DCFE8BE79B46242108A856
:10BD80001AF05AFE594608A81AF056FEF1E7404646
:10BD90001FF0BAFE05490246504622F018F839460F
:10BDA000504604F0A7F93E460446B6E6CE450500E7
:10BDB000D8450500C845050022F06AFD05465046F5
:10BDC00022F066FD43460146044642463846FFF7E8
:10BDD0000AFEB0F1000928DB4A464146304620F011
:10BDE00059FE6FF0004342462946074620F00FFEF9
:10BDF000204620F057FF6FF0004309EB0002314668
:10BE0000384620F004FE5EB1F389A3F500739BB2BF
:10BE1000F381F38903F4F05313B9304620F06AFA42
:10BE20002946204621F0D0FB73E73746F8E700BFEC
:10BE30002DE9F84F07460D4620F03AF918B90024CD
:10BE40002046BDE8F88F002DF9D02846F4F784FF8E
:10BE50000446002866D000201FF056FE52490246D4
:10BE6000284621F0B4FF3946284604F043F96721FB
:10BE70000446284604F0FCF80028E1D01FF095FEA7
:10BE800006460028DBD0DFF82491DFF81CA184B13E
:10BE9000204620F017F88046A8B1E389A3F5007387
:10BEA0009BB2E381E38903F4F05313B9204620F0F9
:10BEB00021FA00201FF028FE3B490246284621F0C7
:10BEC00086FF3446BCE74146204621F081FC4246CD
:10BED00049468346204621F0B3FF22F017FB8046F7
:10BEE000584620F0DFFE59468044304621F082FE5D
:10BEF000E389A3F500739BB2E381E38903F4F05374
:10BF000013B9204620F0F6F940461FF0FDFD5146DA
:10BF10000246284621F05BFF3946284604F0EAF83D
:10BF20000446B4E7284622F0B3FC23460146054602
:10BF300022463846FFF757FD061E26DB1FF035FE6A
:10BF4000044688B9002D3FF47AAFEB89A3F500735E
:10BF50009BB2EB81EB8903F4F053002B7FF46FAFBE
:10BF6000284620F0C7F96BE7294621F0D1FD30467D
:10BF70001FF0CAFD0D490246204621F028FF2A463F
:10BF80000B49204621F023FF5AE7002D3FF457AF1D
:10BF9000EB89A3F500739BB2EB81EC8914F4F054A8
:10BFA0007FF44DAFDCE700BFCE450500D845050066
:10BFB000C845050005201FF03FBDFFF7FBBFFFF799
:10BFC000F9BF2DE9F8430F469046814618B1067A2D
:10BFD0000025AE4201D8BDE8F883D9F80030D9F881
:10BFE000040033F83530184421F088F9044601463E
:10BFF0004046B8475CB1E389A3F500739BB2E38187
:10C00000E38903F4F05313B9204620F073F90135A6
:10C01000DFE722F093BB0000002201491BF0F4BED1
:10C02000AA3905002DE9F04107460C460026236990
:10C03000B34201DCBDE8F081E568013D002D10DA76
:10C04000257A284615F084F948B1617A28460DF022
:10C0500087FC617A207A81F001010DF081FC0136C4
:10C06000E5E714F80580404615F072F920B107F0B5
:10C07000010140460DF074FC7F10DEE710B5044668
:10C0800030B90246054903201BF0C2FC204610BD12
:10C09000C38903F500739BB2C381F7E78E64050083
:10C0A0002DE9F04F89B08946009015F045F84946D2
:10C0B000044602A814F012FB60B3132C40F0068172
:10C0C0009DF80C40204615F043F99DF80D5018B12D
:10C0D000284615F03DF900BB224629468C481BF046
:10C0E00055FBB9F1000F00F00E810122894900983B
:10C0F00021F000FE70B1494621F06CF950B1C389BE
:10C10000A3F500739BB2C381C38903F4F0530BB949
:10C1100020F0F0F809B0BDE8F08F7F49029E7F4B18
:10C1200004EB440405EB45050C440D449E4294F891
:10C1300001806F7858DD7A4B9E42D4BF4FF0806605
:10C140004FF0CD66774A784C13785BB323681BB108
:10C15000764B1021C3F880104FF040234FF0FF3191
:10C16000C3F80813D3F800120021C3F80012C3F873
:10C170000015012184F8221094F8271079B9D3F81A
:10C1800008154FF0A04001F5E07140F2023540F88B
:10C190002150D3F80C3503F5E07340F82350002309
:10C1A00084F8223094F8223001251570FBB1082262
:10C1B0005F4904201BF02CFC9DF80C40204615F034
:10C1C000C7F820B14FF4207120460DF0E3FD9DF833
:10C1D0000D40204615F0BCF8002882D04FF4945151
:10C1E00020460DF0D7FD7CE74FF0CC76AAE79DF80E
:10C1F0001E2084F827209DF81D20A360C4E9003389
:10C2000084F8253084F8243072B34FEA8800B900EE
:10C2100000F1A04001F1A04140F20C624FF0A04BB0
:10C22000C0F8002705FA08FAC1F80027BD4040F21F
:10C230000D620193CBF808A5CBF80855C0F800278C
:10C24000C1F800270420F6F753F9019BDBF810151D
:10C250000D422BD043B14FF0A04A0420CAF80C5530
:10C26000F6F746F9CAF808554FF0A04308F5E07113
:10C2700040F20C6243F8212007F5E07143F82120D9
:10C280004FF040231D46C3F80885C3F80C75C3F86A
:10C29000246522681AB106210420F8F7CDFE052393
:10C2A000C5F80035022384F8223085E70193042085
:10C2B000CBF80CA5F6F71CF9CBF808A50420F6F787
:10C2C00017F9019B0133092BC0D1C4E7002C7FF47F
:10C2D00008AF9DF80C00FF2807D001210DF040FBAE
:10C2E00003219DF80C000DF077FE9DF80D00FF284E
:10C2F0003FF4F7AE01210DF033FB03219DF80D0053
:10C300000DF06AFEEDE60349009822F0D1F901E74D
:10C31000875E05001A450500243A050097AB020028
:10C3200087F50400F0C00020E0BA002000E100E042
:10C33000B65E0500F0B58DB00D4616461C4614F0ED
:10C34000FBFE12289DF8487005D02E4901201BF0F5
:10C350005FFB0DB0F0BD16B90CB90F2403262A4BB4
:10C360001B78F6B2E4B25BB92849ADF810306FF033
:10C37000FF02CDE9011201A8254A03920DF028FD24
:10C38000FF2F03D00021384615F04AFE28461FF043
:10C3900004FE70B1284621F023FA22463146C0B28D
:10C3A000F4F7DAFEFF2FD4D00121384615F038FE1D
:10C3B000CFE728461FF0A7FEE8B1802383F311885A
:10C3C0000122294601A81DF036F901A81AF0DDFA6C
:10C3D000054601A825B91AF099FA85F31188E1E715
:10C3E0001AF0CBFC22463146C0B2F4F7B5FE01A8E4
:10C3F0001AF0FEFBE9E72A46064901201BF008FB7C
:10C40000D0E700BFF2680500E2C00020A08601006E
:10C41000000108001A690500F0B58DB00D461646FA
:10C420001C4614F089FE12289DF8487005D02F494B
:10C4300001201BF0EDFA0DB0F0BD16B90CB90324C4
:10C4400001262B4B1B7806F00F0604F00F045BB996
:10C450002849ADF810306FF0FF02CDE9011201A8B4
:10C46000254A03920DF0B4FCFF2F03D0002138467B
:10C4700015F0D6FD28461FF090FD70B1284621F03A
:10C48000AFF922463146C0B2F4F726FEFF2FD2D0D4
:10C490000121384615F0C4FDCDE728461FF033FED4
:10C4A000E8B1802383F311880122294601A81DF0F9
:10C4B000C2F801A81AF069FA054601A825B91AF0D0
:10C4C00025FA85F31188E1E71AF057FC2246314638
:10C4D000C0B2F4F701FE01A81AF08AFBE9E72A4688
:10C4E000064901201BF094FAD0E700BFCA68050096
:10C4F000E2C00020A0860100000108001A690500C2
:10C5000013B50C4614F018FE8DF8070009380528FD
:10C5100005D80DF10702034920461DF0FDF802B0D1
:10C5200010BD00BFE5C8020010B50C4614F0A1FE16
:10C530002146BDE8104015F073BD08B514F099FE12
:10C540000021BDE8084015F06BBD08B514F091FE60
:10C550000121BDE8084015F063BD70B586B00E46F8
:10C5600002AA01A911F048FC60B16EB9FF2502AA28
:10C57000019930461DF0D0F8FF2D03D00121284647
:10C5800015F04EFD06B070BD31680029EEDD0139B1
:10C59000304621F01DF904461FF068FE30B32046F6
:10C5A00014F067FE0546304622F030F850B1C389DA
:10C5B000A3F500739BB2C381C38903F4F0530BB995
:10C5C0001FF098FE5CB1E389A3F500739BB2E38191
:10C5D000E38903F4F05313B920461FF08BFEFF2DBF
:10C5E000C5D00021284615F01BFDC0E7002CBDD0AA
:10C5F000FF25E8E738B50C46054651F8043B984757
:10C60000002DA2BFA3690133A36100280BDB04F155
:10C610001C05C1B228461AF070FC28461AF0CEFA62
:10C6200063690133636138BD2DE9F04198B00E466E
:10C63000174607A908AA11F0DFFB002800F0A48024
:10C64000FF2F03D00021384615F0EAFC30461FF0DA
:10C65000A4FC80463046B8F1000F1AD021F0C0F893
:10C6600008A920EAE070079B9847002804DA08A987
:10C670004FF0FF30079B98471FF046FA0446FF2F04
:10C6800003D00121384615F0CBFC204618B0BDE898
:10C69000F0811FF00DFD054600284DD01B201FF036
:10C6A000CBF931460446424602A81AF0BDFD464683
:10C6B000DDE902239A4216D3059880BB4645DEDDAC
:10C6C00019F0B0FE0028DAD108A9079B4FF0FF301F
:10C6D00098470DF107018DF80700204608F1010881
:10C6E000F4F7B4F8EAE719F09DFE0028E4D10698C3
:10C6F00008B1029BC05C079B08A99847002806F177
:10C70000010608DB8DF807000DF10701204608F14E
:10C710000108F4F79BF802A81AF00AFAC8E7C389DF
:10C72000A3F500739BB2C381C38903F4F053002BBC
:10C73000C4D11FF0DFFDC1E730461DF05DF90146B1
:10C7400001201DF040FC0446002898D001462A46EE
:10C750000EA8CDE90C551CF02BFF07AA0B4930465B
:10C760001CF0DAFFDDE90C239A4203DB0EA81AF075
:10C77000BDF884E719F056FE0028F7D107A94FF05D
:10C78000FF30FFF737FFEDE704467EE7F5C502000F
:10C790007FB50C46054614F0CFFC21460646684698
:10C7A00011F086FAD0B1122E1AD168460DF010FBA6
:10C7B00074B301221949284621F09CFA70B1214630
:10C7C00020F008FE50B1C389A3F500739BB2C3816A
:10C7D000C38903F4F0530BB91FF08CFD04B070BD96
:10C7E000002EFBD19DF80500FF2802D001210DF09D
:10C7F000F3FB9DF80600FF2802D004210DF0ECFBAE
:10C800009DF80700FF28D3D001210DF0E5FBCFE70D
:10C810000249284621F04CFFE0E700BF1A45050019
:10C82000F4F795B822F014BEF0B589B01FF0BDF949
:10C83000044638B310224FF4D82500210DEB020036
:10C840000095F2F76FFE04A9284622F089FCC8B1D2
:10C8500001AD06AE0027059B01330CD196E803001D
:10C8600085E8030028468DF80C7020F047FD01464E
:10C87000204621F0BFF9002204A9684622F0C2FC3C
:10C880000028E8D1204609B0F0BD38B522F01CFEE2
:10C8900022F01EFD044688B1002120F099FAE389B8
:10C8A000A3F500739BB2E381E38903F4F0530546DB
:10C8B00013B920461FF01EFD284638BD0546FBE78C
:10C8C00008B522F001FEBDE8084022F001BD08B520
:10C8D00022F0FAFDBDE8084022F007BD4FF4D82051
:10C8E00022F02ABD0B78C1B2184614F08DBA0000B0
:10C8F000024B03495868052221F0A2BA582D0020A6
:10C90000386105002DE9F04389B01F4680460C468A
:10C91000914614F011FCA0F10903DBB2052B064689
:10C920003AD80E280FD1374B1B7863B94FF0FF323E
:10C930004FF41651CDE9041204A8334A06928DF83B
:10C940001C30F8F79FFB314D8DF80060B9F1000FF6
:10C9500003D0204621F09CFF04466A462946204623
:10C960001CF0DAFEB9F1000F0CD05CB1E389A3F53D
:10C9700000739BB2E381E38903F4F05313B92046BB
:10C980001FF0B8FC2FB169460D20A84769460A2060
:10C99000A84709B0BDE8F0830028FAD102461C4937
:10C9A000404621F04DFA324605461A49404621F0EC
:10C9B00047FA0DF11008064602462946404613F094
:10C9C000ABFC5EB1F389A3F500739BB2F381F389ED
:10C9D00003F4F05313B930461FF08CFC5DB1EB89C2
:10C9E000A3F500739BB2EB81EB8903F4F05313B909
:10C9F00028461FF07FFC98E80F006D4607C52B7096
:10CA0000054DA3E7F1C000200800010069210400E2
:10CA1000BC5C05001A4505007113040000231A468A
:10CA2000FFF770BF01231A46FFF76CBF00230122F6
:10CA3000FFF768BFF0B585B0044614F07DFB002217
:10CA400005463C49204621F0FBF9064628B93A49FB
:10CA500001201AF0DDFF05B0F0BD00223749204665
:10CA600021F0EEF9324601460746684613F054FCC1
:10CA70003946304620F0A8FD3049204621F018FE06
:10CA80002C49204621F014FEA5F10903DBB2052B49
:10CA900044D900222A49204621F0D2F908B321F0D6
:10CAA00035FDC4B2002120460CF03EFE002013F0FC
:10CAB000C7FB0546A8B121461FF0EEFC044618B19D
:10CAC0000146284621F036FD28461FF019FE20B900
:10CAD0001C4B1D49586821F0EBFD2946204620F0EB
:10CAE00073FD9DF80600FF2802D000210DF074FAB6
:10CAF0009DF80700FF2802D000210DF06DFA9DF887
:10CB00000400FF2802D000210DF066FA9DF8050010
:10CB1000FF28A0D000210DF05FFA9CE7A5F10D03DE
:10CB2000DBB2012BDDD8FF220021284614F09CFC4B
:10CB3000D7E700BF1A45050095680500BC5C0500F5
:10CB4000BC680500582D0020C1680500F7B514F039
:10CB500090FB054614F0FCFB18B90024204603B0F6
:10CB6000F0BDFFF727FA04460028F6D005EB45058F
:10CB7000224B5E195B5D40338DF8043001A8002321
:10CB80008DF8053020F0BAFB1D490246204621F001
:10CB90001EF970781EF0B8FF1A490246204621F0AF
:10CBA00016F9B57885B1FFF705FA074660B11EF0B2
:10CBB000FCFF064690B905F01F001EF0A5FF1249C4
:10CBC0000246204621F003F9FFF7F4F90246002857
:10CBD000C4D00E49204621F0FAF8BFE7AB0606D5CF
:10CBE00001201EF091FF0146304621F003F8324645
:10CBF0000749384621F0EBF8DDE700BF243A05008D
:10CC0000D4640500D9640500E2640500EA64050007
:10CC1000DD640500F0B585B005460F46144614F0F6
:10CC20008BFA0646D4B922465B49284621F008F91A
:10CC3000044622463946684613F06EFBA0B95CB143
:10CC4000E389A3F500739BB2E381E38903F4F05316
:10CC500013B920461FF04EFB05B0F0BDE38903F584
:10CC600000739BB2E381E4E700981EF04DFF4B494F
:10CC70000246284621F0ABF87CB1224646492846B8
:10CC800021F0A5F8A6F10903DBB2052B0AD80E2E78
:10CC9000E2D16846F8F7F6F9DEE73F49284621F089
:10CCA00007FDEFE7002ED7D19DF80500FF2807D03C
:10CCB00001210DF091F901219DF8050015F0B0F961
:10CCC0009DF80400FF280BD005210DF085F96020A8
:10CCD0001EF090FF044660B9314901201AF098FE19
:10CCE0009DF80630FF2BB7D02E4901201AF090FE98
:10CCF000B2E702462C49284621F069F820461FF089
:10CD00006EF9002680F8406004460CF0C7FE009BD8
:10CD10009DF80A2084F85860C4E914369DF808305C
:10CD200013449DF80920B24218BF0133C4E912012F
:10CD300084F8593001219DF804000CF0F5FC0446FC
:10CD400010B31EF0E1FE19490246284621F03FF8D3
:10CD5000012013F075FA06460028C1D02A46214664
:10CD600020F0A0FFF389A3F500739BB2F381F38950
:10CD700003F4F05313B930461FF0BCFA013C0C4BDE
:10CD80000C4A43F82420ABE79DF804200A4901200F
:10CD90001AF03EFEA4E700BF1A450500BC5C050082
:10CDA000106805006D68050036680500BC68050060
:10CDB0004CC100205D0204003E68050010B50C4621
:10CDC00014F0BAF9A0F10903DBB2052B04D821460F
:10CDD000BDE8104015F0DCBB02490120BDE8104061
:10CDE0001AF016BEE567050010B5044618B9002014
:10CDF00000F0010010BD1FF065F80028F7D12046B3
:10CE00001FF0CBF880F00100C0B2F1E770B5054625
:10CE10000E461FF09AF858B928461FF053F80446FA
:10CE200030B92A460E4903201AF0F2FD204670BDA3
:10CE300030461FF08AF818B10A4901201AF0E8FDBF
:10CE4000FFF7B8F804460028F0D028461FF07DF818
:10CE50000028EBD02A460449204620F097FFE5E75A
:10CE60009C610500CF610500AA39050070B5064632
:10CE70000D461FF01DF9044630B932461349032010
:10CE80001AF0C6FD204670BD1149002016F062F868
:10CE900032461049044620F079FF45B128461FF07C
:10CEA00007F968B93246094903201AF0B1FD00209C
:10CEB0001EF02AFE08490246204620F088FFE1E7DE
:10CEC0002A460649204620F061FFF0E72B6705005F
:10CED000B439050056670500CE4505005D670500BD
:10CEE00038B500220849054620F0AAFF044640B99B
:10CEF000064916F02FF8044904460246284620F059
:10CF000045FF204638BD00BFEDA405001E670500A3
:10CF10002DE9F3471F46012313600C690646894635
:10CF200015460CB10B68E45C30782E2800F0E380E5
:10CF30005B282CD101237B7296F801A0BAF15E0F19
:10CF400002D12B6801332B604FF000080CE03B4608
:10CF500001AA4946FFF7DCFF2B68019A48EA00085E
:10CF600013445FFA88F82B602B68F45CF018002CEF
:10CF700000F0C3805D2CEAD101332B6000237B726B
:10CF8000BAF15E0F14BF444688F001040BE05C2840
:10CF900066D102232B607078642808D1303C092CBC
:10CFA0008CBF00240124204602B0BDE8F08744284D
:10CFB00005D1303C092C94BF00240124F3E76628F6
:10CFC00064D06E2864D0722864D0732805D12046BE
:10CFD00002B0BDE8F04719F0EFBB532806D1204658
:10CFE00019F0EAFB80F00100C4B2DCE7742853D0EA
:10CFF000762853D077280DD1A4F13003092B7AD9A4
:10D00000204619F0CDFB002875D15F2C14BF0024F9
:10D010000124C8E757280CD1A4F13003092B66D9A5
:10D02000204619F0BDFB002861D15F3C18BF0124E8
:10D03000B9E7A0F13003DBB2092B31D978280FD141
:10D04000B3786BB1F3785BB104232B60B07819F03F
:10D0500046FB8046F07819F042FB40EA0810C0B267
:10D060007B7AFBB12B68F35C2D2B1BD17881286870
:10D07000013028603B4601AA49463044FFF748FF8B
:10D080002B68019A134404462B608CE70C20E7E7D9
:10D090000A20E5E70D20E3E70920E1E70B20DFE7C1
:10D0A0001846DDE73A7A62B1A4F14103192B98BF23
:10D0B0002034A0F1410398BFE4B2192B9CBF20306B
:10D0C000C0B2B7F90A30B3F5807F12D0DBB22AB113
:10D0D000A3F14102192A9CBF2033DBB24FF48072C6
:10D0E0009C427A8103D3844201D8984263E70024AA
:10D0F00059E784428AE7012455E7024901201AF0E2
:10D1000087FC50E74C69050082B02DE9F047B2B0CA
:10D110000C463AA9064681E80C0019F083F930B1B3
:10D120000025284632B0BDE8F04702B0704733789A
:10D130000BB17C2B5AD158223AA91CA826F0FAFA36
:10D14000DDE93A67DDF8F4801EF02FFDA268236860
:10D150001A440546D21B394630461FF09BFC00217D
:10D1600004460246284620F09DFD5CB1E389A3F504
:10D1700000739BB2E381E38903F4F05313B92046B3
:10D180001FF0B8F80DF1800A4FF00009C1450DDB22
:10D1900038461EF0B9FC91490246284620F017FE99
:10D1A00032468F49284620F0F1FDBAE75AF8041BB1
:10D1B000DAF820203046521A1FF06CFC09F1010900
:10D1C000044602464946284620F06CFD002CDDD07E
:10D1D000E389A3F500739BB2E381E38903F4F05381
:10D1E000002BD3D120461FF085F8CFE75E2B09D165
:10D1F0002368A268D34293D11BF036FB00288FD05E
:10D20000013607E0242B1DD1D4E900329A4206F101
:10D2100001060CD850223CA9684626F08BFA3AAB9E
:10D220000CCB21463046FFF76FFF054679E74C22CD
:10D230003DA9684626F07EFA3AAB0ECB304600F0A8
:10D24000D1F8F2E7282B0FD13D9B2168A2683AA8BC
:10D250000A44191D082B40F8212000EB83014A6382
:10D26000CADC01333D93C7E7292B0AD13D9B002B34
:10D27000C2DD3AAA02EB83032168A2680A441A635A
:10D28000BAE73AAB1BAA21463046FFF741FE1B9F87
:10D29000F35DA3F12A02012A804606EB070500F29E
:10D2A00084800137374450B92B2B08D14C223DA93B
:10D2B000684626F03FFA3AAB0ECB3846BFE7214628
:10D2C00014A814AD19F0AEFE0FCD0DF1700CACE842
:10D2D0000F0050222B68CCF800303CA9684626F09D
:10D2E00029FA3AAB0CCB1CA93846FFF70DFF0546CF
:10D2F0001F9850B1C389A3F500739BB2C381C38942
:10D3000003F4F0530BB91EF0F5FFD4E900239A4261
:10D31000BFF407AFB8F1000F3FF403AF204619F098
:10D3200007FC3AAB1BAA21463046FFF7F1FD214628
:10D33000804614A819F076FE0DF1500EBEE80F00DD
:10D340000DF1700CACE80F005022DEF80030CCF884
:10D3500000303CA9684626F0EDF93AAB0CCB1CA98D
:10D360003846FFF7D1FE81461F9850B1C389A3F517
:10D3700000739BB2C381C38903F4F0530BB91EF051
:10D38000B9FFB9F1000F0ED05DB1EB89A3F50073C1
:10D390009BB2EB81EB8903F4F05313B928461EF0DE
:10D3A000A9FF4D46B1E7A946FBE7D4E900239A421D
:10D3B0000BD250B1204619F0BBFB1BF055FA0028E8
:10D3C0003FF4AEAE1B9B1E4424E74C223DA96846A9
:10D3D00026F0B0F93AAB0ECB284630E7D845050029
:10D3E000C845050084B0F0B59BB021AE054686E87F
:10D3F0000E001BF039FA68B9044620461BB0BDE8A0
:10D40000F04004B070475C2C03D16C78002CF4D051
:10D410003D4601352C78002CEFD07C2C05F101071E
:10D42000F1D1DDE9211215A819F0FEFE502223A941
:10D43000684626F07FF996E80C0015A93846FFF7F4
:10D4400063FE044618980028D7D0C389A3F500735B
:10D450009BB2C381C38903F4F053002BCDD11EF0DE
:10D4600049FFCAE770B504461EF06FFD10B90024ED
:10D47000204670BD00222949204620F0E1FC0646E6
:10D480001EF063FD002837D000222549304620F0E9
:10D49000D7FC05461EF071FD08B35EB1F389A3F514
:10D4A00000739BB2F381F38903F4F05313B9304650
:10D4B0001EF020FF002D2ED02C681A4BE31A5C4280
:10D4C0005C41002DD4D0EB89A3F500739BB2EB81B6
:10D4D000EB8903F4F053002BCAD1284618E05DB164
:10D4E000EB89A3F500739BB2EB81EB8903F4F05356
:10D4F00013B928461EF0FEFE002EB8D0F389A3F51E
:10D5000000739BB2F381F48914F4F054AFD1304628
:10D510001EF0F0FEACE72C46D3E700BFAA390500A9
:10D52000316E05007D030300F7B5064608460D463B
:10D5300014461EF022FD30B92A46334903201AF062
:10D5400067FA03B0F0BD6CB300223049304620F0DA
:10D55000D1FB0090C0B120F017F9012300906A467A
:10D560000020294613F034FD00980028E9D0C38933
:10D57000A3F500739BB2C381C38903F4F053002B5E
:10D58000DFD11EF0B7FEDCE7214F002239463046DE
:10D5900020F056FC044638B92A463946304620F079
:10D5A000F5FBCEE71B4FF0E71EF0C7FC78B129462C
:10D5B000204620F0ADFAE389A3F500739BB2E38126
:10D5C000E38903F4F053002BBBD12046D9E70221B5
:10D5D0006846CDE9004520F052FB39460546024633
:10D5E000304620F0D3FB002DE5D0EB89A3F5007386
:10D5F0009BB2EB81EB8903F4F053002BDBD128467F
:10D600001EF078FED7E700BF6A5C05008E5C05005F
:10D61000605C0500655C050010B500220446FFF75C
:10D6200083FF2046BDE81040FFF75ABC38B51546C9
:10D6300001220446FFF778FF25B100222946204643
:10D64000FFF772FF2046BDE83840FFF749BC0000F5
:10D6500037B5054601910F4848F208011EF09BFAC4
:10D660000446A8B12A460C4920F090FB012301AAE8
:10D670002146284613F0ACFCE389A3F500739BB266
:10D68000E381E38903F4F05313B920461EF032FE20
:10D6900003B030BD67DB0200C23F05002DE9F04159
:10D6A0000F46904618490022064620F0C9FB20F09C
:10D6B0002DFF002205461549304620F0C1FB0446E7
:10D6C000F8B142463946013D20F0ECFA28461EF0FA
:10D6D0001BFA0D490246304620F079FB1DB9214660
:10D6E0003046FFF7B5FFE389A3F500739BB2E381F2
:10D6F000E38903F4F05323B92046BDE8F0411EF05E
:10D70000F9BDBDE8F08100BF13670500196705008A
:10D7100037B5054601910F4848F208011EF03BFA63
:10D720000446A8B12A460C4920F030FB012301AA87
:10D730002146284613F04CFCE389A3F500739BB205
:10D74000E381E38903F4F05313B920461EF0D2FDC0
:10D7500003B030BD61DB0200C23F050038B50022D6
:10D760000D460D49044620F06BFBA0B1C389A3F51B
:10D7700000739BB2C381C38903F4F0530BB91EF04D
:10D78000B9FD2046044920F093FF29462046BDE814
:10D790003840FFF7BDBF38BD196705002DE9F04FD0
:10D7A00085B005461EF0AFFC044640B92A464849FC
:10D7B00003201AF02DF9204605B0BDE8F08F454949
:10D7C000002015F0C7FB04460028F4D048F20801F9
:10D7D00041481EF0E0F906460028ECD022463F49B9
:10D7E000DFF8F8B020F0D2FA1EF0DFF929468246C1
:10D7F00003A819F01AF94FF0000847460398D8B962
:10D80000A7EB08001EF080F935490246204620F0BB
:10D81000DEFA52463349204620F0D9FAF389A3F5BF
:10D8200000739BB2F381F38903F4F053002BC2D150
:10D8300030461EF05FFDBEE71FF0A2FF0546FFF772
:10D8400011FE00283BD048F2600127481EF0A3F9E2
:10D85000814638461EF058F900210246019048469C
:10D8600020F088FD019B5BB1DA89A2F5007292B2CB
:10D87000DA81DA8902F4F05212B918461EF03AFD44
:10D8800022465946484620F081FA49463246284603
:10D89000FFF7CCFE49461FF097FE5DB1EB89A3F57B
:10D8A00000739BB2EB81EB8903F4F05313B9284664
:10D8B0001EF020FD03A8013719F0A2F89EE72A46C2
:10D8C0003946504620F0EEF908F10108E5E700BFBF
:10D8D000EE6605001E6705005DD70200C23F050029
:10D8E00013670500196705009DD602002DE9FF4169
:10D8F00006461046019114461EF01FFB07460028FD
:10D9000052D0214603A819F090F80024039810BBC8
:10D910004549304620F0CCFE4449304620F0C8FE50
:10D9200000224349304620F08BFA414905463046F3
:10D9300020F0BEFE18F074FB804600283ED0014661
:10D940002846FFF7E5FE2A46214640461FF010FE16
:10D9500004B0BDE8F0811FF013FF01AB0122314696
:10D96000054615F025FAEFB950B1C289A2F500724B
:10D9700092B2C281C38903F4F0530BB91EF0BAFC12
:10D980005DB1EB89A3F500739BB2EB81EB8903F4E6
:10D99000F05313B928461EF0ADFC03A819F030F877
:10D9A0000027B3E70446EBE7002CB1D0204601ABDB
:10D9B0000122314615F0FCF90446A9E74DB3204693
:10D9C000FFF750FD50B348F208011A481EF0E3F883
:10D9D00048F20801064618481EF0DDF80746A6B1D1
:10D9E00098B12A461549304620F0D0F92A46134905
:10D9F000384620F0CBF9012231462046FFF794FD4E
:10DA0000424639462046FFF78FFD394630461FF023
:10DA1000DBFD294620461FF0D7FD99E72146284621
:10DA2000FFF716FEF5E700BF605C0500655C0500CA
:10DA3000EDA4050051D6020011D70200C23F050037
:10DA4000414B2DE9F047B2F100080E464FF00002BD
:10DA50003E493F4F054608BF1F4620F0F1F90446F6
:10DA600068B1C389A3F500739BB2C381C38903F472
:10DA7000F053002B66D1BDE8F0471EF03BBC0120FF
:10DA80001EF03AF831490246284620F0A0F9224615
:10DA90003946284620F0D4F9044600284ED10246E3
:10DAA0002C49DFF8B090284620F0CAF90446CCB9DA
:10DAB000B8F1000F3BD032462749284620F066F9DE
:10DAC000002C3FD0224631462846FFF70FFFE3895E
:10DAD000A3F500739BB2E381E38903F4F0538BBB9E
:10DAE0002046C8E700223946204620F0A9F98246A0
:10DAF000024648B131462046FFF7F8FE214650461F
:10DB0000BDE8F0471FF060BD4946204620F098F977
:10DB1000E389A3F500739BB2E381E38903F4F05337
:10DB2000824613B920461EF0E5FB5446BFE7324655
:10DB30000A490120BDE8F04719F06ABFB8F1000FAB
:10DB4000C0D0B8E7BDE8F087655C0500975C0500CC
:10DB5000605C0500EDA405008E5C05009C5C050082
:10DB60000022FFF76DBF0122FFF76ABF2DE9F74FD3
:10DB70000BF094FF894607461CF008FB83460BF028
:10DB80008DFF80468A46FEF715FA0446002800F00D
:10DB9000A580554B55495868002220F051F905469B
:10DBA000002800F09F801EF09FFDEB89A3F5007315
:10DBB0009BB2EB81EB8903F4F053064613B9284678
:10DBC0001EF098FB4A49002501235A1E12018818AD
:10DBD000B0F80EC01CF03F0F0DD0CDE900321EF0A2
:10DBE000F5F90135009B424928B1019A8A580F3254
:10DBF000120913441544013340F6CA029342E4D992
:10DC0000B018AB1B401B00931DF07EFF3949024644
:10DC1000204620F0DCF8009B18461DF075FF3649C1
:10DC20000246204620F0D3F840F6CA001DF06CFFF3
:10DC300032490246204620F0CAF830461DF064FF03
:10DC40002A490246204620F0C2F858461DF05CFFE3
:10DC50002B490246204620F0BAF8B8EB07006AEBE1
:10DC6000090125F025F80022264B25F04FF8264B18
:10DC7000002225F04BF841EC100B1DF033FF234937
:10DC80000246204620F0A3F821481DF03DFF21491F
:10DC90000246204620F09BF800201DF035FF1E496B
:10DCA0000246204620F093F81C481DF02DFF1C4929
:10DCB0000246204620F08BF84FF4D8201DF024FFB8
:10DCC00018490246204620F082F84FF400201DF04B
:10DCD0001BFF15490246204620F079F8204603B084
:10DCE000BDE8F08F06466DE7582D002080660500E0
:10DCF000742D0020886605008D660500936605007A
:10DD00009966050000408F400000B03E9C6605000B
:10DD1000F0CD0020A3660500B3660500ECB5050054
:10DD2000BF660500D0660500E166050010B5FEF788
:10DD300041F9044629481FF0E1FA294902462046E4
:10DD400020F045F827481FF0D9FA27490246204617
:10DD500020F03DF825481FF0D1FA2549024620461B
:10DD600020F035F84FF400201DF0CEFE2149024688
:10DD7000204620F02CF84FF480301DF0C5FE1E49DF
:10DD80000246204620F023F804F03CFD1B490246E1
:10DD9000204620F01CF81A4B1B78093BDBB20A2BFB
:10DDA00096BF184A184852F823001FF0A7FA1749DF
:10DDB0000246204620F00BF815481FF09FFA15493F
:10DDC0000246204620F003F813481DF09DFE13493B
:10DDD000024620461FF0FBFF204610BD08660500E6
:10DDE0001066050018660500206605002B66050014
:10DDF000356605003B660500C076050041660500F6
:10DE0000B82C0020345C050005A705004866050015
:10DE10005066050072660500BC2C00207A6605007D
:10DE200038B508490546002015F094F8044638B185
:10DE300028461DF0BDFE0449024620461FF0C7FFDC
:10DE4000204638BDAA640500AF46050010B513F0A2
:10DE500010FA044613F07CFA20B12046BDE81040C9
:10DE60001DF0A6BE10BD2DE9F74F0D460321044657
:10DE7000CDE900230CF0B0F84FF0000B4FF0010A91
:10DE80004FF08008D94615F1FF3502D203B0BDE846
:10DE9000F08F009B0AEA0306019B0BEA030756EA90
:10DEA000070316D088F31188002120460BF058FD97
:10DEB0000A200BF073F9012120460BF051FD89F384
:10DEC000118837200BF06AF91AEB0A0A4BEB0B0B9F
:10DED000D9E788F31188002120460BF041FD41204D
:10DEE0000BF05CF9012120460BF03AFD89F3118813
:10DEF0000520E7E710B40C780246002320460821ED
:10DF00005DF8044BFFF7AFBF2DE9F8430D46032141
:10DF100007460CF061F8002401264FF08008A14666
:10DF200015F1FF3502D22046BDE8F88388F3118849
:10DF3000002138460BF014FD03200BF02FF90121CE
:10DF400038460BF00DFD0A200BF028F938460BF08F
:10DF5000F3FC00B1344389F3118835200BF01EF92E
:10DF60007600DDE710B5032104460CF035F80021FA
:10DF700020460BF0F5FC4FF4FA700BF00FF901217D
:10DF800020460BF0EDFC50200BF008F920460BF07A
:10DF9000D3FC04464FF4D2700BF000F984F001007A
:10DFA000C0B210BD08B5002203491FF049FFBDE80B
:10DFB000084013F0B9B900BFAF4605002DE9F04F96
:10DFC0008BB00C46FFF7EEFF064613F0C1F928B9F7
:10DFD0004FF0000840460BB0BDE8F08F1DF0E5FDA6
:10DFE00080460028F4D0631EFF2B28BFF024224671
:10DFF000E317CDE900234FF000093046FFF7B2FFE9
:10E000000028E7D0DDE9002308213046FFF72BFF89
:10E0100001240025AA46274601213046FFF774FF58
:10E0200001215FFA80FB3046FFF76EFFBBF1010F65
:10E03000C0B22BD101283AD1402FCBDD9DF80C3056
:10E04000002BC7D005AC0DF10C090025A34619F82B
:10E05000017B380918F0F8F9207007F00F0018F06C
:10E06000F3F90135082D607004F10204EFD10023AB
:10E0700058468DF824301FF041F9014640461FF004
:10E08000B9FDD146BAF1000FA4D0B6E70AAB2B44D4
:10E09000834513F81C3C2DD14F4524DA1C4214BF94
:10E0A0004FF0010B4FF0000BBBF1000F21D00AAB7A
:10E0B0002B444FF0010B13F81C3C23430AAA2A44BB
:10E0C000012102F81C3C30465A4600236400FFF749
:10E0D000CAFE14F0FF0404BF01350124072D07F127
:10E0E000010799DDA8E70CBF4FF0010B4FF0000BC3
:10E0F000DAE7BA4623EA0403E0E770B58AB00C46D3
:10E10000FFF750FF064613F023F968B320461DF0D1
:10E1100044FF18B320461FF063FB0146054601206B
:10E120001BF051FF044650B10146002268461BF027
:10E130003FFA15F1FF3505D2684618F0D7FB2046A7
:10E140000AB070BD08213046FFF7DEFEC1B2684656
:10E1500018F0D3FE684618F031FDEAE70821304692
:10E16000FFF7D2FE1DF0D0FC0446E8E737B50D46B8
:10E170001446FFF717FF8DF8070013F0E9F880B198
:10E180000DF107020C4928461BF0C6FA9DF807005E
:10E190004CB101210BF0E4FB01219DF807000BF0CD
:10E1A0001BFF03B030BD04210BF016FF01219DF8C9
:10E1B00007000BF0D5FBF4E7F5DE020010B5FFF722
:10E1C000F1FE044613F0C4F838B12046CC220023F7
:10E1D0000821BDE81040FFF746BE10BD2DE9F0470D
:10E1E00086B00C46FFF7DEFE074613F0B1F840B1EB
:10E1F00020461DF05DFF38B922463049032019F052
:10E2000007FC06B0BDE8F08720461EF04BFD102845
:10E21000F2D13846FFF7A6FE2146002201A819F0E8
:10E2200003F80024A146A046A246059B0BB1019A23
:10E230009B5C8DF8003001A818F07AFC059B0BB1AF
:10E24000019A9B5C8DF8013001A818F071FC002345
:10E250001A46102168468DF802A018F0B8FAA4F109
:10E260002002C4F12003A14000FA02F220FA03F3D5
:10E270001143A0401943083440EA090641EA080561
:10E28000402CB146A846D0D1049850B1C389A3F51B
:10E2900000739BB2C381C38903F4F0530BB91EF022
:10E2A00029F83846552200230821FFF7DCFD3246C5
:10E2B0002B4640213846FFF7D6FDA2E7B2640500A1
:10E2C00010B5FFF76FFE044613F042F820B1204668
:10E2D000BDE81040FFF746BE10BD73B51DF065FCEC
:10E2E0000646A8B1FEF704FB054688B1014601A821
:10E2F00018F09BFB019C74B9EB89A3F500739BB2EA
:10E30000EB81EB8903F4F05313B928461DF0F2FFBB
:10E31000304602B070BDE38903F500739BB2002262
:10E32000E381114620461FF099FF014630461FF059
:10E3300061FCE389A3F500739BB2E381E38903F4F5
:10E34000F05313B920461DF0D5FF01A818F058FB73
:10E35000D0E710B101211FF0B1BD70472DE9F7439F
:10E3600005460F4690461DF008FE044640B92A4671
:10E370006E49032019F04CFB204603B0BDE8F08342
:10E3800028461DF0A7FD002835D0A98828681DF073
:10E3900002FC04460028EFD02946684618F045FBE9
:10E3A000009E002E37D0F38903F500739BB2F381F2
:10E3B00030461FF0E5F9814630461DF0CDFE20B312
:10E3C000B9F1000F33D0012130461FF077FD05462B
:10E3D00078B1014620461FF0EDFAEB89A3F50073F2
:10E3E0009BB2EB81EB8903F4F05313B928461DF07F
:10E3F00081FF01250AE028461DF0B6FD002814BF64
:10E40000082007201DF018FBC3E7054649463046A3
:10E410001FF0DAF86DB9B8F1000F0ED1009D002D94
:10E4200057D13A46424920461FF0B0FCA4E74D467A
:10E43000ECE7684618F0E4FAB2E7414601A818F0A4
:10E44000F4FA01980028E9D01FF09AF9009D0646D9
:10E45000A5B1EB8903F500739BB2EB8128461DF053
:10E460007BFE88B9EB89A3F500739BB2EB81EB8946
:10E4700003F4F05313B928461DF03CFF3246002147
:10E4800020461FF077FF13E00122002128461FF0ED
:10E49000E5FE314680461EF09DFF414620461FF0B6
:10E4A00089FA284641461FF08FF8684618F0A8FA06
:10E4B0005EB1F389A3F500739BB2F381F38903F492
:10E4C000F05313B930461DF015FF01A818F098FA63
:10E4D000B7E7EB8903F500739BB20122EB8111468C
:10E4E00028461FF0BBFE064678B1014620461FF0C5
:10E4F00061FAF389A3F500739BB2F381F38903F406
:10E50000F05313B930461DF0F5FEEB89A3F5007307
:10E510009BB2EB81EB8903F4F05313B928461DF04D
:10E52000E9FE684618F06CFA78E700BF0D5E05005A
:10E53000C23F05002DE9F04F8FB0814602AF104673
:10E540008A4616461DF0DFFD044600285ED03046A0
:10E550001EF0DCFB4028834680460AD9024630493B
:10E56000012019F055FA002420463437BD46BDE895
:10E57000F08F8300DA1D22F00702ADEB020D02AD31
:10E580002A462B440021934219D101223146381DDD
:10E590001BF051F8381D18F0F8F998B9381D18F02B
:10E5A000B5F900231946CDE90085524648461AF0D0
:10E5B000C7FA2946044640461EF088FFD4E742F8D1
:10E5C000041BE0E7381D18F06EF904461DF057FEF5
:10E5D00058B120461FF004F9061E06DBB34504DDE2
:10E5E000381D18F0D4FD45F826005CB1E389A3F589
:10E5F00000739BB2E381E38903F4F05313B920461F
:10E600001DF078FE381D18F0F3FAC3E72EB132463C
:10E610000449012019F0FCF9A6E7B0463546C0E7E9
:10E620008A5D0500D25D050010B5FEF761F904466C
:10E6300078B120F061F8E389A3F500739BB2E38120
:10E64000E38903F4F05323B92046BDE810401DF0E0
:10E6500051BE10BD2DE9F347044608460D461DF096
:10E660008CFC30B95649032019F0D2F902B0BDE84C
:10E67000F08720461DF02EFC064628461DF02AFC99
:10E68000864208D028461DF025FCE389002855D095
:10E6900043F04003E38120461DF066FC0646284611
:10E6A0001DF062FC86420BD028461DF05DFCE3891C
:10E6B0009BB223F03F03002845D043F00803E381D9
:10E6C00000224049DFF8FC90DFF8FCA020461FF054
:10E6D00011FB00223C49074620461FF00BFB064673
:10E6E000204620F009F8294601A818F09EF9019D5E
:10E6F00065BB7FB1394620461FF05CF9FB89A3F565
:10E7000000739BB2FB81FB8903F4F05313B93846C5
:10E710001DF0F0FD002EA9D0314620461FF04AF929
:10E72000F389A3F500739BB2F381F38903F4F053EB
:10E73000002B9BD130461DF0DDFD97E723F0400311
:10E740001B041B0CA6E743F00703B8E7EB8903F5AE
:10E7500000739BB201A8EB8118F052F94946284694
:10E760001EF07CF8E8B9514628461EF077F8C0B98B
:10E77000012128461FF0A2FB804690B101462046A9
:10E780001FF018F9B8F80E30A3F500739BB2A8F883
:10E790000E30B8F80E3003F4F05313B940461DF0B4
:10E7A000A9FDEB89A3F500739BB2EB81EB8903F420
:10E7B000F053002B9BD128461DF09CFD97E700BF2E
:10E7C000445E0500825E050031A1050070B5064675
:10E7D0001DF06EFC28B91B490120BDE8704019F0FE
:10E7E00017B9FEF785F8054650B3002231461FF0F1
:10E7F0009BFC044690B932461349012019F008F9F0
:10E80000EB89A3F500739BB2EB81EB8903F4F05322
:10E81000B3B92846BDE870401DF06CBD01462846DE
:10E820001FF088FEE389A3F500739BB2E381E389BF
:10E8300003F4F053002BE3D120461DF05BFDDFE72E
:10E8400070BD00BF406105006E6105002DE9F74312
:10E8500005460F4691461DF031FD30B9464903206B
:10E8600019F0D6F803B0BDE8F08338461DF020FC5F
:10E8700008B94249F3E748461DF07FFB28B94846EE
:10E880001DF016FC08B93E49E9E739463D481EF03F
:10E8900011F904460028E5D00146012228461FF060
:10E8A00043FCE389A3F500739BB2E381E38903F49E
:10E8B000F053064613B920461DF01CFD30461EF0ED
:10E8C0005FFF8046002830D1494630461EF082FD69
:10E8D000314640461EF078FE2B4938461DF0BEFFFB
:10E8E0000028BFD00022294928461FF0A9FA01902C
:10E8F0001DF0DEFB48B126492846012301AA12F08B
:10E90000B5FB224928461FF0D3FE01980028A9D064
:10E91000C389A3F500739BB2C381C38903F4F05389
:10E92000002B9FD11DF0E6FC9CE71DF006FB20B1FB
:10E93000494640461FF0ECF8CAE71DF036F941465B
:10E9400004461FF0E5F8494620461FF0E1F821464D
:10E9500030461EF03FFD002CBAD0E389A3F50073CA
:10E960009BB2E381E38903F4F053002BB0D120463E
:10E970001DF0C0FCACE700BF156305004C6305004B
:10E9800083630500DB630500DB380500F73905000C
:10E99000BB390500F8B50646084614461F461EF06A
:10E9A000ADFC3946054620461DF0F5F829460446DB
:10E9B00002463046FFF74AFF29462046BDE8F840A8
:10E9C0001EF002BEF0B585B006460D461DF076FC81
:10E9D00020B93049032019F01BF82CE028461DF01F
:10E9E00067FB50B329462C481EF064F8054610B367
:10E9F0000146012230461FF097FBEB89A3F5007317
:10EA00009BB2EB81EB8903F4F053044613B928461B
:10EA10001DF070FC7CB1214630461FF08BFDE38970
:10EA2000A3F500739BB2E381E38903F4F05313B9B8
:10EA300020461DF05FFC05B0F0BD4DBB314603A87C
:10EA400017F0F3FF154F039C002CF4D0E38903F576
:10EA500000739BB2E38103A817F0D2FF0095002357
:10EA60000122394620461DF06BFE18B12146304682
:10EA70001FF060FDE389A3F500739BB2E381E38996
:10EA800003F4F053002BDED120461DF033FCDAE70F
:10EA900003499FE715630500DB630500E16305009B
:10EAA000E563050038B5054608461EF027FC044618
:10EAB00088B101462846FFF785FFE389A3F5007377
:10EAC0009BB2E381E38903F4F05323B92046BDE808
:10EAD00038401DF00FBC38BDF8B507460C46164649
:10EAE0001DF0ECFB28B935490320BDE8F84018F0CB
:10EAF0008FBF20461DF0DCFA00285CD0214630484C
:10EB00001DF0D8FF0546002857D00146012238469F
:10EB10001FF00AFBEB89A3F500739BB2EB81EB8935
:10EB200003F4F053044613B928461DF0E3FB2046D6
:10EB30001EF026FE054688B186421ED12146384683
:10EB40001FF0F8FCEB89A3F500739BB2EB81EB8916
:10EB500003F4F05313B928461DF0CCFB6CB3E389E2
:10EB6000A3F500739BB2E381E38903F4F05323BB65
:10EB70002046BDE8F8401DF0BDBB1DF0DEF90028C1
:10EB8000E0D03146012228461EF00BFF0646002841
:10EB9000D8D0014628461FF0CDFCF389A3F50073B9
:10EBA0009BB2F381F38903F4F053002BCAD13046B2
:10EBB0001DF0A0FBC6E7034996E7F8BD1563050005
:10EBC000DB6305003A6405002DE9F04387B000AF30
:10EBD00081460C461546E8461DF070FB40B93549A4
:10EBE000032018F015FF1C37C546BD46BDE8F0836D
:10EBF00020461DF05DFA08B92F49F1E721462F485C
:10EC00001DF058FF06460028EDD02946381D17F0A4
:10EC10000CFF0024786830B1042C3FD122462849EB
:10EC2000032018F0F5FE786850B1C389A3F500738E
:10EC30009BB2C381C38903F4F0530BB91DF05AFB97
:10EC40000022314648461FF06FFA1EF09DFDF38901
:10EC5000A3F500739BB2F381F38903F4F0530546E7
:10EC600013B930461DF046FB95B1234607F1080263
:10EC70002946484612F0ACF9EB89A3F500739BB224
:10EC8000EB81EB8903F4F05313B928461DF032FBF6
:10EC900007F1080120461EF019FCA4E71EF070FDE4
:10ECA00007F1080343F82400381D17F0A9FE0134CA
:10ECB000B0E700BF15630500A2620500DB63050035
:10ECC000DB620500F7B5014601A817F0AEFE254F3F
:10ECD0000026019820B31EF053FD044600283CD0C6
:10ECE0001DF0F0F80546002839D120461DF02DF919
:10ECF00030BB22463946032018F08AFE0125E389FD
:10ED0000A3F500739BB2E381E38903F4F05313B9D5
:10ED100020461DF0EFFA01A817F072FE002DD8D0A2
:10ED2000019850B1C389A3F500739BB2C381C38915
:10ED300003F4F0530BB91DF0DDFA304603B0F0BD1B
:10ED400036B9E38903F500739BB2E3812646D6E723
:10ED5000214630461FF045FAD1E70546DBE700259E
:10ED6000CDE700BF8261050070B505460E461DF077
:10ED700004F910B301221649284619F045F8044653
:10ED80001DF04BF8F8B922461249032018F040FE56
:10ED90005CB1E389A3F500739BB2E381E38903F4DB
:10EDA000F05313B920461DF0A5FA25B1EB8903F500
:10EDB00000739BB2EB81284670BD28461DF0C5F854
:10EDC0000028D7D1DBE7314620461EF003FBDFE702
:10EDD000AA3905007D6405002DE9F84304460F4675
:10EDE00016461DF0B2F8054640B9284922460120D2
:10EDF00018F00EFE2C462046BDE8F88330461DF084
:10EE0000A4F8054610B932462149F0E7384620F00B
:10EE1000CFF800221F49814630461FF011F800222A
:10EE200007461D4930461FF00BF88046AFB9A0B920
:10EE300000221A4930461FF003F805462A46494683
:10EE400020461FF0ADF9294648461EF0BDFBE38978
:10EE500003F500739BB2E381CDE706201CF0ECFDC7
:10EE6000054660B11FB13A460A491EF08FFFB8F15E
:10EE7000000F04D04246084928461EF087FF41464D
:10EE800038461EF0A1FB002DD8D1D1E74A6205001B
:10EE900073620500139B0500E36A0500C245050087
:10EEA00073B504460D461DF050F8064640B91949A1
:10EEB0002246012018F0ACFD3446204602B070BD59
:10EEC00028461DF042F8064610B92A461249F0E7D6
:10EED000294601A817F0A9FD019D2DB9E38903F585
:10EEE00000739BB2E381E8E7EB8903F500739BB203
:10EEF000EB8128461EF044FC294606460246204681
:10EF0000FFF76AFF324629461EF032FB01A817F0D0
:10EF100077FDE1E7F56105001F620500F0B50646E3
:10EF200089B0084620F044F8054630461DF0C6F981
:10EF3000044600B30022294630461FF0F5F8D0B150
:10EF4000C389A3F500739BB2C381C38903F4F05353
:10EF50000BB91DF0CFF95DB1EB89A3F500739BB23E
:10EF6000EB81EB8903F4F05313B928461DF0C2F985
:10EF7000204609B0F0BD30461CF0E7FF044608B15A
:10EF80000024E8E730460EF071FC07460028F7D071
:10EF90002022694628461FF051FD6A463146384610
:10EFA0000EF04EFD0028D6D0C389A3F500739BB2A6
:10EFB000C381C38903F4F0530BB91DF09BF90124FD
:10EFC000C9E70000F8B507460C46FFF7A7FF10B9E0
:10EFD00000252846F8BD20461FF0EAFF0122014621
:10EFE0000546384618F07EFE04465DB1EB89A3F570
:10EFF00000739BB2EB81EB8903F4F05313B92846FD
:10F000001DF078F9002CE3D0FCF7D4FF054668B971
:10F01000E389A3F500739BB2E381E38903F4F05322
:10F02000002BD5D120461DF065F9D2E720461CF013
:10F0300024FF064638461BF095F8074601201CF0D1
:10F040005BFD2D49024628461EF0C1FE002F4BD025
:10F050002046B84780F00100C0B200F001001CF06B
:10F060004BFD2649024628461EF0B1FE86F00100FF
:10F07000C0B21CF041FD2249024628461EF0A7FE00
:10F0800020461FF0BFF906461CF0A8FE70B3002210
:10F090001C4930461EF0D4FE1A49024628461EF08E
:10F0A00096FE0022184930461EF0CAFE1649024656
:10F0B00028461EF08CFE5EB1F389A3F500739BB267
:10F0C000F381F38903F4F05313B930461DF012F9BC
:10F0D000E389A3F500739BB2E381E38903F4F05362
:10F0E000002B7FF476AF9DE70120B6E720461EF0A7
:10F0F00047FB06490246DBE7F4620500FD620500B6
:10F1000008630500139B0500E36A0500C24505007E
:10F1100010B5142994B0A8BF14210C461FF022FD8D
:10F1200024EAE4740A2351EC100B009302AA46234C
:10F13000019417F091F902A81EF0E0F814B010BD88
:10F1400030B5044695B008460D461DF070F848B33A
:10F1500020461CF022FF28B328461EF041FB831EE8
:10F16000222B05461ED820461DF061F860B12046CE
:10F170001EF036FB2B46012202A917F08FFA02A8D7
:10F180001EF0BCF815B030BD20461FF0EBFC4FF070
:10F19000FF33CDE9005302AA462351EC100B17F0C0
:10F1A0005BF9ECE720461FF073FBEBE710B5044674
:10F1B0001CF0C3FE40B12CB900242046BDE810402D
:10F1C0001CF0A2BC2468F8E720461CF09AFE08B1A7
:10F1D0006488F2E720461CF06BFF20B120461DF04A
:10F1E00061FD0446E9E720461CF0C7FE90B12046C9
:10F1F0001EF014FD0028DFD0C3890468A3F5007356
:10F200009BB2C381C38903F4F053002BD5D11DF009
:10F2100071F8D2E710BD7FB503901CF096FE40B1A7
:10F22000039CE38903F500739BB2E381204604B09D
:10F2300070BD03981CF081FE0028F1D103981CF0EA
:10F240009CFE04460028EBD103980EF043F818B951
:10F25000FCF7B0FE0446E9E717F078F80546002809
:10F26000F6D01EF08DFA03AB0193012300932246E2
:10F2700023462946064619F063FC314604462846D3
:10F280001EF0A2F9D2E7000070B508B1036823B9F7
:10F290000020BDE870401CF037BC00211EF098FA39
:10F2A00004461CF04AFE002846D00CB1236843B93E
:10F2B00000201CF029FC054634B9002D3DD028461D
:10F2C00070BD012B0ED00025E389A3F500739BB21E
:10F2D000E381E38903F4F053002BEED120461DF0C7
:10F2E00009F8EAE7002120461EF072FA06461CF0F3
:10F2F000DFFEB8B130461CF0F8FE98B100201CF0DB
:10F3000003FC0546002EDFD0F389A3F500739BB202
:10F31000F381F38903F4F053002BD5D130461CF070
:10F32000E9FFD1E730461CF025FF18B930461FF041
:10F33000A7FCE6E70025E5E72CB99FED0F0BBDE83C
:10F3400070401CF0CFBB20461CF0FFFD0546002896
:10F35000B9D120461CF0ACFE40B120461CF0C5FEE1
:10F3600020B128461CF0D0FB0546ADE720461FF033
:10F3700087FCF9E7AFF30080000000000000F87F91
:10F3800038B511F076FF054611F0E2FF044650B1A2
:10F3900028460AF077FA80F01000C0F300142146E6
:10F3A000284612F03DFE204638BD000010B5044648
:10F3B00011F0CEFF28B90B49012018F029FB0020DD
:10F3C00010BD20460AF05EFA00F00F000138C0B20E
:10F3D0000828F4D8044BBDE8104053F820001DF075
:10F3E0008DBF00BFA7460500105C050008B511F0F1
:10F3F00040FFBDE80840FFF7D9BF00001FB50C462D
:10F400008DED000B11F035FF9DED000B8DF80F0019
:10F41000002251EC100B0A4B23F078FC0022094B20
:10F4200023F074FC0022064B23F09AFD23F0CEFF5C
:10F4300023460DF10F02F1F7ADFD04B010BD00BF82
:10F4400000408F400000304108B511F012FFBDE8C8
:10F45000084013F091BC0000F0B585B006461CF0E2
:10F460006CFD074640B3314603A817F0DEFA0024CE
:10F470002646039828B9002E08BF0024204605B070
:10F48000F0BD1EF07DF9054611F0F3FE13F074FC9B
:10F49000640004435DB1EB89A3F500739BB2EB817B
:10F4A000EB8903F4F05313B928461CF023FF03A89B
:10F4B00017F0A6FA0136DCE730461CF046FD48B3EB
:10F4C0003A461849304618F09FFC05461CF055FD99
:10F4D0000446D0B13B4632463946CDE9007728464E
:10F4E00019F02EFB1FF012F80446002DC6D0EB8950
:10F4F000A3F500739BB2EB81EB8903F4F053002B6F
:10F50000BCD128461CF0F6FEB8E70749012018F0E8
:10F510007FFAEAE7304611F0ACFE13F02DFC04460A
:10F52000ACE700BF3B6005004060050070B50646D3
:10F530000D461CF0BDFD28B91F490120BDE87040F3
:10F5400018F066BA28461CF0B3FD20B928461CF016
:10F5500014FD0028F0D0FDF7CBF9044650B328463F
:10F5600016F0D2F8054690B932461449012018F039
:10F570004FFAE389A3F500739BB2E381E38903F4B7
:10F58000F053BBB92046BDE870401CF0B3BE024644
:10F59000314620461EF004FEEB89A3F500739BB2B2
:10F5A000EB81EB8903F4F053002BE2D128461CF0E9
:10F5B000A1FEDEE770BD00BFEF6005001F61050022
:10F5C00070B5A0B005461CF073FD044628B9474944
:10F5D0002A46032018F01CFA0BE0802269462846D0
:10F5E0001FF02CFA7F2807D94149032018F010FAA0
:10F5F0000024204620B070BDFDF77AF905460028AA
:10F60000F6D0002269461EF075FB1EF0BDF8EB89AE
:10F61000A3F500739BB2EB81EB8903F4F05304462E
:10F6200013B928461CF066FE002CE2D13149684629
:10F6300024F0A8F800284BD02F49684624F0A2F8FF
:10F6400000284DD02D49684624F09CF8002849D068
:10F650002B49684624F096F8002845D0684624F0E7
:10F66000A3F8082803D96A4626490120B2E768466C
:10F670001FF039FF1FF02CFE05460028F3D016F0CE
:10F6800043F8EB89A3F500739BB2EB81EB8903F49C
:10F69000F053064613B928461CF02CFE002EE2D08B
:10F6A0003446FDF725F905460028A2D022466946D2
:10F6B0001EF06CFBEB89A3F500739BB2EB81EB8929
:10F6C00003F4F053002B94D128461CF013FE90E76E
:10F6D0000D4800211CF05FFA0028BFD00446E0E787
:10F6E0000A48F6E70A48F4E70A48F2E763670500C4
:10F6F00093670500B8670500BE670500C66705008B
:10F7000069660500D1670500558003003D80030050
:10F71000398003001D800300F8B5154604460F46E6
:10F72000084A194628461E4617F07CFFA40A14F121
:10F73000FF3400D2F8BD3A463146284617F072FF32
:10F74000F5E700BF04A705002DE9F041834E3068BE
:10F75000B0F90240822C8AB0354661D022DC5B2CA5
:10F760006DD00CDC2D2C41D002A9204620221FF0A8
:10F770008FFF02AA7A49022018F04AF93DE07B2C5B
:10F7800000F0A580812CEFD11FF076FF17F086F8EE
:10F7900004460D46306820F01DF9204629461CF02D
:10F7A00013FA1AE0B42C13D008DC832CDCD11FF040
:10F7B0004DFF0446306820F00DF90FE0B52C11D054
:10F7C000B62CD1D120F006F902201CF035F904E066
:10F7D00020F000F901201CF08FF9044620460AB001
:10F7E000BDE8F08120F0F6F80020F4E720F0F2F810
:10F7F00030684388813B012B01D90024EEE7FFF7F5
:10F80000A3FF054600201CF07FF922462946064644
:10F810001AF002F93146044628461DF0D5FEDDE710
:10F820001FF02AFF0021F0F7BFFECDE9000130688C
:10F8300020F0D0F89DED000B1CF054F9CDE71CF042
:10F84000B4F904460028D8D03068464F20F0C2F8FA
:10F850002868B0F902305D2B03D03B8A03F07003B7
:10F860008BB15D2020F032FE0028B7D1E389A3F5EB
:10F8700000739BB2E381E38913F4F055BDD12046B8
:10F880001CF038FDB9E7FFF75FFF064640B12B6873
:10F89000B3F902305D2B08D02C2020F017FE20B9E0
:10F8A000214630461DF090FEA7E7314620461EF067
:10F8B0002FF9F389A3F500739BB2F381F38903F465
:10F8C000F053002BC4D130461CF014FDC0E7FCF708
:10F8D00071FB0446002890D03068DFF8888020F063
:10F8E00079F82868B0F90230832B04D1B8F81030C9
:10F8F00003F070030BB17D20B4E71FF0A7FE1FF0EB
:10F90000F8FB0746286820F065F83A2020F0DEFD75
:10F9100030B900262246314638461DF029FE6CE7F4
:10F920002868FFF711FF06460028F2D02B68B3F9CC
:10F9300002307D2B04D02C2020F0C8FD0028E9D017
:10F94000314638461DF068FB014620461EF032F86D
:10F95000394630461DF038FEC3E700BF18BA002014
:10F96000CF600500582D002070B5A0B01EF090FFAC
:10F970000E4D04462E68C5F800D020F02BFE5CB179
:10F98000E389A3F500739BB2E381E38903F4F053A9
:10F9900013B920461CF0AEFCFFF7D6FE04461FF05C
:10F9A000D9FF20462E6020B070BD00BF18BA0020DD
:10F9B00038B51FF089FD1FF08BFC044680B1FFF7BE
:10F9C000D3FFE389A3F500739BB2E381E38903F4DA
:10F9D000F053054613B920461CF08CFC284638BD70
:10F9E0000546FBE72DE9F74310B10368002B37D13B
:10F9F000514B524C1B88524F013B1D012E19314671
:10FA0000F38903F500739BB2F38101A817F00DF899
:10FA1000019880B930461EF06FFE6319DA89A2F5AD
:10FA2000007292B2DA81DB8903F4F0530BBB3046EB
:10FA30001CF060FC1DE01DF0A3FE0022394681464B
:10FA40001EF0FEF9804611F014FC002109F06CFE56
:10FA5000404649461DF0B8FD01A816F0D1FFD7E792
:10FA600000211DF0B5FE064630B93649012017F0D9
:10FA7000CFFF03B0BDE8F083DFF8BC902F4DB9F89D
:10FA80000040013C05EB04140146E38903F50073D3
:10FA90009BB2E381002220461EF046FBE389A3F5DA
:10FAA00000739BB2E381E38903F4F053074613B973
:10FAB00020461CF01FFC002F38D038461DF060FE99
:10FAC00000221F4904461EF0BBF911F02DFC8046B0
:10FAD0005CB1E389A3F500739BB2E381E38903F48E
:10FAE000F05313B920461CF005FCB9F80040013C66
:10FAF00005EB04143946E38903F500739BB2E381F7
:10FB000020461EF017FD214638461DF05DFD40469B
:10FB100011F0C6FB014610B9404609F005FEF38915
:10FB2000A3F500739BB2F381F3897DE73246064962
:10FB3000012017F06DFFF2E76CC10020742D00204A
:10FB4000AF460500D35E0500105F05002DE9F74FB5
:10FB5000824608468846154611F0FAFB30B9A2489D
:10FB600017F014FE002003B0BDE8F08F404611F0FE
:10FB700097FB08F0EF030D2B28461DBF002400263D
:10FB80000027012404BF0026984F1CF0DEF98346AD
:10FB9000002800F086800022954928461EF050F982
:10FBA000814610B11EF019FE814600229149284677
:10FBB0001EF046F9002800F010811FF045F80246BB
:10FBC0000B4606460F4623F03BFB30B900220023CC
:10FBD0003046394623F00CFB08B1002600270022EE
:10FBE000854928461EF02CF98346D8B11CF0D5F97A
:10FBF00000B358461DF0F4FD002800F3E98014BF5F
:10FC00004FF0FF340024BBF80E30A3F500739BB215
:10FC1000ABF80E30BBF80E3003F4F05313B958466E
:10FC20001CF068FB631C022B20D97449032017F0D9
:10FC3000EFFE97E758461CF03BFA08B9704CE2E734
:10FC4000704958461CF00AFE002840F0C1806E49F9
:10FC500058461CF003FE0446002840F0BB806B4968
:10FC600058461CF0FBFD0028CDD1E7E7002268498B
:10FC700028461EF0E5F81EF0B0FD002265498346D7
:10FC800028461EF0DDF811F04FFB019050461CF0A5
:10FC900074F968B950461CF00BFA48B95E49012066
:10FCA000C5E728461EF04AFDFF2381460193EDE794
:10FCB000FCF780F9054600283AD040461BF078FF53
:10FCC0005649024628461EF082F8B9F1000F07D0C7
:10FCD00001201BF011FF5249024628461EF077F81A
:10FCE000002200233046394623F0A0FA90B10022CA
:10FCF0004C4B3046394623F009F800224A4B23F09A
:10FD00002FF923F063FB1BF0FFFE3A490246284619
:10FD10001EF05DF83CB120461BF0F6FE3649024667
:10FD200028461EF054F85246404928461EF02EF848
:10FD3000404611F0B5FA002845D10121404609F0AE
:10FD4000F3FC00283FD0441E0198394F11F000FB0E
:10FD5000064650BB47F82400BBF1000F08D05046C0
:10FD60001CF0B8F838B350461FF014F847F82400D8
:10FD7000304B1C88631E304C04EB03142946E38986
:10FD800003F500739BB2E3812046F0F795FF294607
:10FD9000461E20461DF018FC002EFFF6E3AE30464E
:10FDA00003B0BDE8F04F1BF0AFBE019B63F0FF0353
:10FDB00047F82430D0E726B12049012017F028FE6B
:10FDC000D6E71F49F9E7BBF1000FD1D01D49F4E791
:10FDD000012418E74FF0FF3415E732463B46304622
:10FDE000394623F02DFAF7E6A74605000000394012
:10FDF000D3460500215F05002A5F0500435F05002B
:10FE000018FCFFFF2F5F0500365F05003E5F050011
:10FE1000885F0500DB3805008C5F0500AF460500F4
:10FE2000AD5F05000000304100408F40B35F05002A
:10FE30004CC100206CC10020742D0020BC5F050067
:10FE4000DF5F050013600500F0B591B00023059356
:10FE5000FF23ADF810303C4B07930C23ADF8203056
:10FE600004AB0993394B0A930B23ADF82C300DF1F9
:10FE700011030C93364B0D9309230546164608468D
:10FE80000124ADF83830032206AB07A906940F937E
:10FE90001AF0B8F858B3069B2846002BD8BF069432
:10FEA0001CF04BF8002834D0294601A816F0BDFDFF
:10FEB0000198059BA0B9002402AF059BA34233DC47
:10FEC0009DF81040204611F043FA18B10121204658
:10FED0000AF082F83A461F49304619F01DFC06E048
:10FEE000072B06DD08221C49012017F091FD11B0F7
:10FEF000F0BD1DF045FC059C11F016FA10AB1C443A
:10FF0000059B04F8380C013301A8059316F078FD21
:10FF1000CEE7059C2846631C059311F0AAF910ABA7
:10FF20001C4404F8380CC6E73D5D284611F010FA71
:10FF300038B1284611F050F918B9012128460AF0C5
:10FF40004BF80134B9E700BFA9600500AD600500BA
:10FF5000D346050025C00200B460050070B5054613
:10FF60000C46164611F0F4F928B930490120BDE8D5
:10FF7000704017F04DBD20461CF09AF8002848D07C
:10FF80002B4920461CF06AFC98BB2A4920461CF0ED
:10FF900065FC80BB284920461CF060FC68BB2749F3
:10FFA00020461CF05BFC50BB254920461CF056FC4B
:10FFB00038BB244920461CF051FC20BB2249204676
:10FFC0001CF04CFC08BB214920461CF047FCF0B952
:10FFD0001F4920461CF042FCD8B1092486F00101DB
:10FFE000284611F0B5F821462846BDE8704009F0D2
:10FFF000F3BF0724F2E70424F0E70524EEE7062424
:020000023000CC
:10000000ECE70124EAE70224E8E70324E6E7082412
:10001000E4E70021284611F09BF834B10D49204651
:100020001CF01CFC08B90C49A0E770BDA7460500F0
:100030004D600500C845050054600500616005007D
:10004000846005008E600500706005008160050019
:100050008B600500473F05009860050010B50C4611
:1000600011F007F921460022BDE81040FFF776BFE6
:1000700070B5002286B00E461D491DF0E1FE044613
:100080001CF016F80546B0B10022214601A817F071
:10009000CBF80025DDE9013293421CD3049850B11E
:1000A000C389A3F500739BB2C381C38903F4F053E2
:1000B0000BB91CF01FF95CB1E389A3F500739BB287
:1000C000E381E38903F4F05313B920461CF012F9DD
:1000D000284606B070BD059800B1C05C864214BFCA
:1000E000284645F00100C5B201A816F021FDD1E770
:1000F0005D6705002DE9F047BAB08046084614AFA9
:100100001EF0C6FB00228349054640461DF098FEBE
:100110001EF0FCF900228049824640461DF090FE08
:1001200006461BF0C5FF044640B9314628461DF07F
:100130004BFA20469837BD46BDE8F08730461CF0A4
:10014000B1FD00F1080323F00703ADEB030D0DF142
:100150005009421C494630461EF070FC5EB1F389DE
:10016000A3F500739BB2F381F38903F4F05313B941
:1001700030461CF0BFF869214046FFF779FF4FF485
:100180008072002387F84800A7F84A202946524683
:1001900007F1180087F84930FB643D6417F044F814
:1001A00007F11801384616F03DFFBC46BCE80F00C9
:1001B00007F12C040FC45022DCF80030236007F153
:1001C00048016846C7F844A023F0B4FA07F1400399
:1001D0000CCB07F12C014846FCF796FF0446B86BA0
:1001E000564650B1C389A3F500739BB2C381C3893E
:1001F00003F4F0530BB91CF07DF807F1180016F06A
:1002000097FC07F1400A1CB9D7E906239A4229D383
:10021000786A50B1C389A3F500739BB2C381C389C7
:1002200003F4F0530BB91CF065F85DB1EB89A3F54D
:1002300000739BB2EB81EB8903F4F05313B92846AA
:100240001CF058F8002C3DD102201BF0F5FB0025D6
:10025000044628461BF058FC2E49024640461DF035
:10026000B6FD66E707F11801384616F0DBFEBC461E
:10027000BCE80F0007F12C040FC40136DCF8003095
:100280002360502207F1480168467E6423F052FA49
:100290009AE80C0007F12C014846FCF735FF0446AC
:1002A000B86B50B1C389A3F500739BB2C381C389F6
:1002B00003F4F0530BB91CF01DF807F1180016F009
:1002C00037FCA0E767214046FFF7D2FE00B30021CC
:1002D00020461DF07DFA00221049064620461DF0FA
:1002E000AFFD1EF013F9054630461CF0DBFC05445B
:1002F000002EAED0F389A3F500739BB2F381F3898E
:1003000003F4F053002BA4D130461BF0F3FFA0E719
:1003100005469EE7CE45050056670500D845050011
:1003200038B5FFF7E7FE054620B11BF0CBFD80F0A6
:100330000100C0B200F001045DB1EB89A3F50073C8
:100340009BB2EB81EB8903F4F05313B928461BF001
:10035000D1FF204638BD00000149002012F0FABD4F
:100360001E67050038B50546FFF7F6FF044610B1D5
:100370002946FDF7CDF9204638BD00002DE9FF41A3
:100380008046FFF7E9FF044600284CD048F20801F8
:1003900027481BF000FC48F20801029025481BF09A
:1003A000FAFB0390029818B1224623491DF0EEFC97
:1003B000039818B1224620491DF0E8FC1F4D2E8AF3
:1003C00002AFB6B2B8F1000F14D00223009300239D
:1003D000019722461946404618F0B2FB50B1C38936
:1003E000A3F500739BB2C381C38903F4F0530BB927
:1003F0001BF080FF394602202E821DF067F815F0B1
:100400000FFE054678B101462046FDF781F9EB89DC
:10041000A3F500739BB2EB81EB8903F4F05313B99E
:1004200028461BF067FF204604B0BDE8F08100BFFE
:1004300051D6020011D70200C23F0500582D0020FE
:1004400070B50646FDF70EF8044638B1F38903F59A
:1004500000739BB2F3813446204670BD30461BF0DA
:1004600074FD40B9FFF778FF04460028F4D0314608
:10047000FDF7EEF8F0E722460F4930461DF0E0FCAC
:1004800005461BF07AFD98B12846FFF777FF044632
:100490005DB1EB89A3F500739BB2EB81EB8903F4AB
:1004A000F05313B928461BF025FF002CD4D1D9E70F
:1004B000002DD7D00446ECE7266705002DE9F04370
:1004C00085B001230192074688461046914901AA4A
:1004D00010F0CCFD0022904901981DF0B1FC0022E3
:1004E00005468E4901981DF0ABFC0446002D60D0F6
:1004F00000285ED000228A4928461DF0A1FC039006
:10050000002849D01CF0CEFB002845D0844928465D
:100510001EF0CEF800228349204617F075FC0646EF
:100520001BF02BFD88B103AB01222146304612F0AF
:100530003FFC50B1C389A3F500739BB2C381C3894B
:1005400003F4F0530BB91BF0D5FE5EB1F389A3F5AC
:1005500000739BB2F381F38903F4F05313B930466F
:100560001BF0C8FE0022704901981DF069FC064688
:100570001DF036F9814603981CF094FBF389A3F52E
:1005800000739BB2F381F389484403F4F053306065
:1005900013B930461BF0AEFE039850B1C389A3F5E2
:1005A00000739BB2C381C38903F4F0530BB91BF0F2
:1005B000A1FE00225D4901981DF042FC1EF00DF9DC
:1005C000002800F08780002C57D059492046FEF7BC
:1005D00069FA58492046FEF765FA00225349204639
:1005E00017F012FC06461BF0C8FC88B100231A461F
:1005F0002146304612F0DCFB50B1C389A3F50073ED
:100600009BB2C381C38903F4F0530BB91BF072FE94
:100610005EB1F389A3F500739BB2F381F38903F410
:10062000F05313B930461BF065FE002241492046C5
:1006300017F0EAFB06461BF0A0FC88B100231A461F
:100640002146304612F0B4FB50B1C389A3F50073C4
:100650009BB2C381C38903F4F0530BB91BF04AFE6C
:100660005EB1F389A3F500739BB2F381F38903F4C0
:10067000F05313B930461BF03DFE5DB32D492846BB
:10068000FEF710FA00222B49284617F0BDFB06465C
:100690001BF073FC88B100231A462946304612F03D
:1006A00087FB50B1C389A3F500739BB2C381C38993
:1006B00003F4F0530BB91BF01DFE5EB1F389A3F5F3
:1006C00000739BB2F381F38903F4F05313B93046FE
:1006D0001BF010FE214628461CF076FFD8F800409B
:1006E00024B1E38903F500739BB2E38121463846C8
:1006F0001DF020FF5CB1E389A3F500739BB2E38199
:10070000E38903F4F05313B920461BF0F3FD05B061
:10071000BDE8F083C65C050056670500D25C0500A5
:10072000F7390500DE5C0500E45C0500CC660500D9
:1007300092600500ED5C0500044B0549002814BFDC
:100740000322002258681DF07BBB00BF582D0020FB
:100750006E6905002DE9F341074600208846FFF742
:10076000EBFF044688B1014601A816F05EF9019836
:1007700070B9E389A3F500739BB2E381E38903F4C5
:10078000F05313B920461BF0B5FD02B0BDE8F0816F
:100790001CF0F6FF0022414606461DF051FBB84210
:1007A000054604D1324601A92046FFF787FE2846B8
:1007B00031461CF009FF01A816F022F9D7E7000026
:1007C00010B504461BF0C1FB28B120460249BDE824
:1007D0001040FFF7BFBF10BD5667050010B50446B7
:1007E0001BF0B3FB28B120460249BDE81040FFF7DB
:1007F000B1BF10BDD25C05002DE9F74F0E4615467E
:100800008046002800F0E080002900F0DD8070497B
:10081000002012F09FFB04460120FFF78DFF824667
:1008200000201BF071F98346002C00F0AF80BAF174
:10083000000F00F0AB80002800F0A880002265497E
:10084000404617F0E1FA002200906349304617F065
:10085000DBFA019000981BF090FB002800F0B280BA
:1008600001981BF08AFB8146002800F0A6802846EC
:100870001BF06BFB0746002800F0988000225749C8
:1008800028461DF0DDFA814698B1024654492046BB
:100890001DF07CFAB9F80E30A3F500739BB2A9F8ED
:1008A0000E30B9F80E3003F4F05313B948461BF07C
:1008B00021FD00224B4928461DF0C2FA00286DD0C8
:1008C0001DF08BFF81462846002247491DF0B8FAEB
:1008D000054600286FD01BF060FB002860D028463A
:1008E0001CF07EFF00285BDD28461CF079FF0746E0
:1008F000EB89A3F500739BB2EB81EB8903F4F05312
:1009000013B928461BF0F6FC4FF40043374A384928
:100910004046FEF73FF80823364A37493046FEF78F
:1009200039F84FF40043354A31493046FEF732F882
:1009300038461BF0E9F82C49024620461DF047FADC
:1009400048461BF0D9F82749024620461DF03FFAD9
:100950002B4A594620461DF09FFA2A4A0546414631
:1009600020461DF099FA284A0746314620461DF0D8
:1009700093FA3946024628461CF0FAFD21465046B5
:100980001DF0C6F8DDE900011CF01EFE5A462146A6
:10099000504603B0BDE8F04F1CF0EABDB94692E7FF
:1009A0001A49032017F034F84027A1E71DB1184970
:1009B000032017F02DF84027A6E71649012017F06D
:1009C00027F8DFE71449F9E703B0BDE8F08F00BF6F
:1009D000F46405003B600500DE5C0500C95C0500B1
:1009E000C65C0500CC660500F9640500C10703007C
:1009F000ED5C05001D0A030092600500DD070300A1
:100A0000E45C050056670500D25C0500036505003F
:100A1000246505004E650500A96505002DE9F7432D
:100A200007461BF092FAD0B10020FFF785FE04467E
:100A3000A8B1014601A815F0F8FFDFF85C80DFF8E7
:100A40005C90019870B9E389A3F500739BB2E381D0
:100A5000E38903F4F05313B920461BF04BFC03B0B9
:100A6000BDE8F0831CF08CFE0022414606461DF0D6
:100A7000E7F98742054607D100201BF03DF84946BB
:100A8000024630461DF0A3F9284631461CF09CFD75
:100A900001A815F0B5FFD4E7D25C0500FE6505009E
:100AA0002DE9F04F91B004468A4691461E461A9FA2
:100AB0001BF029FB88B1204619F054FB0022804628
:100AC000214605A818F0B7FDDFF818B205A815F003
:100AD0005CFF28BB05A815F019FFBAF1000F00F064
:100AE000AD8000200CF02AFE804620461BF02DFA37
:100AF000002852D000227B4920461DF0A1F91CF0AD
:100B000043FE824600284ED120461BF01EFA0028E4
:100B100040F0B78020460CF0A9FE3A46314657E037
:100B200005A815F0C0FE0546B8F1000F18D1002247
:100B3000114628461DF092FB1EF0DBFAD0B95DB1DC
:100B4000EB89A3F500739BB2EB81EB8903F4F053BF
:100B500013B928461BF0CEFB05A816F049F8B5E7F7
:100B6000C0470028E3D0594628461BF077FE0028EE
:100B7000DDD1E4E7014603903846B047039BDA89AC
:100B8000A2F5007292B2DA81DA8902F4F052002AF8
:100B9000D5D118461BF0AEFBD1E720461BF0CDF9AE
:100BA0000028A7D1B0E70CF0C9FDBAF80E30A3F5C4
:100BB00000739BB2AAF80E30BAF80E3003F4F0536B
:100BC000054613B950461BF095FB3A463146284678
:100BD000FBF7F7F9B9F1000F22D020461BF0B5F969
:100BE000002855D00022404920461DF029F905462D
:100BF0001BF0ABF9002851D0012200973346114673
:100C00002846FFF74DFF5DB1EB89A3F500739BB25A
:100C1000EB81EB8903F4F05313B928461BF06AFB10
:100C200020461BF08AF9002848D030481CF066FBAB
:100C3000054601463846B047002D45D120461BF0F9
:100C400035FBD8B10025E9B205A810F0D3FA05A804
:100C50001CF054FB044601463846B0475CB1E389BA
:100C6000A3F500739BB2E381E38903F4F05313B956
:100C700020461BF03FFB0135202DE4D111B0BDE82B
:100C8000F08F20461BF012FB00287FF443AFA1E752
:100C900020461BF072F90028A4D1A8E720460CF0EA
:100CA0004DFD3A4681463146FBF78BF9C845AAD03F
:100CB0003A4631464046FBF784F9A4E720461BF04C
:100CC000F7F90028B1D1B9E7EB89A3F500739BB21E
:100CD000EB81EB8903F4F053002BAFD128461BF0D6
:100CE00009FBABE7316E0500AA390500B06B0500C2
:100CF0002DE9F04F8FB015461E46824689460146C3
:100D0000684615F092FE894A3146284616F08AFC5C
:100D10004FF001080024009F9FB92846844A3146BD
:100D200016F080FC50461BF0DEF800285BD0814AAC
:100D30003146284616F076FC002C60D10FB0BDE895
:100D4000F08FFB8903F500739BB2FB8138461BF0E3
:100D500003FA48B3B8F1000F04D1774A3146284668
:100D600016F060FC6FF00042012138461BF092FE45
:100D7000724A804603463146284616F053FCB8F1C5
:100D8000000F20D0B8F80E30A3F500739BB2A8F87E
:100D90000E30B8F80E3013F4F05B02D140461BF071
:100DA000A9FA4FF000080EE038461BF081F950B167
:100DB000634938461BF052FD28B1009C1CB1204607
:100DC0001CF0DEFC0446FB89A3F500739BB2FB819B
:100DD000FB8903F4F05313B938461BF08BFA6846CD
:100DE00015F00EFE97E7002C00F0998019F008022C
:100DF00013D0544B544A3146284616F013FCE3896D
:100E0000A3F500739BB2E381E38903F4F053002B55
:100E100094D120461BF06EFA90E7214606A816F002
:100E200003FADDE9063293423BD3099850B1C389F6
:100E3000A3F500739BB2C381C38903F4F0530BB9CC
:100E40001BF058FA41484FF0FF383146A84750464A
:100E50001BF08AF810B131463D48A84701A800228E
:100E6000214616F0E1F9DFF8FCA000208146DDE91B
:100E70000132934235D3049850B1C389A3F500736E
:100E80009BB2C381C38903F4F0530BB91BF032FA50
:100E9000304B3148314630EA280028BF1846A84771
:100EA000ADE70A9ACAB1D25C0A2A16D1089A099803
:100EB00003EB020850B1C389A3F500739BB2C38151
:100EC000C38903F4F0530BB91BF014FA1F48234BEA
:100ED00010EA280038BF1846B7E706A815F028FE24
